:020000040800F2
:1000000000800010A56300085570000859700008B2
:100010005D70000861700008657000080000000055
:1000200000000000000000000000000069700008EF
:100030006D7000080000000071700008DD08000805
:10004000DB080008476800084F690008F7690008E6
:10005000036B0008776B0008736C0008876C00085E
:1000600075700008DB6D0008876E00089D3300087E
:10007000A9330008B5330008C1330008CD330008A8
:10008000D9330008E53300081F6F00085F6F0008D0
:10009000B36F000853700008577000087D700008A7
:1000A0005B7000085F7000086370000867700008EC
:1000B0006B7000086F700008737000087B70000898
:1000C00083700008077200085F7200087B720008E6
:1000D000AB720008F1330008FD330008AF78000868
:1000E00027790008077A00080F7A0008277A0008A5
:1000F0002B7A00082F7A0008BF8500089B8600082D
:100100000B880008CF890008FB890008FF8A0008D7
:100110006F8B0008BB8B00085F8C0008038F000802
:100120004F8F0008778F00082F9000089F900008DD
:100130001F910008BB910008EB9100081B9200087A
:100140003B9200089B980008379B000800000000C5
:10015000000000000000000000000000000000009F
:100160000000000000000000000000005B9B000891
:10017000879B00089F9B00083F9D00082B9E00085E
:1001800023A00008CFA000087BA100083BA2000824
:1001900067A20008000000007BA2000863A300081B
:1001A00077A300087BA9000873AC00089FAC000887
:1001B000CBAC000853AE0008A3AE0008CBAE0008DD
:1001C0004BB100088FB1000867B20008A3B4000863
:0801D00067B5000817B600082E
:1001D80084B041F24870C1F20000006845F2ED5168
:1001E800CAF6CE4188420BD141F248710020C1F2D3
:1001F800000108604EF29E60C0F600000BF09DFA08
:1002080003F0BEF902F0C4FF41F28070C1F20000B1
:1002180000684DF68361C4F21B31A0FB01014BF667
:10022800AA60890CC0F600000EF0FCF802F038FE57
:1002380006F08AFB02F0E8FA02F04CFB02F098FBA9
:1002480006F0ACFA06F0FCFA02F0DEFD02F002FE5F
:1002580006F054FC02F0D0FE06F07EFE03F0EAF849
:1002680003F02CF903F072F902F094FD06F054FE45
:1002780002F076FF4EF27C60C0F600000BF05DFAEB
:100288000CF0FAFF05F0BAFF0BF0ACFE05F034FEF7
:10029800032818D8DFE800F00209100240F2000035
:1002A800C1F200000BF010FF0DE040F20000C1F2B7
:1002B80000000BF0C7FF06E040F20000C1F20000AA
:1002C80000210CF0CFF841F2902040F2000AC1F270
:1002D8000000C1F2000A04F0D3F84FF090404FF448
:1002E800806109F025FCB0B9322003F087F94FF09E
:1002F80090404FF4806109F01BFC60B94EF28B60AE
:10030800C0F600000BF019FA40F20000C1F200003C
:1003180001210CF0A7F841F29026C1F20006304600
:1003280004F0AEF806F024FC40F20007DAF81010EA
:10033800BAF81420BAF8163040F68C25C2F2000735
:10034800C1F20005384600950CF0E8FA304604F092
:1003580097F801F065F940F664540025C1F20004ED
:10036800C4F27F052046294608F026F940F6F840F1
:10037800C1F20000294608F01FF940F68C40C1F28E
:1003880000007F2108F018F940F62040C1F2000073
:10039800294608F011F940F6B430C1F200007F2177
:1003A80008F00AF9304604F06BF840F23421C2F242
:1003B80000012046402208F06DF9002840F08782AD
:1003C80040F68C4040F23431C1F20000C2F2000124
:1003D800032203F02FF9002840F0798240F62040EC
:1003E80040F24031C1F20000C2F20001012203F0E4
:1003F80021F9002840F06B8240F6B43040F24431D5
:10040800C1F20000C2F20001042203F013F900282F
:1004180040F05D8241F29024C1F20004204604F0CD
:100428002FF805F03BFA204604F02AF84DF6BF00F5
:10043800C0F600000BF081F90CF0E2FBBAF81800E6
:1004480018B341F290240025C1F200044FF0904007
:100458002021012203F084FD4FF4AF7003F0CEF8A1
:10046800204604F00DF84FF090402021002203F0C0
:1004780077FD4FF4AF7003F0C1F8204604F000F8A0
:10048800BAF8180001358542E0D341F2C0259FED46
:10049800DC8B9FEDDD9B9FEDDEABC1F200050020FC
:1004A80000264FF0000B039008E000BF40F6203014
:1004B800C1F200002221C0F88C10464641F290207B
:1004C800C1F2000003F0DCFF2868012834D140F2B3
:1004D8003424C2F20004B4F8FE0001F019F8B4F8AC
:1004E800FC0001F08DFB01F073FADAF8D800DAF8B5
:1004F800E4104FF47A7281FB000100230DF050FAEA
:10050800CAF80801DAF8D800DAF890114FF47A72CC
:1005180081FB000100230DF043FACAF88401002092
:10052800286040F66450C1F200002146402208F0DD
:10053800B1F8002840F0CB8141F2BC20C1F20000A4
:100548000068012806D140F23430C2F20000006889
:1005580001F0D2FC41F2B820C1F200000068012885
:1005680006D140F24030C2F20000006801F018FDE8
:1005780041F2B420C1F200000068012845D140F2E0
:100588004439C2F20009D9F8000001F099F8D9F805
:10059800040001F085FBD9F8080006F039F858EC9A
:1005A800187B3A46434605F011FF55EC194B224695
:1005B8002B4605F00BFFCDF808B0D346019656EC54
:1005C8001AAB5246334605F001FF0DF07BF9ABF844
:1005D8005001D9F80C0006F01BF83A46434605F0DE
:1005E800F5FE22462B4605F0F1FE5246DA46DDF8C6
:1005F80008B040F200073346019EC2F2000705F03A
:10060800E5FE0DF05FF9AAF8520141F2B020C1F2FF
:100618000000006801280BD105F0FEFB01F018F975
:10062800AAF8980141F2B020C1F20000002101604F
:1006380002F0DEFF841B804618BF0124BAF854017B
:10064800BBF1000F4FF00005C8BF012504281BD3DC
:100658004DF61610C0F600000BF06FF840F2004699
:10066800C4F600064FF0070930464FF40061002237
:10067800AAF8069103F074FC30464FF4805100222A
:10068800AAF8069103F06CFC41F24420C1F2000084
:10069800006801684068039801F00F0686422ED072
:1006A800DAF828010130CAF82801DAF82401013003
:1006B800CAF82401DAF820010130CAF8200141F211
:1006C800AC20C1F20000006820B94FF09040102122
:1006D80009F040FA00F0F8FB01F08EFC0CF0A2FAE9
:1006E8000CF068FB0CF0A6FD02F094FD01F06CFB29
:1006F800AAF89C0101F080F8AAF816010396BAF846
:100708001A00002800F08F8097F82600002840F093
:100718008A80BAF81A0040F2F13188420DDC0138BB
:100728000A2821D8DFE800F0063A3E3320D25343A6
:1007380037475F005046002170E0B0F57D7F1ADB37
:1007480058D040F2D241884266D041F25251884294
:100758000AD141F2487045F2ED51C1F20000CAF6E3
:10076800CE41016003F0B6F84EF6AC50C0F600007A
:100778000AF0E3FF54E040F2F231884236D040F20A
:10078800F3318842F0D1012006F07AFA48E0504669
:100798000BF058FD44E005F065F841E050460BF0D9
:1007A80093FC3DE0504601210BF05CFE38E05046DA
:1007B8000BF0F0FB34E0504600F08EF840F23420A5
:1007C800C2F20000B0F8FC0001F0CAF928E0504677
:1007D8000BF0C0FB40F23420C2F20000B0F8FC007D
:1007E8000CF064F81CE000F023F919E0002006F092
:1007F80047FA15E006F0EEFA12E000BF00BF00BFAE
:10080800000000000070A740000000000000354014
:10081800000000000000F03E504601210BF01EFFD2
:100828000020AAF81A0004EA0500ABEB000B4FF011
:1008380090404FF4806109F07BF998B941F2C025E6
:10084800BBF1000FC1F2000524D10A2002F0D6FE48
:100858004FF090404FF4806109F06AF938B14FF0D9
:10086800000B17E041F2C025C1F2000512E041F289
:10087800AC21C1F20001086810B10020086007E04F
:10088800012008604FF090401021012203F068FB1E
:100898004FF4FA7B384605F02FFC002846463FF413
:1008A8000DAE38460CF0C4F802287FF4FFAD41F2D3
:1008B800AC20C1F200000068464600287FF4FEAD77
:1008C80038460CF001F94646F8E500BFFEE706F0A9
:0208D800CDF958
:0208DA00FEE737
:0408DC0006F0C0BCA6
:1008E0002DE9F04704464CF60A30C0F600000DF042
:1008F0009DFDD4F89C00002800F08780D4F89C006F
:100900000DF020F89FED460B5AEC105B2A4653463B
:100910000CF0DEFE40F2E042C1F2000292ED000B6C
:1009200056EC107B3A4633460CF0D2FE9FED3E0B60
:1009300058EC109B4A46434605F04CFD05F05AFE24
:10094000C4F89400B4F8CE003A46A4F89800B4F87D
:10095000CC003346A4F89A004EF67330C0F600007F
:100960000DF064FDD4F89C000CF0ECFF2A465346D1
:100970000CF0AEFE02464EF65B00C0F600000B46E1
:100980000DF054FDB4F998000CF0DCFF9FED280B3E
:1009900055EC106B32462B460CF09AFE02464EF692
:1009A0006A00C0F600000B460DF040FDB4F99A0055
:1009B0000CF0C8FF32462B460CF08AFE02464CF67D
:1009C0004E30C0F600000B460DF030FDD4F8940018
:1009D00005F022FE4A46434605F0FCFC02464EF670
:1009E000B060C0F600000B460DF020FD4CF6F23072
:1009F000C0F600000DF01AFD40F20000C1F2000048
:100A00000021BDE8F0470BF02DBE4EF69030C0F649
:100A10000000BDE8F0470AF094BE00BF00BF00BF71
:100A20000000000000408F400000000080842E4144
:080A3000000000000000594025
:100A38002DE9F04F81B04EF67500C0F600000DF0BC
:100A4800F1FC40F2000AC1F2000ABAF8CE00AAF896
:100A5800A000BAF9A0000CF071FF9FED490B54EC0F
:100A6800109B4A46234600940CF02EFE02464EF692
:100A78008C00C0F600000B460DF0D4FCBAF9CE008D
:100A8800BAF99810401A0CF059FF4A46234607460F
:100A98008B460CF019FE02464CF61E40C0F60000CC
:100AA8000B460DF0BFFC40F2D040C1F2000090EDC3
:100AB800000B4EF69B0056EC104BC0F60000224689
:100AC80033460DF0AFFCDAF89C000CF037FF9FEDD1
:100AD8002E0B55EC108B42462B460CF0F5FD0246CA
:100AE8004CF6B250C0F600000B460DF09BFCDAF84D
:100AF8009C000CF023FF42462B460CF0E5FD2246F5
:100B080033460CF0E1FD9FED220B53EC102B0CF05B
:100B1800BBFC3A465B460CF0D7FD9FED1F0B54EC2F
:100B2800105B2A46234605F051FC0CF0CBFECAF8B0
:100B3800A400DAF8A4000CF001FF2A4623460CF0C2
:100B4800C3FD009B4A4605F041FC9FED150B53EC95
:100B5800102B0CF099FC02464EF6CE00C0F60000B1
:100B68000B460DF05FFC4EF6C460C0F600000DF0B9
:100B780059FC5046002101B0BDE8F04F0BF06EBDA6
:100B880000000000000059400000000000408F40B5
:100B9800000000000000F0BF0000000065CDCD415E
:080BA800000000000000F03F16
:100BB0002DE9F04F87B04EF61240049041F26C20C0
:100BC00004AD0024C1F2000029460222CDE905440B
:100BD00007F0CEFF8DF812008DF80C40CDE90144EE
:100BE00040F6D05001AC4FF47A77C1F200002946AC
:100BF00022460923009704F005F89DF8040040F20E
:100C0000000AFF28C1F2000A34D19DF805009DF8C2
:100C1000101088422ED19DF806009DF811108842D0
:100C200028D19DF807009DF81210884222D141F288
:100C30006C209DF80C50211DC1F20000042207F029
:100C400097FFA84216D19DF8080000F0CC00842838
:100C500010D19DF909109DF80B209DF80A00CBB228
:100C600042EA034242EA002000F17F42002948BFE5
:100C7000501C07E0BAF882010130AAF8820104F0A2
:100C800011FE002041F2143BC1F2000BDBF8001012
:100C90006FF0004291421CBF0131CBF8001041F2CD
:100CA0001831C1F200010A6802EBD2731044A0EBC4
:100CB0006300086000EBD0704110CAF88811DAF8C0
:100CC0007810C1EB600441F2DC20C1F20000046046
:100CD000DAF8D400DAF88010DAF88820401A5043A5
:100CE0000CF030FE9FED680B58EC109B4A464346D3
:100CF0000CF0EEFC0CF0EAFDCAF88C01251A41F26A
:100D0000E420C1F200000560BAF9CC00BAF97E1007
:100D1000401A0CF017FE0446DAF890000E460CF06C
:100D200011FE2246334605F055FB4A4643460CF079
:100D3000CFFC0CF0CBFD41F2E021281AC1F20001FA
:100D400008600CF0FFFD9FED520B53EC102B05F0EB
:100D500041FB9FED510B53EC102B05F03BFB9FED3E
:100D6000500B53EC102B05F035FB064641EC100BF5
:100D700040F2E040C1F2000080ED000BDAF8940090
:100D80000F4605F049FC9FED480B53EC102B0CF07F
:100D90009FFC32463B4605F01DFB064641EC100B1E
:100DA00040F2D040C1F2000080ED000B0F46BAF9CE
:100DB000CE00BAF99810401A0CF0C4FD0446DAF8D7
:100DC000A4000D460CF0BEFD9FED390B53EC102B2B
:100DD0000CF07EFC22462B4605F0FCFA9FED360B0C
:100DE00053EC102B0CF054FB02460B4630463946B0
:100DF00005F0F0FA044641EC100B40F2D8409FEDAC
:100E0000301BC1F200000E4680ED000B51EC110BBF
:100E10009FED2D0BC80F314660F3DF7153EC102BA3
:100E2000204605F06FFB10B1DAF8900107E020468C
:100E300031464A46434605F0CDFA0CF047FDCAF864
:100E4000E400DBF80000152813DBDAF8E400DAF838
:100E5000E8108842C4BFDAF8E400CAF8E800DAF81B
:100E6000E400DAF8EC108842BCBFDAF8E400CAF813
:100E7000EC0041F2B020C1F200000121016007B096
:100E8000BDE8F08F00BF00BF0000000000408F40B1
:100E90000000000000000840000000000000494081
:100EA000000000000000803E0000000080842E4111
:100EB0000000000065CDCD41000000000000F03FC3
:100EC0000000000000000000000000000020614061
:100ED0002DE9F04F81B02DED028B86B040F2000578
:100EE00040F2F84BC1F20005C1F2000BD5F85CA04E
:100EF000DBE900014EF680620843C0F2360205D1FC
:100F0000D5F82C0100215043CBE9000140F20056F6
:100F1000C1F20006D6E90001084305D1D5F8300139
:100F200000215043C6E90001D5F8E400B5F970107E
:100F3000B0EB010829D4B5F8520005F06DFB9FED28
:100F4000C80B59EC106B32464B460CF0C1FB074600
:100F500040460C4605F060FB02460B4638462146EB
:100F600005F038FA0446B5F9D6010F460CF0EAFC54
:100F7000324640F200564B46C1F200060CF0A8FB88
:100F800002460B462046394642E0E86DB5F8681047
:100F9000B0FBF1F77842804580F2668240460CF063
:100FA000D1FC044641EC180B3846D1468A460CF079
:100FB000C9FC8DED048B9DF81730024683F080004C
:100FC0008DF81700DDE904030F4619463B460CF087
:100FD0007FFB41EC180BB5F8500005F01DFB9FEDB1
:100FE000A20B53EC102B0CF073FB9FEDA10B53ECF9
:100FF000102B0CF04DFA41EC110BB0EE480AF0EE5C
:10100000680A0DF073F951EC100B22465346CA469C
:1010100005F0E0F90CF05AFCC5F8F000D5F8E40052
:10102000B0F1FF3F11DDD6E900014EF6806210EB12
:10103000080041EBE871C0F236020023C6E9000166
:101040000CF0E2FCC5F830011BE0DBE90001C8F15F
:101050000002801841EBE2714EF68062C0F2360267
:101060000023CBE900010CF0CFFCC5F82C01D5F82A
:101070002C014FF47A71EA6D4843B0FBF2F0A5F809
:101080003C01D5F8F000D5E93E120023091842EBE7
:10109000E070C5E93E10D5F8F000D5E958124FF4DC
:1010A0006164091842EBE070C5E95810D5E95801B0
:1010B0004FF461620CF078FCC5F84001D5F80001EE
:1010C00041F2A4290028C1F2000902DCD9F800008D
:1010D00080B1D5E970014FF4616210EB080041EB7B
:1010E000E871C5E97001D5E9700100230CF05CFCE2
:1010F000C5F8C801D5F8E400D5E97812002309182D
:1011000042EBE070C5E97810D5E978014FF46162EF
:10111000AAFB04470CF048FCC5F8D801D5F8D80163
:1011200000284FF47A7006D0D5F84011D5F8D821B0
:10113000484390FBF2F0A5F8D601D5E93E01201A0C
:1011400077EB0100B8BFC5E93E47D5E95801013842
:1011500071F1000008DB0020C5E95800C5F8400126
:10116000C5E97800C5F8D801E86DB5F85410D5F890
:10117000D820B5F8583041F234369A42C1F2000610
:101180001CDD484305F048FA9FEDE10B53EC102BB2
:101190000CF09EFA05F0EEF9D5F8E420D317101AFA
:1011A00073EB01000ADA308801303080B5F8561050
:1011B00000B2884204DDB5F8560000E0002030801F
:1011C000B6F90000B5F8561088425CDB0020C5E98E
:1011D0003E47C5E95800C5F840010CF0CBF8D9F8F6
:1011E0000000002804BF0120C9F8000041F2A82037
:1011F000C1F20000016801293ED100210160D5F84B
:10120000E8014EF68064D5E97023C0F23604A0FBF5
:1012100004010CF0C9FBA5F84401D5F8EC01D5E9AF
:101220006E23A0FB04010CF0BFFBA5F84601D5F826
:101230002811D5F8C821D5F82431B5F94401B5F9FC
:101240004671D5F8D860D5F8E440CDE900074EF6F0
:101250000470C0F60000029603940DF0E7F812E067
:101260000000000000408F400000000000005940D6
:10127000000000000000F0BF0020C5E97000C5F8C4
:10128000C801C5E96E00D5E93E014FF46162002353
:101290000CF08AFBC5F8F400B5F8B800002859D066
:1012A000B5F85001B0F57A7F40F2BD80B5F8520133
:1012B000C0087C2800F2B78041F23230C1F2000051
:1012C000018801318AB20A2A0180C0F0B280D9F8BF
:1012D00000100A220129028040F09380D5F82001F5
:1012E000B0F5616FC0F08D80D5F8200142F6007135
:1012F000C0F20D01884200F2848004F093FD0CF0EE
:1013000023F84FF2F014D5E97001CFF6FF742246AE
:101310004FF0FF330CF048FBC5F8E801D5E96E014A
:1013200022464FF0FF330CF03FFBC5F8EC01D5F837
:101330002811D5F80C21D5F8E831D5F82001D5F8D9
:10134000D870D5F8E460CDE900074EF66A10C0F613
:10135000000053E0D5F8D800B5F88011884262DA71
:10136000D5F8D800B0F57A7F5DDD41F23230C1F2B8
:101370000000018801318AB20A2A018059D3D9F8C4
:1013800000100A22012902803BD1D5F82001B0F5D6
:10139000966F36D3D5F820014FF68041C0F20A018E
:1013A00088422ED804F03EFD0BF0CEFF4FF2F01431
:1013B000D5E97001CFF6FF7422464FF0FF330CF0F1
:1013C000F3FAC5F8E801D5E96E0122464FF0FF3384
:1013D0000CF0EAFAC5F8EC01D5F82811D5F80C2183
:1013E000D5F8E831D5F82001D5F8D870D5F8E46003
:1013F000CDE900074EF62710C0F6000002960DF06A
:1014000015F841F2A8210020C1F200010122C5F81F
:101410002401C9F800000A60C5E97000C5F8C801D8
:10142000C5E96E0005E041F23230C1F20000002152
:101430000180B5F8640048F2A0640428C0F20104F9
:1014400020D8DFE800F0031C16191300EA6DD5E977
:101450003E014FF46167A0FB040301FB0431A2FBD2
:1014600007230CF0A1FA0EE04046D5E504F048FF52
:1014700009E004F0F7FE06E004F00EFF03E004F0DC
:10148000DFFC00E00020C5F80001EA6DD5E93E016F
:101490004FF46167A0FB040301FB0431A2FB0723A7
:1014A0000CF082FA48F21F54C5F2EB1450FB04F022
:1014B000410901EBD070A5F8CC0104F0C1FC50FB50
:1014C00004F0410901EBD070A5F8CE0104F0CAFE8A
:1014D00050FB04F0410901EBD070A5F8D00104F0F5
:1014E000DBFE50FB04F0410901EBD070A5F8D201FE
:1014F00004F006FF50FB04F0410901EBD070A5F8A1
:10150000D40106B0BDEC028B01B0BDE8F08F00BF86
:0815100000000000000059403A
:101518002DE9F04F81B041F20C33C1F20003196894
:101528006FF00042914280461CBF481C186041F28F
:101538001030C1F200000168A1EB51114144016073
:1015480048F20000CFF6FF7000EB51100CF0F6F9EE
:101558009FED2B0B59EC10AB52464B4604F036FF6F
:101568009FED290B5BEC104B22465B4604F02EFFE7
:101578009FED270B55EC106B32462B4604F026FFE7
:101588000CF0A0F940F20007C1F20007C7F8D80034
:1015980041F20C30C1F200000068B0F5A07F13DD05
:1015A800D7F8D800D7F8DC108842C4BFD7F8D800DD
:1015B800C7F8DC00D7F8D800D7F8E0108842BCBFDD
:1015C800D7F8D800C7F8E00040460CF0B7F99FED0F
:1015D800120B53EC102B0BF057FF52464B4604F0FE
:1015E800F5FE22465B4604F0F1FE32462B4604F037
:1015F800EDFE0CF067F9C7F8940101B0BDE8F08F73
:10160800000000000070A740000000000000184023
:10161800000000000000003F000000000000E0C0E3
:1016280080B547F2A850C1F6FF7001889FED221AD5
:1016380000EE101AB8EE400A9FED202A20EE010AAB
:1016480020EE020A41F2D421408CBCEEC00AC1F25D
:10165800000181ED000A10EE101A00EE100AB8EE33
:10166800400A20EE010A20EE020A41F2D820BCEE20
:10167800C00AC1F2000080ED000A10EE100A401AFC
:1016880041F2D021C1F20001086004F0C1FF9FEDD2
:10169800080B53EC102B0CF017F841EC100B40F230
:1016A800C840C1F2000080ED000B80BD00BF00BF44
:1016B800000000000000544000803B4500008039D5
:1016C800B0B540F6B8314843000C04F0A1FF044619
:1016D80041F2D420C1F2000000680D4604F098FFE2
:1016E80002460B462046294604F06CFE40F2C842EA
:1016F800C1F2000292ED000B53EC102B0BF0E4FF4B
:101708009FED0B0B53EC102B0BF0BEFE9FED0A0B5D
:1017180053EC102B04F05AFE0CF0D4F840F2000100
:10172800C1F20001A1F8CC00BDE8B04004F0B8BB9C
:101738000000000000003E4000000000000059408A
:10174800004B000000000100010000000000000044
:101758000000000000000000000000000000000081
:101768000000000000000000000000000000000071
:1017780090D00300000000000000000000000000FE
:1017880040420F000000000040420F00000000002F
:101798000000000000000000FFFFFFFFFFFFFFFF49
:1017A80000D68AEAFFFFFFFF007884C9FDFFFFFF2C
:1017B800DE0369000071020000401F000A000200F9
:1017C800B036703001000200E02ED430D039B03687
:1017D80083FF7D0070177C153CF630F870177C1578
:1017E80054F248F4320038FF102707008403010040
:0817F80001002035640000002F
:10180000B0B540F20005C1F20005B5F83C01C8B121
:10181000D5F8340104F000FF0446D5F838010D4630
:1018200004F0FAFE02460B46204629460BF050FF14
:101830009FED070B53EC102B04F0CCFD0CF046F899
:1018400000B2B0BD4FF6FF7000B2B0BD00BF00BF28
:081850000000000000005940F7
:101858002DE9F04740F2000941F20838C1F20009C9
:10186800C1F20008D9F82801D8F8001040F6E40AB7
:10187800401AC1F2000AA9F89A010AF10400514677
:10188800FC220CF091FC40F2E475C1F20005281D21
:101898002946FC220CF088FCD9F8E4000022CAF89A
:1018A8000000D9F8D800002128606FF0004000231C
:1018B8006FF000465AF82240002C48BF6442B442F8
:1018C80038BF264655F822709C4288BF2346002F11
:1018D80048BF7F42874238BF38468F4202F1010233
:1018E80088BF3946402AE5D19D1B48BF6D42081A7A
:1018F80048BF4042D9F85C10B9F86820B1FBF2F152
:1019080046F26762C6F2666251FB02F1CA1002EB48
:10191800D1718D4205DA6FF00100013000B2BDE8E7
:10192800F087192804D24FF6FE7000B2BDE8F087A0
:1019380000234FF0FF314FF0FF3200BF0AEB83075F
:101948007F685AF82360BF1B48BF7F429742C8BFD1
:10195800194603F10103C8BF3A463F2BEED12029AF
:101968002ED104F055FE044628460E4604F050FEDB
:1019780002460B46204631460BF0A6FE9FED120BA1
:1019880053EC102B04F022FD0BF09CFFA9F81C016E
:10199800D9F8280140F23422C8F8000009F2F220F0
:1019A8000021C2F2000200BF32F8213002EB8107A9
:1019B80020F8803C7B880131402920F80239F3D196
:1019C800002000B2BDE8F087000000000088C34096
:1019D8002DE9F04140F234276FF000404FF0FF311D
:1019E8000023C2F200074FF0FF36002237F82350D9
:1019F800A84228BF284688BF1E46AA429CBF2A463E
:101A080019460133402BF1D107EB810107EB86031F
:101A180049885B88101AA1EB03080BF08FFF9FED34
:101A2800440B53EC102B04F0D1FC0BF04BFF0BF0E4
:101A380085FF40F20005C1F200050446D5F8940080
:101A48000E4604F0E5FD9FED3C0B53EC102B0BF01C
:101A58003BFE2246334604F0B9FC0BF033FF044644
:101A680040460BF06BFF9FED360B53EC102B04F048
:101A7800ADFC9FED350B53EC102B04F0A7FC9FED4C
:101A8800340B53EC102B04F0A1FC0BF01BFFE96D99
:101A9800B5F86820B1FBF2F146F26762C6F26662F9
:101AA80051FB02F18A1002EBD171220048BF624259
:101AB8008A4205DA6FF00100411C08B2BDE8F081E6
:101AC80002004FF6FE7148BF42420A2A2CD30BF09F
:101AD80035FF804620460E460BF030FF02460B4687
:101AE800404631460BF0F0FD9FED1B0B53EC102BDD
:101AF80004F06CFC0BF0E6FEA5F81E01D5F82801F1
:101B0800B81C002130F8022C05EB410382F4004296
:101B1800A3F8F42230F8042B013182F40042402962
:101B2800A3F87423EED1002108B2BDE8F08100BF0C
:101B380000000000804F12400000000080842E4109
:101B4800000000000070A7400000000000001840DE
:101B5800000000000000003F000000000088C340B3
:101B680070B540F20006C1F20006D6F8B010401A6F
:101B7800A0F500400BF0E2FE9FED170B53EC102B85
:101B880004F024FC9FED160B53EC102B04F01EFC04
:101B98009FED150B53EC102B0BF096FD9FED140BDE
:101BA80053EC102B0BF090FD0446D6F89C000D4624
:101BB8000BF0C4FE22462B460BF086FD9FED0E0B64
:101BC80053EC102B04F002FC04F010FDC6F8B4002E
:101BD80070BD00BF00BF00BF000000000070A7403C
:101BE800000000000000003F00000000000044402A
:101BF800FCA9F1D24D62403F0000000080842E41D4
:101C080070B540F20006C1F20006D6F8B010401ACE
:101C1800A0F500400BF092FE9FED170B53EC102B34
:101C280004F0D4FB9FED160B53EC102B04F0CEFB05
:101C38009FED150B53EC102B0BF046FD9FED140B8D
:101C480053EC102B0BF040FD0446D6F8B4000D46BB
:101C580004F0DEFC9FED100B53EC102B0BF034FD61
:101C680022462B4604F0B2FB0BF02CFEC6F890017E
:101C780070BD00BF00BF00BF000000000070A7409B
:101C8800000000000000003F000000000000444089
:101C9800FCA9F1D24D62403F0000000080842E4133
:101CA80010B540F20004C1F2000440F6B831A4F8BF
:101CB800C81004F0ADFC9FED0C0B53EC102B04F096
:101CC80085FB9FED0B0B53EC102B04F07FFB9FED76
:101CD8000A0B53EC102B04F079FB0BF0F3FDA4F87E
:101CE800CA0010BD00BF00BF000000000070A74080
:101CF8000000000000000840000000000000F03E66
:101D080070B50446049816460D4621604A6033B102
:101D1800012B09D14FF480524FF4C06106E04FF413
:101D280080524FF4806101E000210022013818BF81
:101D380001204003C5E902202846296109F024FA58
:101D480038B14EF66240C0F6000009F0F6FC04F027
:101D58008DFF284603F046FCB6F5964F0CD805983B
:101D680004F056FC9FED160B53EC102B04F02EFBE1
:101D780004F03CFC01460BE040F2D6604DF683616E
:101D88007043C4F21B31A0FB0101012000EB91411B
:101D9800284609F037FF28684FF48072016841F03F
:101DA8008061016054F8270B214603F079FB30B1BC
:101DB8004DF2CA00C0F600000CF034FBFEE770BD1F
:081DC8000000000000000C40C7
:101DD000F0B581B040F20004C1F20004B4F858003C
:101DE00004F01AFC9FED420B53EC102B04F0F2FAB6
:101DF0000BF06CFD41F2F425C1F20005B4F8581067
:101E00002E68A4F89E61D4F8D87087420CDC08468E
:101E100004F002FC9FED380B53EC102B04F0DAFABF
:101E20000BF054FD87420CDA41F2EC20C1F20000C5
:101E3000002101606FF001002960013000B201B0A3
:101E4000F0BD41F2EC21C1F200010868002808BF92
:101E50000F60086800F10A02974202DC0A388742E4
:101E600005DA00224FF6FE700A602A60E6E7D4F831
:101E7000E400B4F97020904206DA0020086028607F
:101E80006FF001000138D9E7701C42F63121884219
:101E9000286006D3D4F8E400B4F87010401AA4F80F
:101EA0001801B4F9180101281EDBD4F8280144F206
:101EB0000751CCF22E21A0FB010141F2F020C1F22A
:101EC00000000268090C8A420ED0016041F2F8203D
:101ED000C1F200000168B4F91821A1EB911111447D
:101EE00001608809A4F81A010020A7E700BF00BF1D
:101EF0007B14AE47E17AF03F0AD7A3703D0AEF3F6B
:101F000080B50BF01FFD9FED1E0B53EC102B04F062
:101F100061FA9FED1D0B53EC102B04F05BFA9FED63
:101F20001C0B53EC102B0BF0B3FA9FED1B0B53EC77
:101F3000102B0BF0CDFB9FED1A0B53EC102B04F084
:101F400049FA0BF0C3FC40F20001C1F20001A1F814
:101F5000CE00B1F9CE20B1F9D030B1F9CE009A421D
:101F600002DDA1F8D00080BDB1F9D2209042BCBF03
:101F7000B1F8CE00A1F8D20080BD00BF00BF00BF05
:101F8000000000000070A740000000000000F03ECC
:101F90000000000000C082C00000000000002440DB
:081FA0000000000000005940A0
:101FA80080B5A0F500400BF0C9FC9FED0D0B53EC7C
:101FB800102B04F00BFA9FED0C0B53EC102B04F0D4
:101FC80005FA9FED0B0B53EC102B04F0FFF904F00E
:101FD8000DFB40F20001C1F20001C1F8D40080BD40
:101FE800000000000070A74000000000000018403A
:081FF800000000000000003FA2
:102000002DE9F04F81B040F2E84AC1F2000ADAE966
:10201000000140F2000408434EF68060C1F2000463
:10202000C0F2360005D1D4F8341100224143CAE988
:10203000001240F2F04BC1F2000BDBE90012114339
:1020400005D1D4F8381148430021CBE90001B4F898
:102050007250D4F8E400B4F97010B0EB010826D443
:1020600040460BF06FFC07462846894604F0D4FA38
:102070009FED510B55EC106B32462B460BF028FBB5
:102080003A464B4604F0A6F98146B4F9D6010F460C
:102090000BF058FC32462B460BF01AFB02460B465F
:1020A0004846394604F096F90BF010FC01E0D4F8EC
:1020B000F000C4F87C01D4F87C01D4F8D8104FF4B7
:1020C0007A7281FB000100230BF06EFC226ED4E9D2
:1020D0005C371B184F41C4E95C37D4E95A37C01844
:1020E0007941C4E95A01D4F800014FF46161012833
:1020F000A2FB01560EDBD4F8D8004FF47A7280FBB5
:10210000080100230BF050FCD4E96E2380185941DC
:10211000C4E96E01D4E95C014FF46162281A76EBE0
:102120000100B8BFC4E95C56D4E95A010023013864
:1021300071F10000A4BF0020C4E95A00D4E95A019B
:102140000BF032FCC4F84801D4E95C014FF4616241
:1021500000230BF029FCC4F87801D4F80801D4F866
:102160000811B0F1FF3F12DDDBE900020023401847
:1021700042EBE1714EF68062C0F23602CBE900011B
:102180000BF042FCC4F8380101B0BDE8F08FDAE989
:1021900000024942401842EBE1714EF68062C0F203
:1021A00036020023CAE900010BF02EFCC4F834010A
:1021B00001B0BDE8F08F00BF0000000000408F407C
:1021C00050EC101B4FF0FF3202EB105240F2FE7346
:1021D0009A4280F09A802DE9F84F2DED028B82B063
:1021E00001A809F090FC019F554B54EC105B284668
:1021F000214600220BF04CF981468A46514B284675
:10220000214600220BF044F943F6CE32C6F27F623B
:10221000AA1A4AF29E02C3F6E67274EB0202BCBF2F
:1022200054464D46804644EC105B0E46BEBF5646B3
:10223000C846013F4FF0FF300CF038F851EC100B5E
:10224000414B00220BF024F902460B464046314632
:102250000BF03EFA05460E4602460B4604F0BAF86D
:1022600083468A4641EC180B42F2E879C0F6000931
:1022700048460221B0EE480AF0EE680A09F05BFC1D
:1022800051EC100B314A324B0BF002F904468846F0
:1022900009F110000321B0EE480AF0EE680A09F0D7
:1022A00084FC53EC102B204641460BF011FA5A46A1
:1022B000534604F08FF82A46334604F08BF82A463A
:1022C00033460BF0E5F80646884638460BF03AFBF5
:1022D00004460D461F4A204B04F07CF83246434624
:1022E0000BF0D6F8064688461C4B204629460022AD
:1022F00004F070F8324643460BF0CAF841EC100B7C
:1023000002B0BDEC028BBDE8F88F20F000434A42DA
:1023100040F20002C7F6F07272EB030308D31042DA
:1023200007D00028BCBF002102F5002040EC101BA4
:1023300070479FED010B7047000000000000F0FFA8
:102340000000E0BF0000F0BF0000E03F9AB5B3120C
:10235000FF0750C0A80C615C10D02BBF0030E63FD7
:102360002DE9F04F83B056EC107BC6F30A500138CC
:1023700040F2FE71884280F0A98043F6EF10CFF65C
:10238000FA60C01B42F64260C4F28600B041C0F25F
:10239000B2804BF6D240CDF67A50C01B42F22B30C1
:1023A000CCF28600B041C0F0898044F22320C0F610
:1023B000924026F00041381A49F6A140C3F6C730D2
:1023C00071EB00007DD3544D0195F00F2C4660F366
:1023D000DF74524A524B3846314603F0FBFF00226D
:1023E00023460BF055F80BF071FA02900BF0AAFAA5
:1023F000044688464B4B002203F0ECFF3A46334636
:102400000BF046F806460F46474A484B20464146E1
:1024100003F0E0FF32463B460BF03AF880460C46AC
:1024200002460B4603F0D6FF06460F46404A414B94
:1024300003F0D0FF404A414B0BF02AF832463B46AE
:1024400003F0C8FFA5F5801300220BF021F84246E7
:10245000234603F0BFFF82468B46394A394B30464C
:10246000394603F0B7FF384A384B0BF011F80446F1
:1024700088460020294652465B4603F0A7FF0546E2
:102480008946304639462246434603F0A3FF2A4692
:102490004B460AF0FDFF02460B46504659460BF0EC
:1024A00017F90022019B0AF0F3FF41EC100B029890
:1024B000013003B0BDE8F04F0BF0F8BE9FED100BFC
:1024C00001E09FED130B03B0BDE8F08F26F0004054
:1024D000794240F20001C7F6F07171EB0002F2D3CD
:1024E000484038437FF46FAF002EBCBF0646074616
:1024F00046EC107BE7E79FED040BE4E700BF00BF6D
:102500000000000000000000000000000000F07F5C
:10251000000000000000F03F0000E03F3CF92F9E6B
:102520002C15F73F0030E6BFA80C615C10D02B3FA4
:102530001CDC586FA452F13EE0F6B36FE4707C3FB0
:102540000938DE6F993F403FB35142718E71AC3F05
:102550002DE9F8432DED068BB0EE408AF0EE608A4F
:1025600058EC104B0020C3F6F07088EA00012143BC
:1025700000F0A98055EC116B00F18042154200F08B
:10258000A780C8F30A51013940F2FD73994279D806
:10259000C5F30A51A1F2FF714FF60203CFF6FF73A4
:1025A00099426FD3304629460BF090F907460BF05D
:1025B000C9F9B7F1004F40D07040694008433CD1A1
:1025C0009FED799B002FB0EE49AAF0EE69AA25D0C5
:1025D0003E4648BF7E429FED74AB59EC1A4B55EC1A
:1025E000188B4046294622464B4603F0F3FEF2077D
:1025F00004BF4946204641EC1A0B4FEA56094046B3
:10260000294642462B4603F0E5FE012E04BF29462B
:10261000404641EC180B5FEA0906DED151EC190B7C
:1026200055EC1A8B42462B460BF052F8002F5CBF3C
:102630002946404641EC110B08E020464146002265
:10264000002303F07BFF48B19FED651BB0EE410A0C
:10265000F0EE610ABDEC068BBDE8F8836FF3DF781E
:1026600048EC104BFFF7ACFD53EC102B30462946DD
:1026700003F0B0FE41EC100BBDEC068BBDE8F84357
:10268000FFF76EBE28F00041634272EB01031AD3DC
:1026900025F00043D6F1000972EB0303D6D318EA04
:1026A000020F18D088F0704383F07F63234331D04A
:1026B00082EA080222434FD13DA0002DA8BF083076
:1026C00090ED001BC2E7B0EE481AF0EE681ABDE7C5
:1026D0009FED351BBAE7304629460BF0F7F8074661
:1026E0000BF030F985EA010286EA00031A437FF411
:1026F00060AF37A0002DA8BF08304FEAD872D0E9EC
:102700000010034662F3DF73FA0708BF034643EC89
:10271000111B9BE726A0002DA8BF0830294690ED8D
:10272000008B30460BF0D2F804460BF00BF959EC55
:10273000183B70404FEAD8764A46694066F3DF722C
:10274000084318461CBF4A461846E10704BF4A46DC
:10275000184642EC110B79E700F1004202F1804388
:102760006B40334311D188EA020020439FED0E1BDA
:102770003FF46CAF4FF6FF70C3F6EF7014A28142C6
:1027800088BF083292ED001B60E7814208D388EAD7
:1027900002000BA1204308BF083191ED001B55E753
:1027A0009FED031B52E700BF000000000000F03F58
:1027B0000000000000000000000000000000F07FAA
:1027C000000000000000F07F000000000000F03F6B
:1027D000000000000000F07F00000000000000008A
:0827E000000000000000F87F7A
:1027E800EDAF16204A62304029BD56B31544E9BF03
:1027F80077900D9CFE0B88C07E2615FA8380734067
:082808000FCE674B80D541C0E3
:10281000B0B58CB040F664500024C1F200004FF017
:10282000A0410422C0E9001482614FF480714FF48A
:10283000805281830121C2631C2200F1440C0B945D
:10284000CDE90944CDE90744CDE90544CDE9034488
:10285000CDE90144C0E90244C0E90444016280F8C2
:102860002440C0E90B4480F8384080F840108023B1
:102870008CE81C00016504F019FD002818BF04F065
:10288000F9F94FF40040CDE90A0440F664500625FA
:10289000C1F2000009A9099505F0B8FF002818BF8A
:1028A00004F0E8F90220C0F23040CDE90105012032
:1028B00003900020C4F27F000490042005900020C3
:1028C000069040F66450C1F2000001A905F0B0F88E
:0C28D000002818BF04F0CEF90CB0B0BD19
:1028DC0070B588B040F6F84040F200110024C1F207
:1028EC000000C5F20001C0E900144FF4807181832F
:1028FC004FF4805104250126C1631C2100F14403CF
:10290C00CDE90644CDE90444CDE90244CDE90044C7
:10291C00C0E90244C0E904448561066280F82440A1
:10292C0080F8384080F84060802256C304F0B8FC30
:10293C00002818BF04F098F90820C0F690400090C9
:10294C000620CDE901060020C4F27F00CDE9030585
:10295C0040F6F840C1F200006946059405F062F8B3
:0C296C00002818BF04F080F908B070BD0E
:1029780010B58CB040F68C4040F200410024C1F202
:102988000000C5F20001C0E900144FF48071818392
:10299800032101624FF4805101220823C1631C21E5
:1029A80000F1440C0B94CDE90944CDE90744CDE985
:1029B8000544CDE90344CDE90144C0E90244C0E936
:1029C8000442836180F82440C0E90B4480F8382031
:1029D80080F8402080238CE81A00026504F062FC2D
:1029E800002818BF04F042F940F68C40C1F20000FC
:1029F80009A9099405F006FF002818BF04F036F964
:102A08000220C0F230400190062002900720039077
:102A18007F200490042005900020069040F68C400A
:102A2800C1F2000001A904F0FFFF002818BF04F05C
:102A38001DF941F20000C3F2602001900C200290C1
:102A480040F68C40C1F2000001A904F0EDFF002817
:102A580018BF04F00BF92020C1F2F04001901220B9
:102A6800029040F68C40C1F2000001A904F0DCFF9E
:0C2A7800002818BF04F0FAF80CB010BDE4
:102A840070B59CB0044600201B90CDE91900CDE937
:102A9400170002A8542103F0FDFD206800F1304026
:102AA4004FEA3020062800F27581DFE810F00700B5
:102AB4008800730173014500D60019014FF40040EA
:102AC40002904FF08050139002A801F07FFD00287F
:102AD40018BF04F0CDF841F20431C1F200010A68D4
:102AE40041F24C00C4F20200531C0B6042B901686D
:102AF40041F400510160016801F400510191019910
:102B04000168002641F001010160006817A900F086
:102B14000100019001980320CDE917004FF0904087
:102B2400199606F0B9FE41F23C150820C1F20005E1
:102B3400C4F20200052181E04FF4803002904FF08E
:102B44008040149002A801F041FD002818BF04F051
:102B54008FF841F20031C1F200010A6841F24C00E1
:102B6400C4F20200531C0B6042B9016841F4804175
:102B74000160016801F48041019101990168002616
:102B840041F002010160006817A900F00200019001
:102B9400019842F2030017900320189040F200407D
:102BA400C4F60000199606F077FE0820C4F202006D
:102BB40041F27C052830C1F200052521D0E04FF414
:102BC400004002904FF08050139002A801F0FEFCE8
:102BD400002818BF04F04CF841F20431C1F200019E
:102BE4000A6841F24C00C4F20200531C0B6042B963
:102BF400016841F400510160016801F40051019140
:102C040001990168002641F001010160006817A9DB
:102C140000F0010001900198C02017900320189043
:102C24004FF09040199606F037FE0820C4F20200D7
:102C340041F2DC051430C1F20005242180224FF456
:102C440000734FF4006C28606960AE60EE602A6126
:102C54006B61C5F818C0EE6193E04FF480300290C8
:102C64004FF08040149002A801F0B0FC002818BF77
:102C740003F0FEFF41F20031C1F200010A6841F2A3
:102C84004C00C4F20200531C0B6042B9016841F4C9
:102C940080410160016801F480410191019901685A
:102CA400002641F002010160006817A900F002004B
:102CB400019001984FF4404017900320189040F27F
:102CC4000040C4F60000199606F0E6FD0820C4F2A0
:102CD400020041F21C053C30C1F2000526213FE010
:102CE4004FF4803002904FF08040149002A801F01D
:102CF4006DFC002818BF03F0BBFF41F20031C1F2A4
:102D040000010A6841F24C00C4F20200531C0B603B
:102D140042B9016841F480410160016801F48041D5
:102D2400019101990168002641F0010101600068E8
:102D340017A900F00100019001984FF4407017901A
:102D4400032018904FF09040199606F0A5FD082036
:102D5400C4F2020040F6BC755030C1F200052721D0
:102D640080224FF480734FF4006C4FF0200E2860E3
:102D74006960AE60EE602A616B61C5F818C0C5F881
:102D84001CE028462E6205F069FF08B103F070FFCD
:082D94006565AC621CB070BD66
:102D9C0080B541F26C2043F20001C1F20000C4F294
:102DAC000201016040F201118180FF2300214FF0EC
:102DBC00070C1022C0E9043181610121C0E902C273
:102DCC00016205F015FE002814BFBDE8804080BDEF
:042DDC0003F04ABFF7
:102DE000006843F20001C4F20201884200D070473B
:102DF00081B041F24800C4F20200016841F4805100
:102E00000160006800F480500090009801B07047A5
:102E100080B540F6986046F60001C1F20000C4F2A9
:102E200000010022C0E9001210210123C0E90222A2
:102E3000C0F80F20C0E90513C0E90733C0E9093322
:102E4000C0E90B33C0E90D22C26300F09BFD0028EE
:0C2E500014BFBDE8804080BD03F00CBF43
:102E5C0080B540F6346046F60041C1F20000C4F281
:102E6C0000010022C0E9001210210123C0E9022256
:102E7C00C0F80F20C0E90513C0E90733C0E90933D6
:102E8C00C0E90B33C0E90D22C26300F075FD0028C8
:0C2E9C0014BFBDE8804080BD03F0E6BE1E
:102EA8002DE9F04786B0002741F24C000597CDE99F
:102EB8000377CDE90177C4F20200016840F20048C7
:102EC80041F0040101600168C4F6000801F0040142
:102ED80000910099016808F5806641F020010160C1
:102EE8000168002201F0200100910099016842F276
:102EF800030441F001010160016801F00101009142
:102F08000099016841F002010160016801F00201C5
:102F180000910099016841F008010160006842F2DF
:102F2800030100F0080000900098304601F018F8FE
:102F38004FF09040302100224FF0300901F010F896
:102F480040464FF4E05100224FF4E05A01F008F8EF
:102F580001AD0194012430462946CDE90247049782
:102F680006F098FC4FF090402946CDE90194CDE950
:102F7800037706F08FFC40462946CDE901A4CDE948
:102F8800037706F087FC4FF48060CDE901074FF026
:102F980090402946039406F07DFC042001904FF4EC
:102FA800041608F500602946CDE9026406F072FCB3
:102FB8008020CDE9010640462946039406F06AFCC4
:102FC8004FF40070CDE9010740462946039706F003
:102FD80061FC08200021002200F024FC082000F0F9
:102FE80061FC17200021002200F01CFC172000F0D3
:082FF80059FC06B0BDE8F087AA
:1030000080B541F29C1048F20041C1F20000C4F2C8
:10301000000148F2BE220023C2F2B1024FF0010CBF
:1030200080E80E10C0E90433C0E90633036206F0FD
:10303000B7FD002818BF03F01DFE41F29C10C1F23D
:103040000000002106F0EEFF002818BF03F012FE7A
:1030500041F29C10C1F20000002107F039F800286D
:0C30600014BFBDE8804080BD03F004BE3A
:10306C00B0B59CB00446002502A854211B95CDE9AF
:10307C001955CDE9175503F009FB206848F20041BA
:10308C00C4F20001884236D047F60001C4F20001B8
:10309C00884261D14FF480700290002402A80B94F6
:1030AC0001F090FA002818BF03F0DEFD41F24C0548
:1030BC00C4F20205286817A940F0040028602868AB
:1030CC0000F00400019001984FF44070179012200A
:1030DC00CDE9180408201B9040F60000C4F600004F
:1030EC001A9406F0D5FBE86840F08040E860E86888
:1030FC0000F080402EE04FF40030029002A80C95B6
:10310C0001F060FA002818BF03F0AEFD41F24C0448
:10311C00C4F20204206817A940F004002060206863
:10312C0000F0040001900198C02017901220189014
:10313C000020CDE9190008201B9040F60000C4F6D1
:10314C00000006F0A5FB206940F002002061206918
:0C315C0000F00200019001981CB0B0BD12
:1031680080B541F2902043F20001C1F20000C4F2A0
:1031780000014FF47A73032280E80E00C36006F062
:10318800F9FF002814BFBDE8804080BD03F06EBD84
:1031980070B594B006AC2046382103F079FA0025C2
:1031A8004FF400700595CDE90355CDE9015507F0B9
:1031B80061F807F055F841F29000C4F20200016886
:1031C800032621F0180101602D2006904FF480306D
:1031D8000790012010210890CDE90B0002201091E2
:1031E80008210D90CDE90E60CDE91110139020460D
:1031F80007F0BEF860B90F20CDE9010601A8032148
:10320800CDE90355059507F0B5FB08B914B070BDB5
:0432180003F02CFD96
:10321C00B0B540F2000541F2E821C1F20005C1F25F
:10322C000001D5F828010A68904200D1B0BD0860B1
:10323C0007F014F841F24424C1F2000420460121A5
:10324C004BF6BE6201F0C4FCD5F82C2120460221BD
:10325C0001F0BEFCD5F830212046032101F0B8FC6A
:10326C00D5F834212046042101F0B2FCD5F83821E0
:10327C002046052101F0ACFCD5F82821204606217A
:10328C0001F0A6FCD5F80C212046072101F0A0FC8A
:10329C00D5F810212046082101F09AFCD5F84021E0
:1032AC002046092101F094FCD5F8482120460A213A
:1032BC0001F08EFCD5F8F42020460B2101F088FC9F
:1032CC00D5F8782120460C2101F082FCD5F8D821C4
:0C32DC0020460D21BDE8B04001F07ABC96
:1032E8000A4601464DF69200C0F600000BF09AB867
:1032F80010B596B0044601A8542103F0C9F9206816
:1033080042F60001C4F20001884201D016B010BD97
:103318004FF4002001904FF48070159001A801F03F
:1033280053F9002818BF03F0A1FC41F25800C4F279
:103338000200816B41F400418163016841F48061BE
:103348000160006800F480600090009816B010BD1D
:1033580080B582B041F25800C4F20200816841F0A1
:1033680001018160816801F0010101910199016801
:1033780041F080510160006800F080500090009892
:10338800022003F077FF00F04DF902B0BDE880405D
:0433980006F0E4BF98
:0C339C0041F23C10C1F2000005F0BCBE84
:0C33A80041F2DC00C1F2000005F0B6BEEE
:0C33B40041F27C00C1F2000005F0B0BE48
:0C33C00041F21C00C1F2000005F0AABEA2
:0C33CC0040F6BC70C1F2000005F0A4BE89
:0C33D80040F65C70C1F2000005F09EBEE3
:0C33E40040F6FC60C1F2000005F098BE4D
:0C33F00040F62030C1F2000008F0BAB92D
:0C33FC0040F68C20C1F2000008F0B4B9CB
:10340800802808D0042814D141F2B020C1F200006D
:1034180001210160704740F20000C1F20000B0F8DD
:1034280054110131A0F85411B0F856110131A0F827
:043438005611704772
:10343C0080B540F6203043F60001C1F20000C4F222
:10344C0001014FF49642002380E80E0000F10C01BC
:10345C004FF4806C4FF00C0E81E80850C0E9063335
:10346C00C0E90833836207F08DFE002818BF03F013
:10347C00FBFB40F62030C1F20000002102F00EF9F7
:10348C00002818BF03F0F0FB40F62030C1F200001A
:10349C00002102F075F9002818BF03F0E5FB40F697
:1034AC002030C1F2000008F093FC002814BFBDE8E6
:0834BC00804080BD03F0D8BB85
:1034C40010B540F68C20C1F2000044F2004C4FF4D9
:1034D40080530021C4F2000C4FF496424FF4806EE6
:1034E4000C24C0E90231C0E90611C0E90811816267
:1034F4004FF40041C0E900C2C0E904E4816307F06D
:1035040045FE002818BF03F0B3FB40F68C20C1F23F
:103514000000002102F0C6F8002818BF03F0A8FB41
:1035240040F68C20C1F20000002102F02DF90028A1
:1035340018BF03F09DFB40F68C20C1F2000008F098
:103544004BFC002814BFBDE8104010BD03F090BB35
:1035540080B540F2085045F60041C1F20000C4F2C3
:10356400000101604FF4027181800221C1710021C8
:10357400816000F08DFF002814BFBDE8804080BD4D
:0435840003F076BB1F
:1035880080B5032000F032F90F2000F007F808B1E9
:0C359800012080BDFFF7DCFE002080BD9C
:1035A40041F27071C1F20001096809B310B5044613
:1035B40041F28070C1F200004FF47A720068B2FBED
:1035C400F1F1B0FBF1F005F001FA01460F2C4FF0D8
:1035D40001000CD859B94FF0FF302146002200F009
:1035E40023F941F26C710020C1F200010C6010BD9E
:0435F40001207047FB
:0C35F80041F2A020C1F200000068704702
:10360400B0B50446FFF7F6FF054641F27070C1F20B
:1036140000000068611C18BF044400BFFFF7EAFF04
:08362400401BA042FAD3B0BD27
:10362C003020C4F20100016821F0010101607047F3
:10363C002DE9F041036840F20016C5F20006B342D2
:10364C004FF4C16708BF4FF40277B3F1A04F03F1F9
:10365C00304308BF4FF40277BC594FEA3323062B93
:10366C0026D8012707FA03F313F0730F20D0036851
:10367C009F687F0703D490F85870012F02D1022065
:10368C00BDE8F08104F01F0706F5A0640125A342F4
:10369C0080F8585018BF002F1AD10D46904604469A
:1036AC0004F03CF9F0B1002184F85810BDE8F08129
:1036BC004CF21E13C0F60003804618460F4640F22B
:1036CC00DB711546FFF70AFE39462A464046CEE71F
:1036DC00052FE2D0092FE0D0002180F858100120EE
:1036EC00BDE8F0812168E06D40F6017398432246F5
:1036FC0000F58070B142E06509D040F20050C5F28F
:10370C0000008142084608BF06F5407001E04FF00A
:10371C00A040884211BF002FD06D20F48010D065DE
:10372C00D06D43F29977C0044FF0000044BF106E87
:10373C0020F006001066506D47F60926C0F600070B
:10374C00C0F6000647F611240023C0F60004C0E9B9
:10375C000B761C2744630F6082F858304B68144674
:10376C0043F010034B60CB682A4643F00103CB6057
:10377C004031434605F0FAFB21688A6822F000428A
:0C378C0022F03F0204328A60BDE8F081A8
:103798000146806AC36DC26D13F0500F05D0D20682
:1037A8000FD4406D426B0846104742F40071C16562
:1037B80001680B68CA681B0705D4910709D503F08F
:1037C8005FBB04F02DB912F4406FF8D1C9688904C1
:1037D800F5D4C16D21F48071C165C16DC9045EBFA6
:0C37E800C16D41F00101C16503F04ABB56
:1037F40010B504460338052806D34DF69730C0F6B5
:103804000000A621FFF76EFD4EF60C50CEF200002C
:1038140001684FF6FF02114064F30A2141F0806110
:0838240041F0FD71016010BDCF
:10382C0070B515460E46102A044606D34DF6973051
:10383C00C0F60000BE21FFF751FD102E06D34DF649
:10384C009730C0F60000BF21FFF748FD4EF60C5034
:10385C00CEF2000001684FF0FF33C1F3022181F07A
:10386C000702042A28BF0422033903FA02F238BFE4
:10387C00002126EA02028A4003FA01F125EA01013D
:10388C001143002C4FEA011105D44EF20040CEF248
:10389C000000215470BD04F00F021044017270BD81
:1038AC00B0F1FF3F0DDD00F01F01012202FA01F122
:1038BC001C2202EAD0004EF20012CEF2000281501D
:1038CC0070474DF69730C0F60000D221FFF706BDC9
:0438DC0000F000F800
:1038E0004EF60C50BFF34F8FCEF200000168042259
:1038F00001F4E061C0F2FA5211430160BFF34F8F4F
:0439000000BFFDE720
:10390400B0B55FEA520C10D0D0F800E0002300BF3D
:10391400CC18CD5A6488BCF1010C44EA054403F187
:103924000403CEF80040F3D100E00023D2071EBF09
:0C3934000268C95A118000680068B0BD2C
:1039400070B5D0E913C4D0F854E0CCF80440BEF10F
:10395000000F1CBFD0E9164CC4F804C0D0E910CE4B
:10396000046886680EF01F00012505FA00F0CCF807
:10397000040008466360102E04BF10460A46A0608B
:04398000E26070BDD4
:10398400002800F005812DE9F0410446006846F264
:103994000048C4F20008404513D046F60001C4F2C2
:1039A400000188420DD046F60041C4F2000188426D
:1039B40007D04EF64060C0F600004FF49871FFF750
:1039C40091FC206840450AD16068102807D34EF660
:1039D4004060C0F6000040F23311FFF783FCA0689A
:1039E400002818BFB0F5807F40F0EF80E06805281C
:1039F40007D34EF64060C0F600004FF49B71FFF70A
:103A040071FC207C022807D34EF64060C0F600000B
:103A140040F23711FFF766FC607C022807D34EF6AC
:103A24004060C0F600004FF49C71FFF75BFCA07C83
:103A3400022807D34EF64060C0F6000040F2391168
:103A4400FFF750FC60690138B0F5007F07D34EF6EC
:103A54004060C0F600004FF49D71FFF743FCA0697D
:103A64000138802807D34EF64060C0F6000040F2CB
:103A74003B11FFF737FCE0690138B0F5807F07D3CD
:103A84004EF64060C0F600004FF49E71FFF72AFC2A
:103A9400206A0138802807D34EF64060C0F6000043
:103AA40040F23D11FFF71EFCA068B0F5407F2FD116
:103AB400606A0138202807D34EF64060C0F6000043
:103AC4004FF4A071FFF70EFCA06A0138102807D349
:103AD4004EF64060C0F6000040F24111FFF702FCD0
:103AE400E06A0138202807D34EF64060C0F6000093
:103AF4004FF4A171FFF7F6FB206B0138102807D3B0
:103B04004EF64060C0F6000040F24311FFF7EAFBB6
:103B1400606B1D2807D34EF64060C0F6000040F2EB
:103B24004511FFF7DFFBA06B092807D34EF6406071
:103B3400C0F600004FF4A371FFF7D4FBE06B40F034
:103B44008070B0F1807F07D04EF64060C0F6000070
:103B540040F24711FFF7C6FB94F85C0028B9002037
:103B640084F85D00204602F045FF2068816921F059
:103B740010018161FFF73EFD054600BF20688169A1
:103B8400090707D5FFF736FD401B0B28F6D312E0D3
:103B940001207047816941F001018161FFF72AFD2D
:103BA400054600BF20688169C9071BD1FFF722FDC4
:103BB400401B0B28F6D3206E032140F00100206641
:103BC400012084F85C10BDE8F081B0F5407F3FF43B
:103BD4000DAF4EF64060C0F6000040F23511FFF71D
:103BE40081FB03E78169404541F00201816104BF23
:103BF4006168C8F80011217C8269012922F0400221
:103C040018BF40328261617C8269012922F48042BA
:103C140008BF02F580428261A17C8269012922F4F5
:103C2400805218BF02F5805282618369D4E902127E
:103C340023F440730B438361836923F0A4038361FA
:103C4400036923F0100303619AB1012A0DD0022AFB
:103C540009D08369032A43F080038361036943F035
:103C64001003036105D1202200E0042283691A4372
:103C74008261D4E90552D4E90736571E6FF0FF027A
:103C840002EB032343EA4763771E1F430023CFF667
:103C9400FF7303EB05463743B1F5407FC76110D18D
:103CA400D4E90917D4E90B65013F02EB06223A4334
:103CB4006FF00F0707EB05173A4303EB014111437C
:103CC400C160D4E90D23E16BD0F8C0704AF250769C
:103CD4003943C0F8C01008F5806708F58041B84240
:103CE40004BF4AF25071C4F2000108F50067C4F23F
:103CF4000006B84208BF06F554712164D0F88070FC
:103D040027F4F81747EA0242C0F8802001F1700254
:103D14006264D0F8802022F0706242EA0362C0F844
:103D2400802001F1B000A06401F5C470E06401F5E5
:103D34001870206501F51E70606501F5547000224D
:103D440041F8042B8142FBD300200121A0652066A9
:083D540084F85C10BDE8F08169
:103D5C0070B542F210060446C4F20206FFF746FCA8
:103D6C00054600BF3068C00306D5FFF73FFC401B7B
:103D7C00A042F7D9032070BD30684CF2FA310140F3
:103D8C0008D041F24C70C1F2000042680A43426014
:103D9C00012005E03068C0074FF0000001D0012180
:043DAC00316070BD55
:103DB00042F21400C4F20200016841F000410160C7
:083DC0000068C043C00F70470A
:103DC800416842F2200CC4F2020C06220429026067
:103DD80020D803291ED00722042902601AD8DFE858
:103DE80001F0030B07190F00614651F80C2F0AE088
:103DF800614651F82C2F06E0614651F8102F02E079
:103E0800614651F8302F02F07F0282600968C1F3E1
:103E18000641C160B0B5DCF80010C9B20A46AA294B
:103E280018BFBB22CC2908BF0A460261DCF8001083
:103E3800C26921F0FF01531E012B816173D801680B
:103E480047F2E05541F0080101600021C4F2010188
:103E58000B68C1F6FF75DB05298840F20003C0F640
:103E680004034FF6FF7409D4A1424FF0006E10D03E
:103E780029684FF0006361F358230AE0A14205D096
:103E880029684FF0006E61F3582E00E09E464FF00F
:103E98000063DCF8001049020DD4022A1FD0012A61
:103EA8003BD1DCF804104FF0006361F31213036296
:103EB800DCF808301CE0022A1FD0012A2DD1DCF8DA
:103EC80004104FF6F873C0F2030303EAC10171440A
:103ED8000162DCF8081003EAC10171441CE0DCF857
:103EE80024104FF0006361F312130362DCF82830EA
:103EF8004FF0006163F312110EE0DCF824104FF666
:103F0800F875C0F2030505EAC10119440162DCF83D
:103F1800281005EAC10119444162DCF8081001F0D3
:103F280000411143C1610268C16A42F01003036095
:103F3800DCF850304D1E012D03F4803383620ED817
:103F480042F030020129026004D0022907D10CF1A5
:103F5800540101E00CF150010968C9B20163B0BD18
:103F680070B516460C46054679B1022E07D34EF2B7
:103F78003E70C0F6000040F29B11FFF7B1F918201F
:103F8800002E08BF28202C5070BD4EF23E70C0F69F
:103F980000004FF4CD71FFF7A3F9022EE7D2EEE748
:103FA8002DE9F04381B00446006880690840401A52
:103FB800B0FA80F0400982422CD1DDF82080154605
:103FC8000E461F4603F1010912E000BF2068806910
:103FD8003040801BB0FA80F0400985421ED020682E
:103FE80080693040801BB0FA80F04009854211D1C9
:103FF80020463946424600F089F9D8B9B9F1000F90
:10400800EDD0FFF7F5FA002FE0D0A0EB0800B8429A
:10401800E5D9DBE7002001B0BDE8F083606C40F033
:1040280020006064202084F84100002084F84200C9
:0C40380084F84000012001B0BDE8F083D6
:10404400F0B581B004460068806980071CD4154629
:104054000E464F1C08E000BF20688069800716D513
:104064002068806980070FD4204631462A4600F034
:104074004FF9C0B9002FF3D0FFF7BCFA002EEBD0F4
:10408400401BB042ECD9E7E7002001B0F0BD606C02
:1040940040F020006064202084F84100002084F86F
:0C40A400420084F84000012001B0F0BD93
:1040B00070B5044600688069800619D415460E461E
:1040C00008E000BF20688069800615D520688069F7
:1040D00080060DD4204631462A4600F01BF948B927
:1040E000FFF78AFA002EEDD0401BB042EED9E9E787
:1040F000002070BD012070BD606C40F02000606445
:10410000202084F84100002084F8420084F8400018
:04411000012070BD5D
:1041140000688169890744BF002181628169C907F8
:0C41240002BF816941F001018161704718
:104130002DE9F04F81B08B46591E89B21E461746B5
:104140000229044607D34CF20660C0F6000040F690
:10415000E111FFF7C9F894F8410020280AD10A9D1F
:1041600065B1DDF82C80B8F1000F07D094F840005D
:1041700001280AD1022001B0BDE8F08F4FF4007091
:104180006064012001B0BDE8F08F012084F8400098
:10419000FFF732FA814620464FF4004101221923ED
:1041A000CDF80090FFF700FF0146012011B101B0EA
:1041B000BDE8F08F212084F8410040204FF0000A34
:1041C000DDF830C084F84200C4F844A0656242F2D1
:1041D0000005C8F20005F2B2204659464FF0807340
:1041E000A4F82A80C4F834A00095654605F0A8FD1F
:1041F000204629464A46FFF725FFB0B92068012E20
:1042000008D0390A8162204629464A46FFF71AFF3C
:1042100058B92068F9B281622046802100222B46DD
:10422000CDF80090FFF7C0FE10B184F840A0A8E7D9
:10423000608DB0F5807F08D3FF20208500272046C1
:104240005946FF224FF0807307E0608D00272085DC
:10425000C2B2204659464FF00073009705F070FD3A
:104260000026FF270BE0608D59462085C2B220460C
:104270004FF00073009605F063FD608D70B320462B
:1042800029464A46FFF7DEFE00287FF47AAF606ACF
:10429000216810F8012B8A626062608D01386085A8
:1042A000208D01382085618D0029E6D00004E4D1FD
:1042B0002046802100222B46CDF80090FFF774FEA7
:1042C00000287FF45EAF608DB0F5807FCBD327856B
:1042D00020465946FF224FF08073CBE720462946FF
:1042E0004A46FFF7E5FE00287FF44BAF2068202107
:1042F000C16142684EF60003CFF600631A40426087
:10430000002084F8411084F8420084F8400001B095
:04431000BDE8F08F85
:104314002DE9F04381B00446006816468369DA0645
:1043240002D40026002548E00D461021C161206812
:104334008169890634D4002705F101094FF000088A
:1043440008E048F0200801272068816901F0200175
:10435400394328D1B9F1000FF6D0FFF74BF915B165
:10436400801BA842F0D92068426894F842108369FF
:104374001B040BD512F4804208D1202906D04168D1
:1043840041F480414160FFF735F9064620688069B1
:104394008006D9D4FFF72EF9801B1A28F6D3D0E76C
:1043A4000121042604E0B7FA87F1490948F004061C
:1043B400012500291CBF2021C16120688169CA052B
:1043C4001ED44A0524D489052AD4ADB12046FFF76A
:1043D4009FFE20684EF600024168CFF6006211404D
:1043E4004160606C30436064202084F84100002008
:1043F40084F8420084F84000284601B0BDE8F08308
:1044040046F001064FF480720125C2614A05DAD5EF
:1044140046F008064FF480620125C2618905D4D5AF
:1044240046F002064FF400710125C161CED1E3E7E5
:1044340010B582B004460020CAF6AA2004EA00019E
:10444400814218BF14F47F0007D14EF24F10C0F61A
:10445400000040F23D11FEF745FF41F26000C4F256
:104464000200016841F001010160006800F00100F0
:10447400019001980420C4F2010001682143016005
:0444840002B010BDB5
:0C44880001684AF6AA2200200A60704772
:10449400002859D070B50646006845F60041C4F2BC
:1044A4000001884206D04CF65600C0F60000872171
:1044B400FEF718FF96F8910228B9002086F89002BA
:1044C400304602F09FFE032086F89102306801F026
:1044D400C1F93079A8B100EB8001C90000224FF086
:1044E400010C0023002400BFF51828332C749942D2
:1044F40004F1010485F811C0EA74C5E90822AA622E
:10450400F2D180B106F5B4710022002301F8183C01
:10451400013301F8172C01F8152C41E9022241F866
:10452400282B9842F2D196E8070007F0AFFC002050
:104534000121307386F89112B17A012903D13046F2
:0C45440005F07AFE002070BD01207047D9
:1045500041F20C01C4F2020151F8040C42F2004293
:10456000C0F2F40200F00C00042810462DD051F8DF
:10457000040C00F00C00082847F64000C0F27D1043
:1045800023D051F8043C03F00C030C2B1ED180B552
:10459000D1F800C00B680CF0030CC3F3031E0B68CA
:1045A0000EF1010EBCF1030F08BF02460968B2FB11
:1045B000FEF0C3F30623C1F341610222584302EB2C
:1045C0004101B0FBF1F0BDE880407047002070472A
:1045D0002DE9F04381B004460068000306D14EF295
:1045E0003320C0F600008321FEF77EFEA07841F262
:1045F00088090007C4F2020901D4002575E0206D86
:104600004FEA3020042806D34EF23320C0F60000D3
:104610008B21FEF769FE59F8300C5FEAC0080BD415
:1046200059F8300C40F0805049F8300C59F8300CF3
:1046300000F080500090009847F20007C4F2000795
:10464000386840F480703860FEF7D6FF054600BF3A
:104650003868C60508D4FEF7CFFF401B0328F7D300
:104660000325002E03D437E00025002E34D5D9F8D9
:10467000080010F4407025D0216D884222D0D9F86E
:104680000800D9F8081020F4407241F48031C9F8CC
:104690000810D9F80810C00721F48031C9F80810B3
:1046A000C9F808200ED0FEF7A7FF064641F2893769
:1046B000D9F80800800705D4FEF79EFF801BB8429A
:1046C000F6D3032545B9D9F80800216D20F44070D0
:1046D00008430025C9F80800B8F1000F5EBF59F87B
:1046E000300C20F0805049F8300C2078C00711D0F1
:1046F0006068042806D34EF23320C0F60000E021A3
:10470000FEF7F2FDD9F80000616820F003000843CD
:10471000C9F800002078800713D5A0684FEAB000E0
:10472000042806D34EF23320C0F60000EA21FEF73B
:10473000DBFDD9F80000A16820F00C000843C9F89F
:1047400000002078400713D5E0684FEA30100428B5
:1047500006D34EF23320C0F60000F621FEF7C4FD6A
:10476000D9F80000E16820F030000843C9F80000E3
:104770002078000714D520694FEAB010042807D329
:104780004EF23320C0F6000040F20311FEF7ACFDFC
:10479000D9F80000216920F0C0000843C9F80000E2
:1047A0002078C00614D560694FEA3020042807D36A
:1047B0004EF23320C0F600004FF48871FEF794FDEE
:1047C000D9F80000616920F440700843C9F800007E
:1047D0002078800614D5A0694FEAB020042807D3BA
:1047E0004EF23320C0F600004FF48E71FEF77CFDD0
:1047F000D9F80000A16920F440600843C9F800001E
:10480000207840060ED5E069002818BFB0F5805F1B
:1048100040F04D81D9F80000E16920F44050084390
:10482000C9F80000207800060ED5206A002818BFBD
:10483000B0F5804F40F04881D9F80000216A20F49B
:1048400040400843C9F800006078C0070ED0606A95
:10485000002818BFB0F5803F40F04381D9F8000030
:10486000616A20F440300843C9F80000A07880074E
:1048700012D5A06A032807D34EF23320C0F60000F9
:104880004FF4A471FEF730FDD9F81400A16A20F0AE
:1048900003000843C9F814006078800714D5E06A63
:1048A0004FEAB040042807D34EF23320C0F6000090
:1048B0004FF4AA71FEF718FDD9F80000E16A20F460
:1048C00040200843C9F80000607840071DD5206BE0
:1048D0004FEA3050042807D34EF23320C0F60000D0
:1048E00040F25F11FEF700FDD9F80000216B20F4C3
:1048F00040100843C9F80000B1F5801F02BF59F805
:104900007C0C40F4801049F87C0C607800071DD5C1
:10491000606B4FEAB050042807D34EF23320C0F644
:1049200000004FF4B971FEF7DFFCD9F80000616BAD
:1049300020F440000843C9F80000B1F5800F02BF21
:1049400059F87C0C40F4801049F87C0C6078C00663
:1049500017D5A06B002818BFB0F1807F40F0CE8043
:10496000D9F80000A16B20F040700843C9F800009E
:10497000B1F1807F02BF59F87C0C40F4801049F8F7
:104980007C0C607880061ED5E06B40F00060B0F1D2
:10499000006F07D04EF23320C0F6000040F29711AE
:1049A000FEF7A2FCD9F80000E16B20F0406008435C
:1049B000C9F80000B1F1006F02BF59F87C0C40F457
:1049C000801049F87C0C607840061ED5206C40F0C1
:1049D0000060B0F1006F07D04EF23320C0F6000047
:1049E0004FF4D371FEF780FCD9F80000216C20F061
:1049F00040600843C9F80000B1F1006F02BF59F8E8
:104A00007C0C40F4801049F87C0C6078000616D5C8
:104A1000606C002818BFB0F1805F7CD1D9F800002D
:104A2000616C20F040500843C9F80000B1F1805F8C
:104A300002BF59F87C0C40F4803049F87C0CA07817
:104A4000C00716D0A06CB0F1004F18BF00286FD17E
:104A5000D9F80000A16C20F040400843C9F80000DC
:104A6000B1F1804F02BF59F87C0C40F4803049F816
:104A70007C0CA078400716D5E06C002818BFB0F574
:104A8000801F61D1D9F81400E16C20F44010084374
:104A9000C9F81400B1F5001F02BF59F87C0C40F4AE
:104AA000801049F87C0C284601B0BDE8F083B0F5D1
:104AB000005F3FF4AFAE4EF23320C0F600004FF47B
:104AC0009371FEF711FCA5E6B0F5004F3FF4B4AECC
:104AD0004EF23320C0F600004FF49871FEF704FC4C
:104AE000AAE6B0F5003F3FF4B9AE4EF23320C0F66F
:104AF000000040F23B11FEF7F7FBAFE6B0F1007F9C
:104B00003FF42EAF4EF23320C0F6000040F2851184
:104B1000FEF7EAFB24E7B0F1005F3FF47FAF4EF20F
:104B20003320C0F600004FF4DA71FEF7DDFB75E7C5
:104B3000B0F1804F8CD04EF23320C0F6000040F22E
:104B4000C511FEF7D1FB83E7B0F5001F9AD04EF2F6
:104B50003320C0F600004FF4EC71FEF7C5FB91E77F
:104B600070B504460068C16849061CD4C16841F0AC
:104B70008001C160FEF740FD2168C968490612D472
:104B800005460026FEF738FD401BB0F57A7F84BF4E
:104B9000032684F825602068C068400601D4032EEF
:0C4BA000F0D1F0B270BD0026F0B270BD84
:104BAC00B0B5044600685F21C0F20101C160FEF798
:104BBC001DFD05462068C068800607D4FEF716FD6B
:104BCC00401BB0F57A7FF5D90320B0BD0020B0BDF5
:104BDC00B0B50C462029154607D34EF61230C0F658
:104BEC00000040F2E471FEF779FB42F20050C4F28F
:084BFC00000040F82450B0BD98
:104C04002DE9F04381B0044680681E4615460F46E0
:104C140038B14CF6DA10C0F600004FF49F61FEF78D
:104C240061FBFEF7E7FC94F85D108146012908D189
:104C3400002F4FF0010018BF002D0ED101B0BDE8C8
:104C4400F0836068B0F5827F0DD104294FF0020033
:104C5400F4D1A1680029EBD0F0E7002EEED094F84F
:104C64005C00012803D1022001B0BDE8F0830120DB
:104C740084F85C0094F85D00DDF8208004281CBFF3
:104C8400052084F85D00002020662564A4F84660B1
:104C9400A4F84460A763E687C4E913002068A687E4
:104CA400E1684268B1F5E06F22F48052134698BF80
:104CB40003F58053012E88BF134643600268731EB8
:104CC40052065EBF026842F0400202606268B3FAB4
:104CD40083F3B2FA82F252095B09B1F5E06F43EA59
:104CE40002013DD931B137F8021BC160A763E08FDF
:104CF4000138E087012608F1010500BFE08F20B9E3
:104D0400B4F84600002800F0A38020688168890771
:104D14000CD5E18F51B1012E08D1A16B002631F8D9
:104D2400022BC260A163E18F0139E1878168C90761
:104D34000DD0B4F8461051B1C068216C012621F899
:104D4400020B2164B4F846000138A4F84600FEF7CB
:104D540051FC002DD2D0A0EB09004045CED36DE02C
:104D640000294FF6FE7111D0E28F022A05D337F8DD
:104D7400022BC2604FF6FE7004E03A780273A06B17
:104D8400471C481CA763E28F1044E087012708F101
:104D940001054E1CE08F18B9B4F84600002857D01E
:104DA40020688168890717D5E18FA9B1012F13D134
:104DB400E28FA16B022A05D331F8022BC2604FF6B1
:104DC400FE7004E009780173A06B411C3046A163B6
:104DD400E18F00270844E08720688168C90725D04F
:104DE400B4F8461011B3B4F84610022912D3C168BE
:104DF400226C22F8021B2264B4F846100239A4F88B
:104E04004610B4F8461001290FD8416841F4805186
:104E140041600AE0007B216C0870206C0130206442
:104E2400B4F846000138A4F846000127FEF7E2FB77
:104E3400002DAFD0A0EB09004045ABD3012084F88E
:104E44005D00002084F85C00032001B0BDE8F0831D
:104E5400204641464A4606F077F940B120202066B4
:104E6400002084F85C00012001B0BDE8F08301203B
:104E740084F85D00002084F85C00206E002818BFD0
:084E8400012001B0BDE8F0833C
:104E8C002DE9F04F83B04FF000091E4690460D46B9
:104E9C0083468DF80790FEF7A9FB301A00EB080744
:104EAC00FEF7A4FB41F28071C1F2000109682322D4
:104EBC005143090DDBF800A079430291DAF8081090
:104ECC0029424DD0064608F1010404E0DBF800004D
:104EDC008068284217D0B5F5C06F02BF9AF80C0055
:104EEC008DF807009DF80700002CEFD0FEF77EFB35
:104EFC00801BB8420AD202980299002808BF0746C4
:104F0C00481E0290E2E74FF0000929E0DBE90001BE
:104F1C004268B1F5827F22F0E00242600BD1DBF8EF
:104F2C000810B1F5004F02D0B1F5806F03D10168C4
:104F3C0021F040010160DBF82810B1F5005F07D1CA
:104F4C00016821F400510160016841F400510160D5
:104F5C0001208BF85D0000208BF85C004FF00309FA
:084F6C00484603B0BDE8F08FD8
:104F7400F0B581B015460E460446FEF73BFB281AF1
:104F84008719FEF737FB41F28071C1F2000109680D
:104F9400C1F3CB317943009121688968090602D4B1
:104FA400002001B0F0BD0546013603E020688068AA
:104FB4000006F5D5002EF9D0FEF71CFB401BB842C5
:104FC40007D200980099002808BF0746481E0090A1
:104FD400ECE7D4E900014268B1F5827F22F0E002F7
:104FE40042600AD1A168B1F5004F02D0B1F5806FDB
:104FF40003D1016821F040010160A16AB1F5005FAD
:1050040007D1016821F400510160016841F40051A5
:105014000160012084F85D00002084F85C00032016
:0450240001B0F0BD2A
:10502800F0B581B00446406841F63121C0F21E1146
:10503800884207D34EF2FC70C0F6000040F6DD311E
:10504800FEF74EF9A068002818BFB0F5805F40F061
:10505800C68048F200072168C4F20007E068B94238
:1050680014D04FEA3030042807D34EF2FC70C0F653
:10507800000040F6E531FEF733F9206A40F400609D
:10508800B0F5006F0FD040F6E63106E040F400506E
:10509800B0F5005F07D040F6E1314EF2FC70C0F683
:1050A8000000FEF71DF92069002818BFB0F5806FD1
:1050B80040F0A280606910B130F00C0007D04EF2C9
:1050C800FC70C0F6000040F6EA31FEF709F9A06965
:1050D8004FEA3020042807D34EF2FC70C0F60000D7
:1050E80040F6EB31FEF7FCF8E06940F40040B0F51B
:1050F800004F07D04EF2FC70C0F6000040F6EC31CD
:10510800FEF7EEF8606A0C2807D34EF2FC70C0F682
:10511800000040F6ED31FEF7E3F804F108014EC94E
:105128002068194341EA0603E169066846F6F31563
:10513800CCF6FF752E4033430B4303604368B842F7
:1051480023F4405342EA03024260A2691CBF236A67
:105158001A43836823F06E4323F430631A43826052
:10516800C26A636A22F00F021A43C26244F6FF72EF
:10517800C4F2000290424FF0100218DC44F20043DF
:10518800C4F20003984244D044F60003C4F200037A
:1051980098424CD044F60043C4F2000398425BD1D5
:1051A80041F28802C4F20202126892094CE045F208
:1051B8000003C4F20003984232D0B8423ED043F60E
:1051C8000003C4F20103984246D141F28802C4F2B6
:1051D8000202126845F23063C0F6000338E0B0F10D
:1051E800805F3FF436AF4EF2FC70C0F6000040F628
:1051F800DE31FEF775F82CE7B0F5C06F3FF45AAF13
:105208004EF2FC70C0F6000040F6E931FEF768F88F
:1052180050E741F28802C4F202021268920813E0D1
:1052280041F28802C4F202021268120A0CE041F24A
:105238008802C4F202021268120905E041F28802EB
:10524800C4F202021268920A45F24063C0F60003F3
:1052580002F0030253F82220B84242F20040C0F2A2
:10526800F40013D0B1F5004F1ED1082A00F2648073
:105278000026DFE802F00569736171616161B500BC
:1052880005F0F4FC002840F06A809DE0082A4ED81A
:105298000026DFE802F0054C1E4C184C4C4C1C0054
:1052A80005F0E4FCB8B98FE0082A49D80026DFE801
:1052B80002F0054F7447724747479C0005F0D6FC3B
:1052C80000286BD180E0FFF73FF920B97CE04FF46C
:1052D8000040002878D0616A4EF29422C0F600029D
:1052E80032F811206568B0FBF2F305EB45018B42FB
:1052F8004FF001016BD32F03BB4268D80021002374
:1053080008F07EFB090241EA1061000210EB55002B
:1053180041F100012A46002308F072FB4FF60052C3
:10532800A0F54071C0F20F0291424BD34EE000202D
:1053380001260028CFD147E00020012678B943E0B4
:105348000020012650BB3FE005F0A6FC38B93BE041
:1053580005F0A2FC10BB37E0FFF7F6F8A0B3616ACE
:105368004EF29422C0F6000232F811106268B0FBC7
:10537800F1F0510801EB4000B0FBF2F04FF6EF728C
:10538800A0F11001914221D84FF6F0710140C0F30D
:105398004200084416E0FFF7D7F8A8B1616A4EF258
:1053A8009422C0F6000232F811106268B0FBF1F0E6
:1053B80000EB5200B0FBF2F04FF6EF72A0F11001D3
:1053C800914203D82168C860314600E001214FF0BE
:1053D80001100022A06662670846A26701B0F0BD0E
:1053E8004FF400400028BAD1EEE74FF400400028FF
:0453F800D4D1E9E73C
:1053FC002DE9F04704460068C0690840401AB0FA2D
:10540C0080F04009824237D1DDF82080A1F14000C4
:10541C0015460E46994630F0400A08F1010718BFB0
:10542C004FF0010A09E000BF2068C0693040801BC2
:10543C00B0FA80F0400985421ED1002FF4D0FEF75F
:10544C00D5F80146B8F1000F4FF0030015D0A1EBD1
:10545C000901414511D8206801680AEA9101012926
:10546C00E2D1C16909070AD4C1690905DCD5032554
:10547C0020264FF4006105E00020BDE8F0870125EF
:10548C00082108260162204606F026F90020C4F8FF
:0C549C00906084F884002846BDE8F0878A
:1054A800D0F88C30202B07D100294FF0010318BF0A
:1054B800002A04D118467047022318467047002373
:1054C800C366D0F800C048F20003C4F200039C454C
:1054D80012D080B5DCF804301B020BD5036853E802
:1054E800003FD0F800C043F080634CE8003EBEF1B6
:0C54F800000FF3D1BDE8804000F000B8C8
:10550400B0B513460A46816500210446A0F85C3014
:10551400C0F890102220C4F88C00D4F88000E8B1C0
:105524004BF27165C0F60005456325684BF6594C8E
:105534004BF6E94EC0F6000CC0F6000E816305F18F
:105544002401C0E90BCE03F015FD38B11020C4F8D6
:1055540090002020C4F88C000120B0BD206948B11F
:10556400206850E8000F216840F4807041E8000290
:10557400002AF5D12068083050E8000F216840F077
:105584000100083141E80002002AF3D12068083004
:1055940050E8000F216840F04000083141E8000263
:0855A400002AF3D10020B0BD84
:1055AC00016851E8001F026821F0C00142E80013B5
:1055BC00002BF5D10168083151E8001F026821F475
:1055CC000001083242E80013002BF3D12021C0F86F
:0455DC00881070477C
:0C55E000806A0021A0F85E1000F0E8BC1A
:1055EC00016848F20002C4F20002914209D0D0F8DE
:1055FC008820202A03D190F88420012A03D102208C
:10560C007047012070472422C0F888204A6842F471
:10561C0000024A602021C0F88810002180F8841014
:04562C0000207047A3
:10563000010000000400000002000000080000005B
:10564000000000000400000002000000080000004C
:10565000416E19B380B501684EF6A06C8A688968FE
:10566000C0F6000C490F4EF6A86E1CF80130C0F6CB
:10567000000E1EF80110DB00B3FBF1F1C2F3426231
:10568000A0F86A101CF802101EF80220C900B1FB35
:10569000F2F1BDE88040A0F8681070470121A0F841
:0856A0006A10A0F868107047C1
:1056A800B0B50446006844F6FF72C4F200029042A6
:1056B80012DC44F20042C4F20002904228D044F6C0
:1056C8000002C4F20002904222D044F60042C4F222
:1056D800000290421CD011E045F20002C4F2000220
:1056E800904215D048F20002C4F2000290420FD056
:1056F80043F60002C4F20102904209D04CF66E2033
:10570800C0F600000D464FF41971FDF7E9FD294672
:1057180081F000404FEA7070072828D8012202FA69
:1057280000F010F0F30F22D094F88400012801D182
:105738000220B0BD012084F884002420C4F8880029
:1057480020680568026822F001020260826822F07F
:105758006042114381602046FFF776FF20680560AC
:105768002020C4F88800002084F88400B0BD4CF6DE
:105778006E20C0F600000D4640F26521FDF7B0FD31
:045788002946D1E7F6
:10578C0070B50446006844F6FF72C4F20002904201
:10579C000D4612DC44F20041C4F20001884226D0CE
:1057AC0044F60001C4F20001884220D044F60041C6
:1057BC00C4F2000188421AD011E045F20001C4F293
:1057CC000001884213D048F20001C4F20001884263
:1057DC000DD043F60001C4F20101884207D04CF60B
:1057EC006E20C0F6000040F29521FDF777FD4FEAE0
:1057FC007560062807D34CF66E20C0F6000040F208
:10580C009621FDF76BFD94F88400012801D102204C
:10581C0070BD012084F884002420C4F8880020681E
:10582C000668016821F001010160816821F0606166
:10583C00294381602046FFF705FF20680660202081
:0C584C00C4F88800002084F8840070BDBF
:105858000146B0F8400044F27F0202400020A1F85F
:045868004020704725
:10586C0040F20000C1F20000B0F8CC104FF47A7393
:10587C00A0F88C10B0F98C10B0F97E20891A41F286
:10588C00E422C1F2000212685A4392FBF1F20021A9
:08589C00C0F8902006F0E0BE08
:1058A4002DE9F04F89B040F60004C4F60004204608
:1058B40001210122FEF756FB9620FDF7A1FE41F2DD
:1058C4009025C1F200052846FEF7DCFD20460221A2
:1058D4000022FEF747FB9620FDF792FE2846FEF7CE
:1058E400D1FD204602210122FEF73CFB9620FDF764
:1058F40087FE2846FEF7C6FD204601210022FEF75A
:1059040031FB40F6D05440F64620C1F2000406AD07
:1059140006904FF47A76204629462A4602230096BA
:10592400FFF76EF926208DF81800204629462A46EE
:1059340003230096FFF764F99DF81A000A2864D13E
:105944009620FDF75DFE41F29020C1F20000FEF7C3
:1059540099FD40F6D054C1F200042046202106F0FF
:10596400AFFA06AD2327204629462A4603238DF89D
:1059740018700096FFF744F99DF81A004FF0430899
:1059840000F0EF008DF81900204629462A4602232C
:105994008DF818800096FFF733F9204629462A46E9
:1059A40003238DF818700096FFF72AF906AD2046F8
:1059B40029462A4603238DF818700096FFF720F92C
:1059C4009DF81A00294600F09F0020308DF8190038
:1059D40020462A4602238DF818800096FFF710F916
:1059E400204629462A4603238DF818700096FFF7AF
:1059F40007F99DF81A0080060FD44EF60C10C0F675
:105A0400000005F09CFE00BFFEE74EF6E060C0F625
:105A1400000005F094FE00BFFEE743F2514040F65B
:105A2400D054ADF818000020C1F2000406AD8DF882
:105A34001A004FF47A78204629462A460223CDF8E4
:105A44000080FFF7DDF831208DF818002046294644
:105A54002A460323CDF80080FFF7D2F89DF81A00F8
:105A6400342805D04CF64E70C0F6000005F067FEF1
:105A740040F6D059002704244EF6254AC1F2000905
:105A840006AD04AE4FF0000B06E000BF002010BBD3
:105A9400002CA4F101041ED04846294632460323B3
:105AA400CDF818A08DF81270ADF81070CDF8008004
:105AB400FFF7A6F89DF81000FF28E7D19DF8110024
:105AC4009DF818108842E1D19DF812004FF0010BA7
:105AD40003900120DCD0BBF1000F4DD0039840F6B9
:105AE400D05540F060074FF0000804244FF04509FA
:105AF4004FF47A7AC1F2000506AE0DF1100B0020C6
:105B0400039000BF284631465A4602238DF8189068
:105B14008DF81970ADF81080CDF800A0FFF770F87B
:105B24009DF81000FF2809D19DF811009DF8181068
:105B3400884203D101210120039100E0002018B91B
:105B4400002CA4F10104DDD10398F8B10BF1040099
:105B540041F26C2A40F6D0590190002505264EF6F4
:105B64002544C1F2000A06AF4FF47A78C1F2000965
:105B74000020039016E000BF4FF09040202103F076
:105B8400EBFFC820FDF73CFDF6E700BF4FF0904067
:105B9400202103F0E1FFFA20FDF732FDF6E700BF14
:105BA400013E4AD0504639460222CDE9064502F06C
:105BB400DDFF8DF81A00484639465A460623ADF8EB
:105BC40014500495CDF80080FFF71AF89DF81000E2
:105BD400FF282DD19DF811009DF81810884227D177
:105BE4009DF812009DF81910884221D19DF81300E8
:105BF4009DF81A1088421BD19DF815000199029056
:105C04005046012202F0B2FF0299884210D19DF859
:105C1400140000F060006028039808BF012003907E
:105C24004FF0000008BF0C200E2804D1B8E700BFD5
:105C34000E200E28B4D00028B2D00398002863D0D8
:105C440041F29020C1F20000FEF71CFC41F26C2AE4
:105C540040F6D0574FF0000804244EF6F249C1F242
:105C6400000A06AE4FF47A75C1F200070DF1100B6D
:105C740000200390504631460222CDF8189002F0DD
:105C840075FF8DF81A00384631465A460423CDF87C
:105C940010800095FEF7B4FF9DF81000FF2815D181
:105CA4009DF811009DF8181088420FD19DF812003C
:105CB4009DF81910884209D19DF813009DF81A1017
:105CC400884203D101210120039100E0002018B98A
:105CD400002CA4F10104CDD10398F8B10BF1040018
:105CE40041F26C2A40F6D0590190002505264EF663
:105CF4002144C1F2000A06AF4FF47A78C1F20009D8
:105D04000020039016E000BF4FF09040202103F0E4
:105D140023FF4FF49670FDF773FCF5E74FF09040C6
:105D2400202103F019FF4FF4AF70FDF769FCF5E78C
:105D3400013E4AD0504639460222CDE9064502F0DA
:105D440015FF8DF81A00484639465A460623ADF821
:105D540014500495CDF80080FEF752FF9DF8100012
:105D6400FF282DD19DF811009DF81810884227D1E5
:105D74009DF812009DF81910884221D19DF8130056
:105D84009DF81A1088421BD19DF8150001990290C4
:105D94005046012202F0EAFE0299884210D19DF990
:105DA40014000121B0F1FF3F4FF00700C8BF0020ED
:105DB400039AD8BF0A460392092804D1B8E700BF62
:105DC40009200928B4D00028B2D00398A0B141F228
:105DD4009024C1F200042046FEF754FB9620FDF700
:105DE4000FFC2046FEF74EFB00F010F82046FEF7AD
:105DF40049FB09B0BDE8F08F4FF09040202103F03B
:0C5E0400ABFE4FF4C870FDF7FBFBF5E7A8
:105E100040F60000C4F6000001210122FEF7A4B8FC
:045E2000FAF7C6BE09
:105E240040F20000C1F20000D0F84011D0F8402147
:0C5E3400002948BF5242C0F80C21704702
:105E400040F20001C1F20001D1F84001B0F1FF3F82
:105E5000DABFD1F8400140420020D1F80C21002ADD
:105E600003DDD1F80C21D31701E0CA6D002310B572
:105E700048F29F64C0F20104611C80FB010107F03D
:105E800093FD48F2A062C0F20102121A201A4FF0EC
:105E900000008841B8BF0022002944BF48F2A06238
:085EA000C0F20102104610BD22
:105EA80010B582B040F20004C1F20004B4F85A0000
:105EB800A4F88001B4F9CC00B4F96A10884219DA60
:105EC800B4F8CCC0B4F9CC00B4F96C108842D8BF8F
:105ED800B4F86CC0B4F96C00B4F96E10B4F96A2067
:105EE800B4F95A300FFA8CFCCDF800C006F09CF8D3
:085EF800A4F8800102B010BD06
:105F000010B582B00DF1070200200021012300F03E
:105F100019F89DF80700411CC8B202280ED845F6B2
:105F2000B072C0F6000252F82000C900C9B24FF4A6
:105F3000813222FA01F405F004FC00E00324E0B20F
:045F400002B010BDDE
:105F44002DE9F04F83B0924606465818012241F2DB
:105F5400F0181D4602EB901700204FF47A79C1F235
:105F6400000800BF8BB213FA85F32C4641EA86126F
:105F7400402B28BFC1F140041FFA80FB1AFA80F0BD
:105F8400A1B2CDE9000192B24046A0210223CDF88E
:105F9400089003F049FF01362D1B1BFA84F0013FE2
:0C5FA4004FF00001DED103B0BDE8F08F2B
:0C5FB0001ED00008ADE90008E9EB000875
:105FBC0010B5044640F20000C2F200000121017548
:105FCC00002180F83112D4F88010B4F85C200968F4
:105FDC004968511AC0F82812D4F89000D4F89000EF
:105FEC00042805D14EF66870C0F6000008F018FAC7
:105FFC00D4F89000012805D14EF67870C0F6000058
:10600C0008F00EFAD4F89000022805D14EF68870EC
:10601C00C0F6000008F004FAD4F89000102805D15E
:10602C004EF64040C0F6000008F0FAF9D4F89000A3
:10603C00102805D14EF64040C0F6000008F0F0F9EB
:10604C00D4F89000082805D14EF65140C0F6000057
:10605C0008F0E6F9A16D20464FF48072FFF71EFAA6
:10606C0038B14EF61320C0F60000BDE8104008F021
:04607C00D7B910BDC3
:1060800040F20000C2F20000002180F826107047A4
:1060900003460068B3F82C224FF00C0C03F22711D2
:0860A00083F826C005F060BA88
:1060A8004FF6FF72C1B1B0B54FF0000C4AF2010EC5
:1060B80010F80C305A406FF0070300BF8EEA520404
:1060C800D50708BF540801332246F7D30CF1010C59
:0C60D8008C45EDD1BDE8B04090B270479F
:1060E40070B58E1E0C4631460546FFF7DBFFA95BF3
:0C60F400814218BF4FF0FF34204670BD01
:04610000007D704767
:1061040070B540F2000CC1F2000C002BBCF8184032
:1061140018BFA3420AD18B7891F803E04EEA032416
:10612400B4F5FE7F08D340F2862101E040F68631C3
:1061340081520220104470BD0D790CEB4406757039
:106144004D7986180CF8145006258554737086F81A
:1061540002E00879F070487930710520104470BD70
:106164002DE9F04140F20006C1F20006002B378B06
:1061740018BFBB420CD10F7991F8058048EA072774
:10618400A7F17C0515F17C0F05D84FF4647110E07C
:1061940040F686310DE091F802C091F803E04EEA32
:1061A4000C243D19A5F2FD1313F5FE7F06D24FF41E
:1061B4002471815202201044BDE8F0818FB14FEA6E
:1061C4004C2343EA4E03334408315E1C11F8013C6E
:1061D400013406F8023B11F8023BAC4206F8033CDA
:1061E400F4D31023811883540020C8700520104470
:1061F40081F801C081F802E081F80480BDE8F081F3
:1062040040F20000C1F20000016E4FF2F012CFF62E
:0C621400FF725143CA17C0E95A127047CC
:1062200010B540F20004C1F20004D4F80C010028BB
:106230004FF6FF700ED4D4F80C11E26D91420CD2DF
:10624000E26D3AB14FF47A70E26DA1FB00010023D8
:1062500007F0DAFBA4F8140110BD4FF47A70A4F82B
:04626000140110BD58
:1062640040F20000C1F20000026E8AB180B5D0E9AC
:106274005C0148F2A06CC0F2010CA0FB0C034FF4CB
:10628400616E01FB0C31A2FB0E2307F08BFB80BD7A
:04629400002070472F
:1062980040F20001C1F20001D1F84801B0F1FF3F1E
:1062A800DABFD1F8480140420020D1F81021002A75
:1062B80003DDD1F81021D31701E00A6E002310B5D1
:1062C80048F29F64C0F20104611C80FB010107F0E1
:1062D80067FB48F2A062C0F20102121A201A4FF0BE
:1062E80000008841B8BF0022002944BF48F2A062DC
:0862F800C0F20102104610BDC6
:1063000040F20000C1F20000D0F81011002907DDB2
:10631000D0F80C11D0F8402111444FEAE17C05E09F
:10632000C16DD0F840214FF0000C114470B5D0F889
:10633000D830B0F88061D0F81051012D03DBD0F8CF
:106340001041E51701E0046E0025981900EBD073A9
:106350005E10A1FB0602DB1701FB03214FF47A72EA
:106360000CFB0611002307F01FFB48F2A066C0F2E9
:106370000106A0FB060201FB062122462B4607F080
:1063800013FB20EAE070B042B8BF0646304670BD4D
:10639000034C206804348047FBE7F9F71DFFFEE754
:0463A000E4F000081D
:1063A40007F004F84EF60850CEF2000005490160EB
:1063B4004EF68850CEF20000016851F4700101607D
:0863C400FFF7E4FF00000008F0
:0863CC0083F0004307F05EB806
:1063D400F0B540F2FF7681EA030C16EA115E1EBFA7
:1063E400B64516EA1355B54252D021EA465141F456
:1063F4008011A1FB024723EA465343F48013AE44C1
:10640400A0FB03650CF0004C36197D41A1FB03474A
:1064140047F10003A0FB0217F619654153F100038D
:10642400094218BF46F0010640F2FE74B3F5007F3E
:1064340013D2AEF5806EA64523D24CEA033128036D
:1064440041EA155140EA16503203450872F1004200
:1064540050F1000051EB0E51F0BDAEF2FF3EA645E7
:106464000FD24CEAC321E80241EA555140EA5650A2
:10647400F202450872F1004250F1000051EB0E5156
:10648400F0BD1EEA0E0F2DD50CF000410020F0BD2A
:1064940016EA115F04BF01F000410020004218BF5A
:1064A40041F0010116EA135F04BF03F00043002228
:1064B400124218BF43F0010306EA1354B44218BF52
:1064C400B64503D00CF000410020F0BD21F000419E
:1064D40023F00043B1EB065F0CD8B3EB065F09D899
:1064E40041B13BB10CF0004141F0FE4141F4700177
:1064F4000020F0BD40F20001C7F6F8710020F0BDA5
:106504004FF4001C1CEB410F98BF1CEB430F11D838
:1065140051EA030C50EA4C0C5CEA020C0AD004D297
:1065240082428B4180414042704790429941804170
:0865340040427047002070474F
:10653C004FF4001C1CEB410F98BF1CEB430F11D800
:10654C0051EA030C50EA4C0C5CEA020C0AD004D25F
:10655C009042994180414042704782428B41804138
:08656C00404270470020704717
:10657400C1F30A5240F21E439A1A15DA203225DD7D
:10658400CB17C90241EA5051C00241F00041D14148
:10659400D04048409140D14048405B1C18BF7047F0
:1065A400404263EB01017047CB17C90241EA5051E5
:1065B400C00241F00041202A28BF202231FA02F013
:1065C400190008BF70474042894170474B000042A0
:1065D40018BF43F0010313F5001F88BF21F00041E9
:1065E400002011F000415CBF6FF00041C0437047D0
:1065F4000B0D40F21E42D21A09DBCB0243EA505083
:1066040040F00040202A28BF2022D0407047490093
:04661400804170470A
:1066180050B140F21D42B0FA80F1521A8840C30AC4
:0C662800400503EB025170470100704771
:08663400004870477C170010BC
:10663C005AB3844690EA01039B071FD1830707D006
:10664C0011F8013B00F8013B521EF7D11CE08446C7
:10665C00203A09D32DE9F007B1E8F807A0E8F807CC
:10666C00203AF9D2BDE8F0071C3205D451F8043BAE
:10667C0040F8043B121FF9D2043205D011F8013B4B
:0C668C0000F8013B521EF9D16046704737
:1066980000220B0011001A0084465AB3830704D065
:1066A80000F8011B521EF9D124E0C9B241EA0121C8
:1066B80041EA0141202A11D3203A2DE9F0030B4683
:1066C8000C460D460E460F4688468946A0E8FA0352
:1066D800203AFBD2BDE8F00320320BD0042A05D3C0
:1066E80040F8041B121F05D0042AF9D200F8011B38
:0866F800521EFBD16046704701
:1067000000B50549FFF796FF4158044A002908BF24
:106710008118084600BD00BF080000000C00000002
:0C6720005AB600084C6700082C670008FF
:10672C000DE600082DE6000839E6000845E60008ED
:10673C0065E6000871E6000883BE0008ABBD0008E2
:10674C008ED40008CED60008CED60008CED60008CF
:10675C00CED60008CED60008CED60008CED600087D
:10676C00CED60008CED60008FFFFFFFFFFFFFFFFCD
:10677C00FFFFFFFFFFFF0000C2D3000838ED000849
:10678C00A5EA000855ED0008FCEA000826ED000813
:08679C002FED000803EB0008DB
:1067A400B0B588B040F6204040F200510024C1F258
:1067B4000000C5F20001C0E900144FF48071042503
:1067C400818301211C2200F1440CCDE90644CDE96A
:1067D4000444CDE90244CDE90044C0E90244C0E9DF
:1067E40004448561016280F82440C0E90B4480F8C8
:1067F4003810C46380F8401080238CE81C000165C5
:1068040000F052FD002818BF00F032FA1020C1F247
:10681400C000009006200190072002900020C4F2DE
:106824007F00CDE9030540F62040C1F2000069462F
:10683400059401F0FBF8002818BF00F019FA08B01D
:02684400B0BDE5
:02684600FEE76B
:10684800B0B588B040F6B43040F200610024C1F21F
:106858000000C5F20001C0E900144FF48071012264
:106868000823818304251C2100F1440CCDE906444A
:10687800CDE90444CDE90244CDE90044C0E902442D
:10688800C0E904428361056280F82440C0E90B44F2
:1068980080F83820C46380F8402080238CE81A00F0
:1068A800026500F0FFFC002818BF00F0DFF9102097
:1068B800C9F2C000009006200190072002907F20B6
:1068C800CDE9030540F6B430C1F2000069460594ED
:1068D80001F0AAF8002818BF00F0C8F90020CCF28F
:1068E800527000900C20019040F6B430C1F20000C4
:1068F800694601F099F8002818BF00F0B7F904209C
:10690800C0F6600000901220019040F6B430C1F249
:106918000000694601F088F8002818BF00F0A6F9C1
:106928000220C0F2304000901820019040F6B430A8
:10693800C1F20000694601F077F8002818BF00F09E
:0669480095F908B0B0BD96
:02694E00FEE762
:1069500080B582B041F24800C4F202000168002212
:1069600041F004010160016801F004010191019905
:10697000016841F0010101600068002100F00100A0
:10698000009000980B20FCF751FF0B20FCF78EFFC6
:106990000C2000210022FCF749FF0C20FCF786FFA9
:1069A0000D2000210022FCF741FF0D20FCF77EFFA7
:1069B0000E2000210022FCF739FF0E20FCF776FFA5
:1069C0000F2000210022FCF731FF0F20FCF76EFFA3
:1069D000102000210022FCF729FF1020FCF766FFA1
:1069E000112000210022FCF721FF112002B0BDE898
:0669F0008040FCF75BBFD4
:0269F600FEE7BA
:1069F80010B59CB0044600201B90CDE91900CDE9E4
:106A0800170002A85421FFF743FE206846F600410C
:106A1800C4F20001884233D046F60001C4F20001F6
:106A2800884268D14FF4805002904FF00070109067
:106A380002A8FDF7C9FD002818BF00F017F941F2B8
:106A4800FC21C1F200010A6841F24C00C4F20200C4
:106A5800531C0B6042B9C16841F00071C160C16844
:106A680001F0007101910199016841F00201016092
:106A78000068602100F002000190019809202CE0D4
:106A88004FF4805002904FF00070109002A8FDF76C
:106A98009BFD002818BF00F0E9F841F2FC21C1F283
:106AA80000010A6841F24C00C4F20200531C0B605A
:106AB80042B9C16841F00071C160C16801F000715C
:106AC80001910199016841F00201016000681821F3
:106AD80000F00200019001980B20179102211891F3
:106AE80000211B9040F20040CDE91911C4F60000C6
:0A6AF80017A902F0CFFE1CB010BD7C
:026B0200FEE7AC
:106B040080B541F2F01047F60001C1F20000C4F272
:106B1400000141F22E220023C0F2E2024FF0010CE8
:106B240080E80E10C0E90433C0E90633036203F0C1
:106B340035F8002818BF00F09BF841F2F010C1F2BC
:106B44000000002103F06CFA002818BF00F090F850
:106B540041F2F010C1F20000002103F0B7FA00285E
:106B640018BF00F085F84FF48000BDE88040FDF7C1
:026B74005FBC04
:026B7600FEE738
:106B7800B0B541F24420C1F20000012104F08EF9C1
:106B88004BF6BE6188426FD14BF63E70C0F60000EE
:106B980004F0D3FD41F24424C1F20004204602214E
:106BA80004F07CF940F20005C1F20005C5F82C019B
:106BB8002046032104F072F9C5F83001204604216B
:106BC80004F06CF9C5F834012046052104F066F993
:106BD800C5F838012046062104F060F9C5F82801F7
:106BE8002046072104F05AF9C5F80C01204608216F
:106BF80004F054F9C5F810012046092104F04EF9B3
:106C0800C5F8400120460A2104F048F9C5F84801B2
:106C180020460B2104F042F9C5F8F40020460C2167
:106C280004F03CF9C5F8780120460D2104F036F946
:106C3800C5F8D801D5F840014FF4616180FB010225
:106C4800C5E95802D5F8D80180FB0102C5E97802E8
:106C5800D5F8480180FB0102C5E95A02D5F8F400CD
:0A6C680080FB0101C5E93E01B0BD4B
:026C7200FEE73B
:106C74004EF2B96072B6C0F6000004F060FD00BFC9
:026C8400FEE729
:026C8600FEE727
:106C8800B0B58EB001AD044628463421FFF700FDAB
:106C98002846FDF795F88CB34EF6D850C0F600009C
:106CA80004F04BFD0598AA2837D102200190BB209B
:106CB800059002F07FFA28B14EF2C860C0F60000D5
:106CC80004F03BFD02F08EFA28B14BF6D670C0F600
:106CD800000004F032FD4EF6F850C0F6000004F053
:106CE8002CFD01A802F0A6FAE0B14DF6F310C0F6AB
:106CF800000004F022FD02F08DFA4CE00598BB2854
:106D080026D102200190AA20059002F053FA10B370
:106D18004EF2C860C0F600003BE04DF6D610C0F653
:106D2800000013E002F076FA4EF60860C0F60000A4
:106D380004F003FDFDF738F84CF22200C0F600001D
:106D480004F0FBFC4EF62060C0F6000004F0F5FCF1
:106D580001200EB0B0BD4BF68A70C0F6000004F0FA
:106D6800ECFC02F03FFA20B14BF6D670C0F60000FA
:106D78000FE04DF62F10C0F6000004F0DEFC01A86D
:106D880002F058FA50B102F045FA4DF68710C0F6F5
:106D9800000004F0D2FC00200EB0B0BD4EF6BC508E
:106DA800C0F6000004F0C9FC02F034FA4EF60860A0
:106DB800C0F6000004F0C1FCFCF7F6FF4CF222001C
:106DC800C0F6000004F0B9FC4DF66610C0F60000ED
:026DD800BCE716
:026DDA00FEE7D2
:106DDC0010B58EB001AC20463421FFF757FC20468D
:106DEC00FCF7ECFF06200190BB2005904FF4C4404B
:106DFC0006904FF4C040079002F0DAF928B14EF239
:106E0C00C860C0F6000004F096FC02F0E9F928B165
:106E1C004BF6D670C0F6000004F08DFC4EF6F85020
:106E2C00C0F6000004F087FC01A802F001FA044649
:106E3C0040B14DF6F310C0F6000004F07CFC02F0FB
:106E4C00E7F915E002F0E4F94EF60860C0F6000030
:106E5C0004F071FCFCF7A6FF4CF22200C0F6000017
:106E6C0004F069FC4EF62060C0F6000004F063FCF0
:0A6E7C00B4FA84F040090EB010BD16
:026E8600FEE725
:106E8800006800F130414FEA312106293BD8DFE89C
:106E980001F0043A3A3A1C2E3B0040F2006341F2FA
:106EA800C021C5F20003C1F20001012298420A6024
:106EB8002AD040F20051C5F20001884217D040F2B2
:106EC8000041C5F2000188421DD140F2006341F241
:106ED800BC21C5F20003C1F20001012298420A60F8
:106EE80012D040F20051C5F2000188420BD140F2A5
:106EF800006341F2B821C5F20003C1F2000101228A
:106F080098420A6000D0704741F2B420C1F20000F4
:066F180001210160704739
:026F1E00FEE78C
:106F200080B541F2442042F60001C1F20000C4F2F3
:106F3000000100224FF0804E7F234FF0FF0C80E8CD
:106F40000E10C0E90422C0E9062E026203F0BEFE64
:0E6F5000002814BFBDE8804080BDFFF78BBE57
:026F5E00FEE74C
:106F6000B0B540F6D05043F60041C1F20000C4F283
:106F700000014FF4827200234FF4E06C4FF0010ED9
:106F80004FF48024102580E80E100721C0E9043E4C
:106F9000C0E90645C0E90833C0E90A31C0E90C334D
:106FA00003F094FF002814BFBDE8B040B0BDFFF768
:026FB00061BEC0
:026FB200FEE7F8
:106FB400F0B587B0006843F60041C4F20001002533
:106FC4008842CDE90555CDE90355029501D007B0B6
:106FD400F0BD41F24C00C4F20200C16802AC41F4BD
:106FE4000041C160C168022601F400410191019988
:106FF4000168062741F001010160016801F0010107
:1070040001910199016841F0040101600068214681
:1070140000F00400019001984FF4004002904FF0FA
:107024009040CDE903650595069702F035FC4FF4D1
:10703400E050CDE9020640F60000C4F60000214607
:0E704400CDE90455069702F027FC07B0F0BD19
:02705200FEE757
:02705400FEE755
:02705600FEE753
:02705800FEE751
:02705A00FEE74F
:02705C00FEE74D
:02705E00FEE74B
:02706000FEE749
:02706200FEE747
:02706400FEE745
:02706600FEE743
:0270680070476F
:02706A00FEE73F
:02706C0070476B
:02706E00FEE73B
:02707000704767
:02707200FEE737
:06707400042002F087BDBC
:02707A00FEE72F
:06707C00802002F083BD3C
:02708200FEE727
:107084002DE9F0419CB00446002602A854211B9629
:10709400CDE91966CDE91766FFF7FCFA206844F2DA
:1070A4000041C4F2000188423CD043F60001C4F21E
:1070B4000101884240F0A28001200290002402A82D
:1070C4000394FDF783FA002818BFFFF7D1FD41F2BE
:1070D4005800C4F20200816841F4804181608068F4
:1070E40000F480400190019841F24C00C4F2020087
:1070F400016841F004010160006817A900F0040070
:1071040001900198302017900220CDE9180407203F
:107114001B9040F60000C4F600001A9402F0BCFB79
:10712400252463E0022502A802950496FDF74EFA91
:10713400002818BFFFF79CFD41F25800C4F202007A
:10714400016841F24C0641F4003101600068C4F268
:10715400020600F40030019001983068002740F0E6
:1071640001003060306817A900F001000190019817
:107174000C20CDE9170507201B904FF09040CDE976
:10718400197702F089FB40F65C75A6F57E60C1F2C2
:1071940000051A214FF0800885E883002846C5E9D8
:1071A4000378C5E90577C5E9077701F057FD00289D
:1071B40018BFFFF75DFDC4F88050AC6240F6FC6573
:1071C400A6F6CC70C1F200051B21102285E88701C8
:1071D4002846C5E90577C5E9077701F03FFD002892
:1071E40018BFFFF745FDE567AC6226242046002161
:1071F4000022FCF719FB2046FCF756FB1CB0BDE847
:02720400F08117
:02720600FEE7A1
:1072080010B596B0044601A85421FFF741FA20684A
:1072180045F60041C4F20001884201D016B010BD05
:107228004FF4005001900020109001A8FDF7CCF910
:10723800002818BFFFF71AFD41F25800C4F20200F7
:10724800016841F400010160006800F4000000904A
:06725800009816B010BD05
:02725E00FEE749
:1072600041F2707041F2A021C1F20000C1F20001B0
:0A72700000680A68104408607047C7
:02727A00FEE72D
:10727C0010B504466FF00200044207D04CF27600C1
:10728C00C0F6000040F2A221FCF728F83020C4F22E
:0E729C000100016821F002012143016010BDD4
:0272AA00FEE7FD
:1072AC0070B582B0044600200190ECB1206800F16A
:1072BC0030404FEA3020062838D8012101FA00F07E
:1072CC0010F0730F32D06068B0F5801F0FDBB0F593
:1072DC00001F19DAB0F5C01F36DAB0F5801F44D0A4
:1072EC00B0F5A01F41D038E0012002B070BDB0F560
:1072FC00403F13DBB0F5002F21DAB0F5403F34D01E
:10730C00B0F5802F31D028E0B0F5201F21DAB0F590
:10731C00001F2AD0B0F5101F27D01EE028B3B0F5FF
:10732C00803F22D0B0F5003F1FD016E04CF21E106B
:10733C00C0F6000040F29B11FBF7D0FFC3E714D05E
:10734C00B0F5402F11D008E00FD0B0F5E01F0CD0F5
:10735C0003E00AD0B0F5301F07D04CF21E10C0F677
:10736C0000004FF4CE71FBF7B9FFA0684FEAF000B4
:10737C00042807D34CF21E10C0F6000040F29D11F9
:10738C00FBF7ACFFE06840F40040B0F5004F07D0CD
:10739C004CF21E10C0F600004FF4CF71FBF79EFFAD
:1073AC00206944F20A01884207D34CF21E10C0F641
:1073BC00000040F29F11FBF791FF6069022807D390
:1073CC004CF21E10C0F600004FF4D071FBF786FF94
:1073DC00607F022807D34CF21E10C0F6000040F26A
:1073EC00A111FBF77BFF206B4FEAB020042807D3D9
:1073FC004CF21E10C0F600004FF4D171FBF76EFF7B
:10740C00E06AA0F588614FEA71111C2900F2D48161
:10741C00012202FA01F14DF6E572C1F601021142A8
:10742C0000F0CA81606B002818BFB0F1806F40F08B
:10743C00DD8094F83800022807D34CF21E10C0F6F9
:10744C00000040F2A511FBF749FFA069042809D000
:10745C00082807D04CF21E10C0F600004FF4D37170
:10746C00FBF73CFFE06B40F48050B0F5805F07D039
:10747C004CF21E10C0F6000040F2A711FBF72EFFD5
:10748C00207F022807D34CF21E10C0F600004FF4E8
:10749C00D471FBF723FF94F84000022807D34CF279
:1074AC001E10C0F6000040F2A911FBF717FF60692F
:1074BC0038B3206A0138102807D34CF21E10C0F6DE
:1074CC00000040F2AD11FBF709FF94F824000228EC
:1074DC0007D34CF21E10C0F600004FF4D771FBF727
:1074EC00FDFE94F8240001280BD1A06A013808286D
:1074FC0007D34CF21E10C0F600004FF4D971FBF705
:10750C00EDFE94F8240001280AD1607F012807D1F0
:10751C004CF21E10C0F6000040F2B711FBF7DEFE75
:10752C00E06D30B92046FBF7A7FA0020206684F8FE
:10753C0058002168886880004FF6C070C5F6FF704F
:10754C0042BF8A6802408A608A68D2001CD48A686A
:10755C0000F18050104040F08050886041F2807003
:10756C00C1F20000006842F663528009C0F23E523C
:10757C00A0FB02029009022202EB4000019001984C
:10758C0010B101980138F9E78868C00009D4E06DA2
:10759C0040F01000E065206E40F0010020660120F4
:1075AC0000E000208A68E36D02F0040203F010038F
:1075BC00D218E26D16D122F481720232E2658A6829
:1075CC00D20740D140F2001341F48072C5F200039F
:1075DC009A4240F20802C5F2000214D11368D2F8A4
:1075EC00005118E042F010010120E2E0B0F1006F10
:1075FC003FF41FAF4CF21E10C0F600004FF4D271D6
:10760C00FBF76CFE15E7D2F800C4D2F80055D2F89F
:10761C00003645EA0C052B43DB0714D102F1F803C5
:10762C0099424FF4E063D4F804C008BF4FF44073A0
:10763C00B1F1A04F08BF4FF44073D55825F47C1519
:10764C0045EA0C05D550627FE36BD4E902C543EAE9
:10765C0042322A4394F8243042EA0C02012B42EACB
:10766C00034206D1A36A0025CFF6FE7505EB434312
:10767C001A43E36A23B1256B03F478732B431A4343
:10768C00CB6844F20705CFF6F0752B401A43CA605D
:10769C000A69636B22F040621A430A618A68120716
:1076AC0078D494F83820237F520042EA8332CB6896
:1076BC0044F20205AB431A43CA6022690B694AB112
:1076CC0043F480330B61D1F8C03043F6FF75AB4304
:1076DC001A4307E023F480320A61D1F8C02043F644
:1076EC00FF739A43C1F8C02094F84020012A4DD171
:1076FC00616C05464FEAB101082908D34CF21E1003
:10770C00C0F6000040F27621FBF7E8FD2846A16C9C
:10771C004FEA7111092908D34CF21E10C0F6000073
:10772C0040F27721FBF7DAFD2846E16C41F4007159
:10773C00B1F5007F08D04CF21E10C0F600004FF4DB
:10774C001E71FBF7CBFD2846216D40F2014241F43E
:10775C008061914208D04CF21E10C0F6000040F23D
:10776C007921FBF7BBFD28462168D4E911E3D4E964
:10777C00135C0A6940F2FD76B24342EA0E021A43E8
:10778C002A4342EA0C0242F0010202E00A6922F0AA
:10779C0001020A61216862690B6B012A23F00F0256
:1077AC0002BF236A013B1A430A63E16D012262F3B3
:1077BC000101E16502B070BD21686FF0030301F1B6
:1077CC00304203EB3223032B0ED2B0F58C6F1EDB51
:1077DC00B0F5986F33DAB0F58C6F3FF423AEB0F59B
:1077EC00946F3FF41FAE53E04FEA3222012A4CD87B
:1077FC00B0F5986F17DAB0F58C6F27DAB0F5806FAB
:10780C003FF410AEB0F5846F3FF40CAE2BE00028C3
:10781C003FF408AEB0F5806F3FF404AEB0F5846F62
:10782C003FF400AE34E0B0F5CC6F16DAB0F5986FDB
:10783C003FF4F8ADB0F5BC6F3FF4F4AD13E03FF49A
:10784C00F1ADB0F5BC6F3FF4EDAD21E03FF4EAAD26
:10785C00B0F5946F3FF4E6AD05E03FF4E3ADB0F561
:10786C00D06F3FF4DFAD40F20042C5F2000291420E
:10787C00ABD040F20062C5F200029142A5D040F2BA
:10788C000052C5F2000291429FD000283FF4CAADCD
:10789C004CF21E10C0F6000040F2A311FBF71EFDC7
:0278AC00C0E535
:0278AE00FEE7F3
:1078B000B0B5016804468A688868C0074FF00000C8
:1078C00030D012F002022DD1886800F00D0001289E
:1078D0001FD1886820F0004020F03F00023088600F
:1078E00003200860FBF788FE21688968C90701D179
:1078F0000020B0BD054603E020688068C007F7D0CF
:10790000FBF77AFE401B0328F6D320688068C00787
:10791000F2D0E06D40F01000E065206E40F0010014
:0679200020660120B0BD4D
:02792600FEE77A
:1079280070B582B004460020019021688A68D207A9
:1079380011D14FF6C076C7F6FF76886806F17F0248
:1079480010420AD0E06D40F01000E065206E40F073
:1079580001002066012002B070BD88684FF4C16242
:10796800304040F00100886040F20010C5F200008D
:10797800814208BF4FF40272B1F1A04F08BF4FF423
:1079880002721058000220D4FBF732FE21680A6800
:10799800D20717D1054603E021680868C00711D14E
:1079A8008868C00704D18868304040F001008860CA
:1079B800FBF71EFE401B0328EED320680068C007B3
:1079C800EAD1BFE7002002B070BD41F28070C1F279
:1079D8000000006842F663518009C0F23E51A0FBE6
:1079E8000101880900EB40000C2101EB800000BF79
:0E79F800019001980028C7D001980138F8E7E7
:027A0600FEE799
:067A0800806A00F00FB8D7
:027A0E00FEE791
:107A1000806AC16D41F04001C165016E41F0040111
:067A2000016600F001B850
:027A2600FEE779
:027A28007047A5
:027A2A00FEE775
:027A2C007047A1
:027A2E00FEE771
:107A30002DE9F04381B0814600200090D9F8000084
:107A40000D4600F130404FEA3020062800F2EF806A
:107A5000012101FA00F010F0730F00F0E88068686F
:107A6000B0F5007F19DAA0F58071182908D8012235
:107A700002FA01F141F24102C0F2041211421BD19B
:107A8000182800F2E680012101FA00F041F24001DD
:107A9000C0F2041108420FD1DBE0A0F500711829F3
:107AA00000F2CE80012202FA01F141F24102C0F25D
:107AB0000412114200F0C480A868062873D2E86856
:107AC00040F200087F28C4F27F0809D0404507D063
:107AD0004CF21E10C0F6000040F6D521FBF704FC66
:107AE0002869052807D34CF21E10C0F6000040F6A6
:107AF000D621FBF7F9FBD9F800006969C0680622B6
:107B000002EA900040F6FF7222FA00F0814207D9A3
:107B10004CF21E10C0F6000040F6D721FBF7E4FB44
:107B2000286904280BD099F84000012807D14CF2AD
:107B30001E10C0F6000040F6DB21FBF7D5FBE9681C
:107B40002868414540F2FF11C2F2B05114D1884279
:107B50003BDC7F21C1F65051884200F38380022133
:107B6000C0F23041884200F0E0814021C1F620118E
:107B7000884200F0DA81A5E088423BDC3F21C1F673
:107B8000201188427CDC012800F0CF810221C0F264
:107B90003041884200F0C9810421C0F6600188426A
:107BA00000F0C381C6E0B0F1004F3FF488AF20F091
:107BB000010006283FF483AF4CF21E10C0F600000F
:107BC00040F6D421FBF790FB79E740F2FF71C2F653
:107BD0003061884268DC40F20021C2F2B051884234
:107BE00000F0A38140F20041C2F60021884200F07B
:107BF0009C8167E040F6FF71C3F26021884200F388
:107C0000848040F20021C2F2B051884200F08D81A0
:107C100040F20041C2F60021884200F0868140F621
:107C20000001C2F63061884200F07F8182E04CF2B0
:107C30001E10C0F6000040F6D221FBF755FB0EE700
:107C4000B0F5407F3FF438AF40F2063188423FF450
:107C500033AF4CF21E10C0F6000040F6D321FBF704
:107C600043FB29E78021C1F65051884200F05D8135
:107C700040F20011C2F28011884200F0568121E0EA
:107C80004021C1F62011884200F04F818021C1F6C9
:107C90005051884200F0498140F20011C2F2801137
:107CA000884200F0428145E040F60001C2F63061B2
:107CB000884200F03A8144F20001C3F6C0218842B4
:107CC00000F03381D9F8002002F130414FEA31232E
:107CD000062B40F6E42100F27683DFE813F007007C
:107CE000750074037403B000DA0011010F21C1F2B2
:107CF000C001884249DC0421C0F66001884200F0DE
:107D000014810821C0F6904148E041F20001C3F21D
:107D10006021884200F0098144F20001C3F6C021CD
:107D2000884200F0028148F20001C3F6F061884207
:107D300000F0FB80D9F8002002F130414FEA3123F6
:107D4000062B4FF42E6100F23E83DFE813F00700AC
:107D500043033C033C038803C50302044FF6FF7151
:107D6000CCF68331884240F302830F21C1F2C00177
:107D7000884200F30D830021CCF68431884200F064
:107D8000D4800821C0F690410BE31021C1F2C0015C
:107D9000884200F0CA802021C1F2F041884200F000
:107DA000C480A2F1A041A1F580714FEA3123052BD7
:107DB00040F6E42100F20783DFE813F00600050334
:107DC000050341006B00A2001F21C1F2F04188426F
:107DD0000FDC0421C0F66001884200F0A680082173
:107DE000C0F69041884200F0A0801021C1F2C0018D
:107DF00010E02021C1F2F041884200F0968041F26B
:107E00000001C3F26021884200F08F8042F200013D
:107E1000C3F29061884200F0888040F20061C5F2B0
:107E200000018A426CD040F20051C5F200018A4242
:107E30002FD040F20041C5F200018A4272D10F21D9
:107E4000C1F2C00188420EDD1021C1F2C00188429A
:107E50006BD02021C1F2F041884266D048F2000187
:107E6000C3F6F06107E00421C0F6600188425CD0EF
:107E70000821C0F69041884257D040F20061C5F217
:107E800000018A423CD040F20051C5F200018A4212
:107E900048D11F21C1F2F04188420FDD41F6FF7148
:107EA000C3F29061884217DC2021C1F2F041884280
:107EB0003BD041F20001C3F2602117E00421C0F67B
:107EC0006001884231D00821C0F6904188422CD010
:107ED0001021C1F2C00109E042F20001C3F2906139
:107EE000884222D048F20001C3F6F06188421CD0DB
:107EF00040F20831C5F2000101F53E718A4211D10C
:107F000041F20001C3F2602188420ED042F200012A
:107F1000C3F29061884208D048F20001C3F6F061D4
:107F2000884202D040F6E4214DE299F85800012839
:107F300003D1022001B0BDE8F0830121D9F800008F
:107F400089F858108168490732D4D5E900121F26F4
:107F5000C2F3012300EB83031F6B02F01F02964064
:107F6000C1F38461B74391403943196381688268E2
:107F700001F0040102F00802891840F0CC802F685B
:107F800000F114010422C7F34066AB6802EAD7523D
:107F900051F82640C7F304560727B740B3F1004F06
:107FA00024EA07070CD18F50096841F000410DE029
:107FB000D9F85C0040F02000C9F85C000120D0E155
:107FC000B3403B438B50096821F000414161D5E942
:107FD0000412C36804290BD1016E006E2968C0F336
:107FE00084604A034AD091FAA1F1B1FA81F147E0E5
:107FF000062707EA93039A402B6800EB8100016E85
:108000004FF20007C0F2FF3703F0F84339401A433C
:10801000114341F000410166A86940F08070B0F161
:10802000807F07D04CF21E10C0F6000040F61C31D5
:10803000FBF75AF9287F022807D34CF21E10C0F62E
:10804000000040F61D31FBF74FF9D9F8000029690F
:108050006030AA6950F8213023F080731A4340F849
:10806000212029692A7F50F82130012A23F000734A
:1080700008BF03F1007340F821304CE0C1F3846184
:1080800088424FF6FF70C0F2070005D1D9F8001002
:108090000A6E22F000420A66D9F800104A6E496E54
:1080A0002A68C1F38461024257D092FAA2F2B2FA6E
:1080B00082F2914205D1D9F800104A6E22F00042B6
:1080C0004A66D9F800108A6E896E2A68C1F3846105
:1080D000024247D092FAA2F2B2FA82F2914205D15C
:1080E000D9F800108A6E22F000428A66D9F8001092
:1080F000CA6ECA6E29680142C2F3846037D091FA11
:10810000A1F1B1FA81F1884205D1D9F80000C16E20
:1081100021F00041C166D9F800008168C90740F02C
:108120008E802A68EF684FF6FF71C0F20701D0F821
:10813000B060134607F018046FF3DF4321FA04F42C
:108140009E43144026434745C0F8B06077D19BB1A9
:1081500092FAA2F2B2FA82F20FE0C2F38462914282
:10816000A9D0AEE7C2F384629142B9D0BEE7C1F3B1
:1081700084618842C9D0CEE7920E013202F01E031C
:108180002A68092B02EA01030AD80BB192FAA2F27B
:108190002A680A420FD092FAA2F2B2FA82F20BE0F7
:1081A0000BB192FAA2F22A680A4213D092FAA2F212
:1081B000B2FA82F20FE0920E013202F01F032A6837
:1081C00001270A4207FA03F113D092FAA2F2B2FA97
:1081D00082F20FE0920E013202F01F032A6801279B
:1081E0000A4207FA03F10DD092FAA2F2B2FA82F231
:1081F00009E0920E013202F01F0202EB420241EA54
:1082000002510DE0920E013202F01F02002302EB38
:108210004202CFF6206303EB0252114341F000719A
:10822000C1F3406300EB8300AA684369C1F30451C2
:1082300007278F40BB4302FA01F1194341612B68C4
:108240000020C8F20800034200F08A8040F2083C97
:10825000C5F2000CD9F800600CF58062ACF502752F
:108260001046AE4204BF40F20830C5F20000B6F13D
:10827000A04F04BF40F20830C5F20000016800279B
:10828000CCF22137BB4201F0E07E04D01024C9F2C9
:10829000C004A3422FD10C022DD440F20061C5F2DC
:1082A00000018E4202D0B6F1A04F59D1016821F0F1
:1082B000E07141EA0E0141F40001016041F2807079
:1082C000C1F20000006842F663518009C0F23E51DD
:1082D000A0FB0101880900EB40000C2101EB8000AC
:1082E00000900098E0B300BF00980138009000981B
:1082F0000028F9D134E00024CCF25274A34208BF24
:108300005FEA1E6417D00020CCF6843083424FF021
:10831000000008BF11F4800123D1B6F1A04F13D0A3
:1083200040F20010C5F20000864219D0701BB0FA6E
:1083300080F0400909E0016821F0E07141EA0E0196
:1083400041F0807101600BE00120002818BF6246F7
:10835000106820F0E07040EA0E0040F480001060E9
:108360000020002189F8581001B0BDE8F08342F2E6
:108370000001CBF2906188423FF4D7AD0021CCF2EE
:10838000213188423FF4D1AD0021CCF2527108E096
:108390001021C1F2C00188423FF4C7AD2021C1F2D3
:1083A000F04188423FF4C1ADA2F1A041A1F5807136
:1083B0004FEA3123052B4FF42E6104D8DFE803F098
:1083C0000A03034F8CC94CF21E10C0F60000FAF7E6
:1083D0008BFFAAE50F21C1F2C00188420FDD41F6F3
:1083E000FF71C3F29061884219DC1021C1F2C00113
:1083F00088423FF49AAD2021C1F2F04119E00021FA
:10840000CCF2293188423FF490AD0021CCF68C317A
:1084100088423FF48AAD0821C0F6904109E042F25B
:108420000001C3F2906188423FF47FAD0021C4F2A5
:10843000527188423FF479AD40F20061C5F200010B
:108440008A4200F0868040F20051C5F200018A4263
:1084500042D040F20041C5F200018A4276D10721A4
:10846000C0F6904188420EDD1F21C1F2F0418842E2
:108470001ADC0821C0F6904188423FF456AD102125
:10848000C1F2C00119E042F20001CBF298618842CA
:108490003FF44BAD0021CCF2527188423FF445AD20
:1084A0000021CCF6843108E02021C1F2F04188425D
:1084B0003FF43BAD0021C4F2213188423FF435AD99
:1084C00040F20061C5F200018A4242D040F2005100
:1084D000C5F200018A4239D10F21C1F2C0018842A0
:1084E0000FDD41F6FF71C3F29061884219DC102163
:1084F000C1F2C00188423FF418AD2021C1F2F04121
:1085000019E00021CCF25A7188423FF40EAD0021EF
:10851000CCF6843188423FF408AD0821C0F6904182
:1085200009E042F20001C3F2906188423FF4FDACE1
:108530000021C4F2213188423FF4F7AC40F2083107
:10854000C5F2000101F53E718A4202D04FF42E615E
:1085500039E74FF6FF71CCF2517188424FF42E612A
:108560000FDD41F6FF72C3F29062904219DC0022E7
:10857000CCF2527290423FF4D8AC0022CCF6843256
:1085800019E00822C8F6904290423FF4CEAC102287
:10859000C9F2C00290423FF4C8AC2022C9F2F042B6
:1085A00009E042F20002C3F2906290423FF4BDAC97
:0E85B0000022C4F2213290423FF4B7AC03E740
:0285BE00FEE7D6
:1085C000B0B582B004460020019020680D4600F14D
:1085D00030404FEA302006284BD8012101FA00F044
:1085E00010F0730F45D07F2D0BD00020C4F27F0018
:1085F000854206D04DF63630C0F600008521FAF7E8
:1086000073FE94F85800012802D1022002B0B0BDD8
:10861000012084F858002046FFF74AF9E16D10B1B7
:1086200041F0100133E041F2021291430231E16561
:10863000216805F080438A6822F0404222F03F0220
:108640001A4402F100428A604DF60262C0F204024E
:108650008B68B3F1FF3F16DC019B01330193019B53
:108660009342F5D3E06D40F0100020F002010120AC
:108670000DE04DF63630C0F600008421FAF734FEE6
:108680007F2DB2D1BDE7E16D012262F30101E16509
:0A869000002184F8581002B0B0BDBC
:02869A00FEE7F9
:10869C002DE9F0419CB00446006840F2004740F4DC
:1086AC008060C5F200071546B8420E4607D04DF65D
:1086BC003630C0F6000040F26531FAF70FFE607FED
:1086CC00022807D34DF63630C0F6000040F2663172
:1086DC00FAF704FE206B4FEAB020042807D34DF6BE
:1086EC003630C0F6000040F26731FAF7F7FD94F827
:1086FC003800022807D34DF63630C0F600004FF490
:10870C005A71FAF7EBFD20688168490703D494F895
:10871C005810012903D102201CB0BDE8F08140F2B1
:10872C0000180121C5F2000884F858100021B0F19E
:10873C00A04F1891199104D0B8420FD108F5806060
:10874C0000E0404601902046FFF7E8F890B1B0B148
:10875C00002184F858101CB0BDE8F0810020019075
:10876C00E16D41F02001E16584F8580001201CB056
:10877C00BDE8F08101A8FFF7D1F80028E8D1226804
:10878C00606DE16D40F60173994301F58071E1650F
:10879C0043F2997147F609274FF0000CC0F600011F
:1087AC00C0F60007C4F860C047F61123C0E90B17E8
:1087BC0040F20C71C0F60003C5F200011C274363A4
:1087CC0008F50373424508BF1946176084F858C072
:1087DC005768B2F1A04F08BF194647F01003536019
:1087EC0032462B4600F0C2FB21688A6822F0004218
:0E87FC0022F03F0204328A601CB0BDE8F0811A
:02880A00FEE787
:10880C0070B582B00446006840F2004640F48060C7
:10881C00C5F20006B0420D4607D04DF63630C0F614
:10882C00000040F64C01FAF759FD2868092800F2BF
:10883C008480012101FA00F040F2EF2108427CD043
:10884C00286890B16868002818BFB0F5004F2BD18C
:10885C00A8684FEA30200C2807D34DF63630C0F606
:10886C00000040F65101FAF739FD94F85800012840
:10887C0002D1022002B070BD0120002384F8580000
:10888C0001930093226840F2080CC5F2000CB2F17F
:10889C00A04F0CF1F80013D0B2421ABF00210123F3
:1088AC000CF59F6173B13EE0B0F5404FD0D04DF662
:1088BC003630C0F600004FF40561FAF70FFDC7E73C
:1088CC00014683BB89689368194349072BD44FF43D
:1088DC00E061D5F800E0824208BF4FF44071B2F17C
:1088EC00A04F08BF4FF440715CF80100BEF1000FBF
:1088FC0020F460402AD06E6894F8383042F48072CC
:10890C0046EA4333184340F20013C5F200039A427F
:10891C004CF801002CD1DCF80000DCF800211043ED
:10892C00C0074CD12EE0E06D40F02000E065012046
:10893C00002184F8581002B070BD4DF63630C0F6E8
:10894C00000040F64D01FAF7C9FC79E740F200133C
:10895C0042F48072C5F200039A424CF801001BD11C
:10896C00DCF80000DCF800211043C00727D11DE023
:10897C00DCF80004DCF80025DCF800361043184362
:10898C00C0071CD15CF8010040F61F72AB68904325
:10899C00184340EA0E000EE0DCF80004DCF8002579
:1089AC00DCF8003610431843C00708D15CF801000E
:1089BC0040F61F7290434CF801000020B8E70020ED
:0289CC00B6E70C
:0289CE00FEE7C2
:1089D0000138010E01D0012070474EF21001CEF295
:1089E000000148604EF62350CEF20000F0220270E3
:0A89F0000020072288600A6070472B
:0289FA00FEE796
:1089FC0060B310B50446006843F20001C4F20201F2
:108A0C00884206D04CF2EE10C0F600007021FAF746
:108A1C0065FC607F20B9002020772046FAF7DAF950
:108A2C00022060772079022806D34CF2EE10C0F6B3
:108A3C0000007E21FAF752FC207948B1D4E90212E9
:108A4C00204600F0B5F868B1012010BD0120704738
:108A5C00206841F6B751C0F2C1414161816821F0F3
:108A6C00180181606079022806D34CF2EE10C0F632
:108A7C0000009021FAF732FC6079002814BF2069BD
:108A8C004FF0FF30616922684FEA711104291061BF
:108A9C0006D34CF2EE10C0F600009C21FAF71EFC37
:108AAC002068D4E90512836842F0800223F0600349
:108ABC001943802A816006D04CF2EE10C0F60000FB
:108ACC00A021FAF70BFC2068A169226A8368013A9D
:108ADC0023F080031943032A816006D34CF2EE1075
:108AEC00C0F60000A521FAF7F9FB01206077002001
:028AFC0010BDAB
:028AFE00FEE791
:108B000010B593080ED0D0F800E04FF0000C00BF75
:108B100051F80C40013B24BA0CF1040CCEF8004093
:108B2000F6D101E04FF0000C02F00302DFE802F0A2
:108B30001C02071111F80C100268117014E001EB0F
:108B40000C0211F80C105278036842EA01211980D6
:108B50000AE001EB0C0211F80C105378046843EAA8
:0E8B600001212180917821700068006810BD0D
:028B6E00FEE720
:108B7000B0B505460220687728682B6A8468012B07
:108B800044F00104846010D0022B0AD0032B10D1D2
:108B90002AB100BF51F8043B013A0360FAD10068E2
:108BA00008E02846FAF7AEFE04E02846FFF7A8FFE3
:0A8BB00000E0002001216977B0BD4C
:028BBA00FEE7D4
:108BBC00F0B581B04FEAF20714460D46042F064675
:108BCC0006D34EF2EE00C0F600005F21FAF786FBEA
:108BDC00E8070BD10120002232B131684D618A685F
:108BEC0022F0180222438A6001B0F0BD1F2100BFA1
:108BFC0049B1013901F01F0025FA00F0C007F7D088
:108C0C00032F04D9E6E74FF0FF31032FE2D8002001
:108C1C000122DFE807F002030C15DDE710294FF005
:108C2C00000238BF01220F2988BF0120D4E7082990
:108C3C004FF0000238BF0122072988BF0120CBE783
:108C4C0007294FF0000238BF0122062988BF0120F6
:028C5C00C2E76D
:028C5E00FEE72F
:108C6000D0B12DE9F0410446006840F20741C4F25A
:108C70000201884212DC5721C4F20201884222DC40
:108C80002F21C4F20201884238DC0821C4F202011B
:108C9000884257D01C2150E00120704740F25741D4
:108CA000C4F2020188421ADC40F22F41C4F20201F0
:108CB00088422ADC40F20841C4F20201884241D0D5
:108CC00040F21C4139E07F21C4F20201884225DCD8
:108CD0005821C4F20201884234D06C212DE040F2C8
:108CE0007F41C4F2020188421FDC40F25841C4F2C5
:108CF0000201884226D040F26C411EE03021C4F2CD
:108D0000020188421ED0442117E040F23041C4F2F3
:108D10000201884216D040F244410EE08021C4F2A4
:108D2000020188420ED0942107E040F28041C4F253
:108D30000201884206D040F29441C4F20201884206
:108D400040F0D780A068002818BF102840F0AD8000
:108D5000E06840F04000402806D04CF20E40C0F6DB
:108D60000000A521FAF7C0FA206940F080008028B1
:108D700006D04CF20E40C0F60000A621FAF7B4FA75
:108D80006069002818BFB0F5807F40F09A80A06924
:108D9000002818BFB0F5806F40F09F80E06940F078
:108DA0002000202806D04CF20E40C0F60000A92179
:108DB000FAF79AFA206A4FEA3030042806D34CF2C8
:108DC0000E40C0F60000AA21FAF78EFA60687428F7
:108DD00006D34CF20E40C0F60000AC21FAF784FA3C
:108DE00040F2000CC4F2020C20684FF6F8330CF588
:108DF0008162CBF6FD73904238BF03F5806303EBCD
:108E000000024CF6CD43CCF6CC43A2FB03230CF579
:108E100080616FF00302D4E90287D4F810E03CBF10
:108E20000021C4F2020102EA9302C4E910120221F5
:108E300084F82510016847F6F072914304F114029A
:108E400041EA08016CCA394341EA0E011143194352
:108E5000294331430160204600F054F8A06804F132
:108E60004801B0F5804F04BF0020606060680EC903
:108E7000C7B2013803280F60536009D8204600F0BC
:108E800067F804F1540007C8002303604A6003E058
:108E90000020C4E91500E06500200121E06384F8AA
:108EA000251084F82400BDE8F081B0F5804F3FF430
:108EB0004FAF4CF20E40C0F60000A421FAF714FAAE
:108EC00046E7B0F5007F3FF462AF4CF20E40C0F6CB
:108ED0000000A721FAF708FA59E7B0F5006F3FF450
:108EE0005DAF4CF20E40C0F60000A821FAF7FCF985
:108EF00054E74CF20E40C0F60000A321FAF7F4F953
:028F000020E768
:028F0200FEE788
:108F040080B501684CF6CD4301F0FC02083ACCF67A
:108F1400CC43A2FB032C40F20842C4F20202D0F874
:108F240044E002F58363914238BF02F57E732EF06C
:108F3400030103EB010ECCF30413012102F58F624C
:0A8F44009940C0E912E2016580BD0A
:028F4E00FEE73C
:108F5000017940F600120139C4F2020202EB8103EA
:108F600002F1400C01F01F01012202FA01F1C0E9F7
:068F7000153CC1657047CD
:028F7600FEE714
:108F7800F0B581B016464FF6FF720F46591EC0F283
:108F880003021D469142044607D34CF20E40C0F638
:108F9800000040F2AB11FAF7A3F994F82400012875
:108FA80020D0012084F8240094F82500012816D147
:108FB800022084F825000020E0632068324601681A
:108FC8002B4621F00101016020463946FAF7B4FC2E
:108FD8002068226B016842B141F00E010BE00020CD
:108FE80084F82400022001B0F0BD21F004010160E2
:108FF800016841F00A010160A06C0168C90342BF21
:10900800016841F480710160606D00281EBF01682D
:1090180041F4807101602068016841F0010101603C
:06902800002001B0F0BDC4
:02902E00FEE75B
:10903000014690F82500022827D180B50868D1E9BB
:1090400010CE8A6C036823F00E030360136823F4C8
:1090500080731360026822F0010202600EF01F00AC
:10906000012202FA00F0CCF80400D1E9132050608C
:10907000486D30B1026822F480720260D1E91602B4
:1090800042600020BDE8804002E00420C863012067
:0E909000012281F82520002281F8242070475B
:02909E00FEE7EB
:1090A00090F82510022930D180B50168D0E910CEA2
:1090B000826C0B6823F00E030B600B6823F0010336
:1090C0000B60116821F4807111600EF01F02012104
:1090D00001FA02F2CCF80420D0E913325A60426D52
:1090E00032B1136823F480731360D0E91623536000
:1090F00080F82510826B002180F824100AB1904777
:109100000021BDE88040084670470421C163012169
:0E911000002280F8251080F8242008467047C1
:02911E00FEE76A
:10912000B0B5D0E910C30268DCF8001003F01F03EB
:109130000424D2F800E09C400C4218BF1EF0040545
:109140001AD102249C400C4218BF1EF002051FD108
:10915000D94009071BD51EF0080118D0116821F06D
:109160000E011160012101FA03F2CCF80420C16361
:1091700080F82510416B18E0116889065EBF116800
:1091800021F004011160CCF80440016B91B9B0BD2D
:109190001168890606D4116821F00A0111600121C5
:1091A00080F82510CCF80440C16A0022002980F81C
:0A91B0002420ECD0BDE8B0400847D1
:0291BA00FEE7CE
:1091BC0042F20800C4F20200C168B1F1FF3F01DDC8
:1091CC000020704740F22311C4F26751016048F649
:0E91DC00AB11CCF6EF510160C068C00F7047B8
:0291EA00FEE79E
:1091EC0042F20C00C4F202008168490001D4002054
:1091FC00704742F63B21C0F61901016046F67F61CB
:0E920C00C4F65D4101608068C0F38070704759
:02921A00FEE76D
:10921C0042F21400C4F20200016841F08041016086
:0E922C000068012100F0804081EA90707047D8
:02923A00FEE74D
:10923C002DE9F04F85B004460068402807D34EF264
:10924C00DB60C0F6000040F23B11FAF747F841F240
:10925C004C79C1F2000999F80000012803D10220D1
:10926C0005B0BDE8F08F0120002589F80000C9F891
:10927C000450207842F2140B47F2E058C4F2020B6F
:10928C00C1F6FF78C0074FF6FF7A00F08080D4E972
:10929C000175E668042F56D8032F54D0B8F8000097
:1092AC00504504D0B8F80000B0F5007F31D18020D3
:1092BC00854207D34EF2DB60C0F600004FF42A71F2
:1092CC00FAF70CF8B8F80000504504D0B8F80000D4
:1092DC00B0F5007F2AD18020864207D34EF2DB60A6
:1092EC00C0F6000040F2A921F9F7F8FF4FF47A70AC
:1092FC00FAF72EFD08B1012549E0042F3AD8DFE832
:10930C0007F003302B39350045EA0640CBF818003E
:10931C0030E0B8F8000050454FF02000C8D0B8F845
:10932C000010B1F5807F08BF4020C1E7B8F80000FD
:10933C0050454FF02000CFD0B8F80010B1F5807F29
:10934C0008BF4020C8E74EF2DB60C0F6000040F2D8
:10935C00A721F9F7C3FFA1E745EA0640CBF838008F
:10936C0008E045EA0640CBF81C0003E045EA06405D
:10937C00CBF83C00DBF8000040F40030CBF80000E8
:10938C004FF47A70FAF7E4FC050018BF0125207839
:10939C00800701D42F461EE02669AA2E18BFBB2ECB
:1093AC003CD14FF47A70FAF7D3FC012798B9DBF86B
:1093BC000C0020F0FF003043CBF80C00DBF8000071
:1093CC0040F40030CBF800004FF47A70FAF7C0FC90
:1093DC00002808BF2F462078400740F1E680D4E9EA
:1093EC0005654FF6FF71701EC0F20101884207D36C
:1093FC004EF2DB60C0F6000040F21931F9F76EFF57
:10940C004FF47A70FAF7A4FC08B10127CDE0F0070D
:10941C0004970ED10020039000211AE0CC2EC0D06E
:10942C004EF2DB60C0F600004FF43A71F9F756FFCC
:10943C00B7E705F4E060B0F5A06F039007D34EF2E8
:10944C00DB60C0F6000040F22F31F9F747FF4FF414
:10945C00E06106F0060341EAC32106F4805341EAB9
:10946C00830106F0780741EA473706F0800147EAA6
:10947C00413705EAC620029705F4000700F4805036
:10948C0005F480120197770705F4005E009248BF3F
:10949C007044002B05F4804B18BF5844370705F473
:1094AC00803848BF4044F70605F4003C48BF40EA0A
:1094BC000C00B70605F4802948BF40EA090077067E
:1094CC0005F4002A48BF40EA0A000029009B18BF97
:1094DC001843B305019B48BF184305F08072730510
:1094EC0048BF104305F0007E320548BF40EA0E002D
:1094FC0005F0806705F00061B20448BF3843720480
:10950C0048BF0843039940EA01074FF0607106F425
:10951C00C04001EA863141EA40303104029901EB46
:10952C00000808D441F24C7942F2140BC1F2000944
:10953C00C4F2020B16E041F24C7942F2140B15F016
:10954C00405AC1F20009C4F2020B07D14EF2DB60A3
:10955C00C0F6000040F2BB31F9F7C0FE47EA0A073B
:10956C0048F0405805F0804116F4803018BF0F4386
:10957C00DBF80C1048EA803021EA00003843CBF8C5
:10958C000C00DBF8000040F40030CBF800004FF486
:10959C007A70FAF7DDFB47F2E058049FC1F6FF78CA
:1095AC004FF6FF7A002818BF01272078000740F1FA
:1095BC00E080D4E90865AE4200F0DB80E0690497F6
:1095CC00029000F00300039001384746022807D3AD
:1095DC004EF2DB60C0F600004FF47D71F9F77EFEB1
:1095EC0040F2000AC0F6040AB6F1006F0AF58028B2
:1095FC000CD338884FF6FF71884240461EBF39683D
:10960C004FF0006061F39920864207D34EF2DB6085
:10961C00C0F6000040F2F631F9F760FEB5F1006FCC
:10962C000BD338884FF6FF7188421EBF38684FF055
:10963C00006860F39928454507D34EF2DB60C0F60D
:10964C00000040F2F731F9F749FE4FF47A70FAF75F
:10965C007FFB10B1B846012789E00020C4F201005D
:10966C0001683888C905039AB8464FF6FF710AD4C9
:10967C0088424FF0006111D0D8F800004FF0006A1A
:10968C0060F3582A0AE0884251461EBFD8F8000001
:10969C004FF0006160F358214FF0006ADBF80C00CA
:1096AC004002029800F0004012D4012A21D1DBF8CC
:1096BC00102047F6FF7306F178419A4342EA1111E4
:1096CC00CBF8101005F1784109090BF1140233E0C5
:1096DC00012A1FD1DBF8103047F6FF77721ABB4313
:1096EC0043EAD202691ACBF81020C9080BF1140214
:1096FC0022E0022A26D1DBF8302047F6FF7306F170
:10970C0078419A4342EA1111CBF8301005F17841B7
:10971C0009090FE0022A15D1DBF8302047F6FF7358
:10972C00A6EB0A019A4342EAD101CBF83010A5EB23
:10973C000A01C9080BF13402136847F6FF77BB43E3
:10974C0019431160DBF8141021F000410843CBF8E9
:10975C001400DBF8000040F40030CBF800004FF4AC
:10976C007A70FAF7F5FA049F002818BF01274FF614
:10977C00FF7A2078800654D5D4E90B65701E022838
:10978C0007D34EF2DB60C0F6000040F26541F9F7FA
:10979C00A5FDB8F80000504504D0B8F80000B0F5AD
:1097AC00007F1DD18020854207D94EF2DB60C0F6C8
:1097BC00000040F26641F9F791FD4FF47A70FAF728
:1097CC00C7FA08B101272CE0022E16D0012E1BD1AE
:1097DC00DBF85C0020F0FF002843CBF85C0013E0C2
:1097EC00B8F8000050454FF02000DCD0B8F800105D
:1097FC00B1F5807F08BF4020D5E7DBF8600020F092
:10980C00FF002843CBF86000DBF8000040F4003088
:10981C00CBF800004FF47A70FAF79AFA002818BFC8
:10982C0001272078C00601D438462AE0A46A6FF4D8
:10983C008030044207D04EF2DB60C0F6000040F2EC
:10984C009A41F9F74BFD4FF47A70FAF781FA002838
:10985C004FF0010015D1DBF85C0020F48030204380
:10986C00CBF85C00DBF8000040F40030CBF80000D3
:10987C004FF47A70FAF76CFA01460120002908BF00
:0E988C003846002189F8001005B0BDE8F08FC5
:02989A00FEE7E7
:10989C002DE9F04F85B0039000F138404FEAB0202D
:1098AC0007280D46019006D34EF23E70C0F600001C
:1098BC00A921F9F713FD2868010C01D180B230B948
:1098CC004EF23E70C0F60000AA21F9F707FD686859
:1098DC00B0F5881F80F20781122800F21E81012149
:1098EC0001FA00F00F21C0F20601084200F01581C8
:1098FC002868002800F0F480039A4FF0000902F168
:10990C002001009141F20041C4F600018A424FF05F
:10991C00060208BF052201994FF0030C4FF0000816
:10992C004FF0000B052938BF0A4602920BE000BF2E
:10993C0028680BF1010B30FA0BF108F1020809F160
:10994C00040900F0CD80012101FA0BFA10EA0A0794
:10995C00EED0686800F00300013801281FD8E868D1
:10996C00042808D34EF23E70C0F60000BB21F9F774
:10997C00B5FC4FF0030C039B0CFA08F198686A686D
:10998C008843E96801FA08F1084398605868C2F303
:10999C00001120EA0A0001FA0BF1084358606868CC
:1099AC0000F00300032815D0A868032808D34EF252
:1099BC003E70C0F60000CC21F9F790FC4FF0030C80
:1099CC00039B0CFA08F1D868AA68884302FA08F1DC
:1099DC000843D860686800F00300022827D101987A
:1099EC00072808D34EF23E70C0F60000D921F9F7D3
:1099FC0075FC4FF0030C2869102808D34EF23E700A
:109A0C00C0F60000DA21F9F769FC4FF0030C6FF097
:109A1C000300009C00EA5B00215809F01C020F2394
:109A2C002E699340994306FA02F211432150039B8D
:109A3C000CFA08F118686A68884302F0030101FA0D
:109A4C0008F1084312F4403F18603FF471AF41F243
:109A5C006001C4F20201086840F2004440F00100C9
:109A6C0008600868C4F2010400F001000490049836
:109A7C002BF003004FF608462044CFF6FF768159B1
:109A8C0009F00C020F2393409943029B03FA02F254
:109A9C0011438151A068696840EA070240F20C4604
:109AAC00CB0258BF20EA0702A260C4F2010630685C
:109ABC008B0240EA070258BF20EA07023260606856
:109ACC008B0340EA070258BF20EA07026260206855
:109ADC00C90340EA070258BF20EA0702226027E7C1
:109AEC0005B0BDE8F08FB0F5081F0CDAB0F5881F93
:109AFC003FF4FEAEB0F5901F3FF4FAAEB0F5041F84
:109B0C003FF4F6AE09E03FF4F3AEB0F5441F3FF47A
:109B1C00EFAEB0F5481F3FF4EBAE4EF23E70C0F620
:0A9B2C000000AB21F9F7DAFBE2E6D6
:029B3600FEE748
:109B3800B0B50C46054639B94EF23E70C0F6000085
:109B48004FF4BD71F9F7CCFB2869204018BF0120FC
:029B5800B0BD9E
:029B5A00FEE724
:109B5C00B0B50C46054639B94EF23E70C0F6000061
:109B6C0040F2B311F9F7BAFB686900EA040124EA80
:0A9B7C00000040EA0140A861B0BDFE
:029B8600FEE7F8
:109B880040F21441C4F201010A68024214BF08609D
:069B98007047F9F735BC2F
:029B9E00FEE7E0
:109BA00088B110B50446006847F2FF71C4F20001A5
:109BB00088420ADC45F20041C4F20001884218D014
:109BC00045F6000109E00120704747F60001C4F2A4
:109BD000000188420DD048F20041C4F200018842E1
:109BE00007D04CF20660C0F600004FF40871F9F798
:109BF0007BFBA068B0F5806F07D34CF20660C0F61F
:109C0000000040F22121F9F76FFBE06801380228DB
:109C100007D34CF20660C0F6000040F22221F9F7AB
:109C200063FB206940F40040B0F5004F07D04CF2D0
:109C30000660C0F6000040F22321F9F755FB606989
:109C4000B0F5807F07D34CF20660C0F600004FF4F9
:109C50000971F9F749FBA069082807D34CF206609F
:109C6000C0F6000040F22521F9F73EFBE06940F420
:109C70000020B0F5002F07D04CF20660C0F60000BF
:109C800040F22621F9F730FB206A40F40030B0F5AD
:109C9000003F07D04CF20660C0F6000040F22721DA
:109CA000F9F722FB94F8410028B9002084F840001D
:109CB0002046F9F7DBF9242084F8410094E80310EA
:109CC000E368026821F0706122F001020260016124
:109CD0008168012B21F4004181604FF4044108BFE9
:109CE0004FF4004141EA0C0181604168022B21F4EC
:109CF000006108BF01F500614160416841F00071F9
:109D000041F400414160C16821F40041C16004F1A7
:109D100010010EC9114341EA0321C160D4E90712C1
:109D200011430160016841F0010101600020202120
:0E9D3000606484F84110206384F8420010BD86
:029D3E00FEE73E
:109D40002DE9F04190460446006847F2FF72C4F2E4
:109D500000021D4690420F4608DC45F20041C4F265
:109D60000001884216D045F6000107E047F60001E1
:109D7000C4F2000188420DD048F20041C4F2000153
:109D8000884207D04CF20660C0F6000041F67141EF
:109D9000F9F7AAFA069E002D18BFB5F1807F38D1D9
:109DA00043F6FF70C8F2000086420CDC42F200006D
:109DB000C8F20000864215D042F20040C8F200000E
:109DC00086420FD006E044F20000C8F2000086424E
:109DD00008D03EB14CF20660C0F6000041F6734177
:109DE000F9F782FA6FF39F2721684FF4806347EAFF
:109DF000084003EA565328434A6883F07C433043C3
:109E000083F41C4320F000401A4010434860BDE832
:109E1000F081B5F1007FC3D04CF20660C0F60000BF
:0A9E200041F67241F9F760FABAE763
:029E2A00FEE751
:109E2C002DE9F04F81B00D46591E89B21E461746DA
:109E3C000229044607D34CF20660C0F6000040F637
:109E4C006A21F9F74BFA94F8410020280DD1DDF87E
:109E5C0028A0BAF1000F0CD0DDF82C80B8F1000F5F
:109E6C0007D094F8400001280AD1022001B0BDE8C7
:109E7C00F08F4FF400706064012001B0BDE8F08FEA
:109E8C00012084F84000F9F7B1FB814620464FF4DD
:109E9C00004101221923CDF80090FAF77FF8014612
:109EAC00012011B101B0BDE8F08F0C9942F20042D3
:109EBC002220C8F2000284F8410040204FF0000B31
:109ECC0084F84200C4F844B0C4F824A09246A4F824
:109EDC002A808846A2F5806CF2B2204629460023DF
:109EEC00C4F834B0CDF800C0FFF724FF204641463B
:109EFC004A46FAF7A1F8B0B92068012E08D0390A01
:109F0C008162204641464A46FAF796F858B92068CD
:109F1C00F9B281622046402100224346CDF80090E0
:109F2C00FAF73CF810B184F840B0A5E7608DB0F5B5
:109F3C00807F07D3FF20208520462946FF224FF043
:109F4C00807306E0608D29462085C2B220464FF012
:109F5C000073CDF800A0FFF7EDFE0026FF270BE005
:109F6C00608D29462085C2B220464FF000730096C2
:109F7C00FFF7E0FE608D90B320460421002243469B
:109F8C00CDF80090FAF70AF800287FF475AF206836
:109F9C00616A406A0870606A218D01306062481EF7
:109FAC002085618D01396185618D0029E2D0000425
:109FBC00E0D12046802100224346CDF80090F9F7ED
:109FCC00EDFF00287FF458AF608DB0F5807FC7D3CC
:109FDC00278520462946FF224FF08073C7E720468D
:109FEC0041464A46FAF75EF800287FF445AF2068F0
:109FFC002021C16142684EF60003CFF600631A407F
:10A00C004260002084F8411084F8420084F840003B
:06A01C0001B0BDE8F08F69
:02A02200FEE757
:10A02400B0B50446006847F2FF72C4F200029042E1
:10A034000D4608DC45F20041C4F20001884215D007
:10A0440045F6000107E047F60001C4F2000188422A
:10A054000CD048F20041C4F20001884206D04EF20E
:10A064004F10C0F600006321F9F73CF96FF48050FB
:10A07400054206D04EF24F10C0F600006421F9F7F5
:10A0840031F994F84100202803D194F840000128C4
:10A0940001D10220B0BD242084F841002068016869
:10A0A40021F001010160016821F48051016001681F
:10A0B40029430160016841F001010160202084F816
:0AA0C4004100002084F84000B0BD08
:02A0CE00FEE7AB
:10A0D000B0B50446006847F2FF72C4F20002904235
:10A0E0000D4608DC45F20041C4F2000188420ED062
:10A0F00045F6000107E047F60001C4F2000188427E
:10A1000005D048F20041C4F2000188422BD1102D45
:10A1100006D34EF24F10C0F600009221F9F7E4F892
:10A1200094F84100202803D194F84000012801D17F
:10A130000220B0BD242084F841002068016821F08D
:10A1400001010160016821F4706141EA05210160AB
:10A15000016841F001010160202084F841000020E5
:10A1600084F84000B0BD4EF24F10C0F600009121BF
:0AA17000F9F7BAF8102DCCD2D2E7AF
:02A17A00FEE7FE
:10A17C0000285AD0B0B50446006843F20001C4F27E
:10A18C000001884206D04EF29D70C0F60000B52149
:10A19C00F9F7A4F86068072806D34EF29D70C0F654
:10A1AC000000B621F9F79AF8A068B0F5805F06D3E5
:10A1BC004EF29D70C0F60000B721F9F78FF8E068F9
:10A1CC00B0F5805F06D34EF29D70C0F60000B8214A
:10A1DC00F9F784F894E807004CF6CC43036045F299
:10A1EC005553036041608260F9F700FA2168CA6830
:10A1FC00520710D0054603E02168C86840070AD012
:10A20C00F9F7F4F9401B3228F6D32068C0684007F0
:10A21C00F2D00320B0BD0A69E068824206BF4AF65C
:0EA22C00AA20086008610020B0BD0120704724
:02A23A00FEE73D
:10A23C0001220168C0F8D022002280F8C822B1F8AF
:10A24C00540040F00100A1F85400B1F8540040F063
:0AA25C0002020020A1F85420704710
:02A26600FEE711
:10A2680047F20000C4F20000016841F48071016007
:02A2780070472D
:02A27A00FEE7FD
:10A27C0010B547F200040028C4F200043DD0B0F53C
:10A28C00007F10D0B0F5806F06D04EF2D210C0F621
:10A29C0000009D21F9F722F82068022161F34A2081
:10A2AC002060002010BD2068D4F8801000F4C0603D
:10A2BC0041F48071B0F5806FC4F88010F1D1206842
:10A2CC00012161F34A20206041F28070C1F200004C
:10A2DC000068322250434DF68362C4F21B32A0FB5D
:10A2EC00020201EB924000216369013841F1000246
:10A2FC005B052BD5002AF7D128E02068D4F8801014
:10A30C0000F4C06021F48071B0F5806FC4F8801047
:10A31C00C7D12068012161F34A20206041F280708E
:10A32C00C1F200000068322250434DF68362C4F241
:10A33C001B32A0FB020201EB924000216369013841
:10A34C0041F100025B0501D5002AF7D16069400597
:06A35C00A7D5032010BD8F
:02A36200FEE714
:10A3640047F20800C4F20000016841F48041016032
:02A37400704730
:02A37600FEE700
:10A3780000285CD02DE9F04182B00446006850B155
:10A3880010F02F0007D14CF6C600C0F6000040F2CE
:10A398004511F8F7A5FF207841F20006C007C4F27E
:10A3A800020646D12078800767D42078000700F19C
:10A3B800A3802078400740F18D81A068052805D842
:10A3C800012101FA00F010F0230F07D14CF6C60066
:10A3D800C0F600004FF4FA71F8F782FFB06D5FEA3B
:10A3E800C00808D4B06D40F08050B065B06D00F082
:10A3F80080500190019847F20007C4F200073868BE
:10A40800C00500F1CB80386840F480703860F9F7F7
:10A41800EFF805463868C00500F1C080F9F7E8F89C
:10A42800401B0228F6D9032002B0BDE8F0810120C4
:10A4380070476068002818BFB0F5803F40F0A180E1
:10A44800B06800F00C01F068082978D0032281F088
:10A458000C0122EA00000844B0FA80F040096ED1ED
:10A4680065683068B5F5A02F00F0B580B5F5803F78
:10A4780040F0B88040F48030BAE0E06840F4807082
:10A48800B0F5807F07D04CF6C600C0F600004FF448
:10A49800C071F8F725FF2069802807D34CF6C6005D
:10A4A800C0F6000040F28111F8F71AFFB068F168B1
:10A4B80000F00C0004284BD001F0030180F00C00E0
:10A4C80081F002010844B0FA80F0400940D1E16807
:10A4D8003068002900F0A78040F480703060F9F7F8
:10A4E80087F805463068400500F1B280F9F780F832
:10A4F800401B0228F6D9D6E06069022807D34CF63B
:10A50800C600C0F600004FF4E471F8F7E9FE61698F
:10A51800D6F8940000294BD040F00100C6F894000A
:10A52800F9F766F8054600BFD6F8940080073FF5AE
:10A5380040AFF9F75DF8401B0228F5D9B3E0306861
:10A5480080037FF52FAF606800287FF42BAF0DE103
:10A558003068400503D5E068002800F0078170687E
:10A56800216920F0FE4040EA0160706041F26C70A1
:10A57800C1F200000068F9F711F8002840F0F680F1
:10A5880013E7B0F5A02F3FF45BAF4CF6C600C0F65A
:10A59800000040F24B11F8F7A3FE51E7A568D6F882
:10A5A8009000052D5CD0012D63D140F0010068E0DA
:10A5B80020F00100C6F89400F9F71AF8054600BF24
:10A5C800D6F8940080077FF5F4AEF9F711F8401B30
:10A5D8000228F5D967E040F480203060306840F404
:10A5E800803005E020F480303060306820F480202E
:10A5F8003060F8F7FDFF002D054610D03068800365
:10A608003FF5D0AEF8F7F4FF401B6428F6D94AE0CE
:10A61800F8F7EEFF401B64284FF0030015D83068A8
:10A628008003F5D4BEE620F480703060F8F7E0FFD0
:10A63800054600BF306840057FF5B7AEF8F7D8FF8C
:10A64800401B02284FF00300F4D902B0BDE8F081A6
:10A658007068216920F0FE4040EA01607060A4E65D
:10A6680040F00400C6F89000D6F8900040F00100D1
:10A6780007E020F00100C6F89000D6F8900020F01E
:10A688000400C6F89000F8F7B3FF002D054641F224
:10A69800883714D0D6F89000800714D4F8F7A8FFAC
:10A6A800401BB842F6D9032002B0BDE8F08100BFD4
:10A6B800F8F79EFF401BB8424FF00300C5D8D6F804
:10A6C80090008007F4D4B8F1000F5EBFB06D20F0A1
:10A6D8008050B065207880064CD4E069032807D301
:10A6E8004CF6C600C0F600004FF41971F8F7F8FDF3
:10A6F800E069002800F02781B16801F00C010C29FD
:10A708005CD1012832D0F068216A00F003028A4245
:10A718002CD1626A6FF00F0300F0F00103EB021214
:10A72800914223D1A16A00F4FE4209028A421DD156
:10A73800E16A00F07842C9068A4217D1226B0023E9
:10A74800CFF6E07303EA025200F4C001A2F500124A
:10A7580091420BD1616B4FF07E4202EA016100F039
:10A76800C06001F17E41884200F0ED80012002B016
:10A77800BDE8F081A069022807D34CF6C600C0F6F0
:10A78800000040F23B21F8F7ABFDA169D6F898002C
:10A7980000296ED040F00100C6F89800F8F728FFAD
:10A7A800054600BFD6F89800800796D4F8F720FF32
:10A7B800401B02284FF00300F4D946E702286CD169
:10A7C800206A032801D8012807D14CF6C600C0F634
:10A7D800000040F26E21F8F783FD606A0138102806
:10A7E80007D34CF6C600C0F6000040F26F21F8F718
:10A7F80077FDA06A0838782807D34CF6C600C0F65B
:10A8080000004FF41C71F8F76BFDE06A02381E284F
:10A8180007D34CF6C600C0F6000040F27121F8F7E5
:10A828005FFD206B082800F29280012101FA00F0F8
:10A8380010F4AA7F00F08B80606B082800F29080EB
:10A84800012101FA00F010F4AA7F00F08980306835
:10A8580020F080703060F8F7CBFE05463068800144
:10A868002DD5F8F7C5FE401B02284FF00300F5D997
:10A87800EBE620F00100C6F89800F8F7B9FE0546A7
:10A88800D6F8980080077FF528AFF8F7B1FE401B8F
:10A8980002284FF00300F3D9D7E6306820F0807023
:10A8A8003060F8F7A5FE04463068800144D5F8F713
:10A8B8009FFE001B02284FF00300F5D9C5E6F0689B
:10A8C80048F20C01C0F29F1100EA010C04F12001CA
:10A8D8008EC96FF00F00D4E90C5400EB021000226F
:10A8E800CFF6E07241EA0C0102EA05520843A2F5EC
:10A8F80000124FF07E4540EA032005EA0465104344
:10A9080005F17E4540EAC7602843F060306840F0B2
:10A9180080703060F06840F08070F060F8F768FE92
:10A928000446306880010ED4F8F762FE001B022846
:10A938004FF00300F5D988E6F0684FF6FC71CFF6C2
:10A94800EE610840F060002002B0BDE8F0814CF6EE
:10A95800C600C0F6000040F27221F8F7C1FC6BE7B0
:10A968004CF6C600C0F6000040F27321F8F7B8FCB8
:02A978006DE789
:02A97A00FEE7F6
:10A97C002DE9F047002800F03381044600680D46AD
:10A98C000F2802D810F00F0007D14CF6C600C0F605
:10A99C00000040F20B31F8F7A1FC102D07D34CF658
:10A9AC00C600C0F600004FF44371F8F797FC42F272
:10A9BC00000AC4F2020ADAF8000000F00F00854227
:10A9CC000DD9DAF8000020F00F002843CAF8000077
:10A9DC00DAF8000000F00F00A84240F00181207866
:10A9EC0041F20808C007C4F202080CD14FF000096C
:10A9FC002068810759D4B9F1000F77D0D8F800003E
:10AA0C0020F0F00070E060680138032807D34CF6A2
:10AA1C00C600C0F6000040F22331F8F75FFC616815
:10AA2C0058F8080C022900F0D980032940F0DB808B
:10AA3C00800140F1D580D8F80400D8F8041000F05B
:10AA4C000300032842F20040C1F30311C0F2F400EA
:10AA5C00D8F8042001F1010104BF47F64000C0F210
:10AA6C007D10B0FBF1F0D8F80410C2F3062250436D
:10AA7C00C1F34161022202EB4101B0FBF1F04BF258
:10AA8C000041C0F2C44188420CD9D8F8000010F043
:10AA9C00F00F00F0B3802078800703D5A068002861
:10AAAC0000F0AC804FF00009B1E0410742BFD8F88C
:10AABC00001041F4E061C8F80010000706D5D8F882
:10AACC000000072161F30D20C8F80000A0686FF0AA
:10AADC00070101EB3011082980F0B780D8F800008D
:10AAEC00A16820F0F0000843C8F80000DAF8000074
:10AAFC0000F00F00854219D2DAF8000020F00F00A8
:10AB0C002843CAF80000F8F771FD064641F2883771
:10AB1C00DAF8000000F00F00A84207D0F8F766FD45
:10AB2C00801BB842F4D90320BDE8F0872078400799
:10AB3C0019D5E0686FF0030101EB302104290AD329
:10AB4C004FEA302038B14CF6C600C0F600004FF486
:10AB5C006771F8F7C3FBD8F80000E16820F4E060F7
:10AB6C000843C8F80000207800071AD520696FF058
:10AB7C00030101EB302104290AD34FEA302038B10C
:10AB8C004CF6C600C0F6000040F2A331F8F7A6FB65
:10AB9C00D8F80000216920F4605040EAC100C8F8E0
:10ABAC000000F9F7CFFCD8F800104FF20802C1F3FF
:10ABBC000311C0F60002515C41F2807201F01F01DA
:10ABCC0020FA01F141F26C70C1F200000068C1F290
:10ABDC0000021160BDE8F047F8F7DEBC800304D436
:10ABEC000120BDE8F0874005FAD5F9F7ABFC4BF234
:10ABFC000041C0F2C44188427FF654AFD8F800003F
:10AC0C00082161F307104FF00109C8F80000D8F8CB
:10AC1C000000616820F003000843C8F80000F8F752
:10AC2C00E5FC064641F28837D8F80000616800F070
:10AC3C000C00890088423FF4DBAEF8F7D7FC801B90
:10AC4C00B842F1D90320BDE8F0874FEA3010002854
:10AC5C003FF444AF4CF6C600C0F6000040F27A3127
:06AC6C00F8F73CFB3AE79B
:02AC7200FEE7FB
:10AC740041F2807041F20801C1F20000C4F2020105
:10AC8400006809684FF21802C1F30221C0F60002FD
:0AAC9400515C01F01F01C840704739
:02AC9E00FEE7CF
:10ACA00041F2807041F20801C1F20000C4F20201D9
:10ACB000006809684FF21802C1F3C221C0F6000211
:0AACC000515C01F01F01C84070470D
:02ACCA00FEE7A3
:10ACCC0088B310B50446406840F04000402807D0D7
:10ACDC004CF66A10C0F6000040F23511F8F7FEFA97
:10ACEC00A068802807D34CF66A10C0F600004FF419
:10ACFC009B71F8F7F3FAE068B0F5004F07D34CF608
:10AD0C006A10C0F6000040F23711F8F7E7FA206934
:10AD1C00B0F5800F09DB14D0B0F5C00F11D0B0F135
:10AD2C00806F0ED005E00120704750B1B0F5001FC8
:10AD3C0007D04CF66A10C0F600004FF49C71F8F77F
:10AD4C00CDFA606940F00040B0F1004F07D04CF6EE
:10AD5C006A10C0F6000040F23911F8F7BFFAA0698A
:10AD6C0040F48010B0F5801F07D04CF66A10C0F686
:10AD7C0000004FF49D71F8F7B1FAE06940F08040A3
:10AD8C00B0F1804F07D04CF66A10C0F6000040F2CC
:10AD9C003B11F8F7A3FA206A40F00050B0F1005FC5
:10ADAC0007D04CF66A10C0F600004FF49E71F8F70D
:10ADBC0095FA94F8250028B9002084F82400204640
:10ADCC00F8F794FA022084F825002068C168C906B7
:10ADDC000CD4CA214162532141622046F9F7BAFED4
:10ADEC0058B108B32168FF224A6200E00020002815
:10ADFC0004BF012184F8251010BD94E8035082692A
:10AE0C0022F08E6222F04002826122691143A26913
:10AE1C0083691143194381614EEA0C41016120465B
:10AE2C0000F012F80028DDD12168D4F814C0D4E960
:10AE3C0007E28B6923F060431A4342EA0E0242EAAE
:06AE4C000C028A61CEE752
:02AE5200FEE719
:10AE540010B504460068C16821F08001C1608169B1
:10AE6400890609D42046F9F79FFE00280EBF00206A
:10AE7400032084F8250010BD816921F0200181613F
:10AE84002046F9F791FE00281ABF032084F8250014
:0EAE9400002021688A6942F020028A6110BD08
:02AEA200FEE7C9
:10AEA40010B50C46202907D34EF61230C0F6000028
:10AEB40040F2FC71F8F716FA42F20050C4F20000B6
:06AEC40050F8240010BD4F
:02AECA00FEE7A1
:10AECC00A8B1B0B50446006842F6FF71C4F20101A6
:10AEDC0088420EDC43F60001C4F2000188421CD00B
:10AEEC0043F60041C4F20001884216D00DE0012067
:10AEFC00704743F20001C4F2010188420DD043F6C1
:10AF0C000041C4F20101884207D04CF6DA10C0F6B9
:10AF1C00000040F24711F8F7E1F9606850B1B0F564
:10AF2C00827F07D04CF6DA10C0F600004FF4A47103
:10AF3C00F8F7D4F9A068002818BFB0F5806F40F07E
:10AF4C008680E068A0F540704FEA30200D2807D3CA
:10AF5C004CF6DA10C0F600004FF4A571F8F7BEF904
:10AF6C00A069002818BFB0F5007F7DD1606B40F060
:10AF7C000800082807D04CF6DA10C0F600004FF491
:10AF8C00A671F8F7ABF9E0694FEAF000082807D38F
:10AF9C004CF6DA10C0F6000040F24D11F8F79EF9AD
:10AFAC00206A40F08000802807D04CF6DA10C0F6FA
:10AFBC0000004FF4A771F8F791F9606A40F01000A7
:10AFCC00102807D04CF6DA10C0F6000040F24F11F2
:10AFDC00F8F784F9606A80B1E0694FEAF00008285C
:10AFEC0007D34CF6DA10C0F6000040F26111F8F706
:10AFFC0075F90020C4E9040045E0206940F0020026
:10B00C00022807D04CF6DA10C0F600004FF4A971F4
:10B01C00F8F764F96069022807D34CF6DA10C0F629
:10B02C00000040F25311F8F759F96068B0F5827FCF
:10B03C0027D1E0694FEAF000082824D34CF6DA1047
:10B04C00C0F6000040F25711F8F748F91BE0B0F5D4
:10B05C00004F3FF476AF4CF6DA10C0F6000040F229
:10B06C004911F8F73BF96CE7B0F5802F3FF47EAF50
:10B07C004CF6DA10C0F6000040F24B11F8F72EF93E
:10B08C0074E70020E0610025A56294F85D0020B90A
:10B09C00204684F85C50FBF787FF022084F85D00A3
:10B0AC002068D4F80CE00268BEF5E06F22F0400294
:10B0BC0002604EF4006298BF0125B2F5706F1CBFA0
:10B0CC000023A3624FEA053CD4E90135D4E90421FD
:10B0DC0003F4827305F404452B4402F002021A4473
:10B0EC00A36901F00101E569114403F400721144F4
:10B0FC0005F03802256A114405F08002A56A114456
:10B10C0005F40052114301600421626A0EF470656B
:10B11C0001EA1341636B45EA0C0502F01002294366
:10B12C0003F00803114319434160C16921F4006124
:0EB13C00C16100200121206684F85D10B0BDC5
:02B14A00FEE71E
:10B14C0070B515460E464FF4C05132462B46044698
:10B15C00F9F796FE68B9204631462A46F9F704FFFE
:10B16C0038B920464FF4C06132462B46F9F788FEB9
:10B17C0028B1206E40F020002066032070BD002016
:02B18C0070BD94
:02B18E00FEE7DA
:10B1900010B5002853D00446006844F6FF71C4F28D
:10B1A0000001884212DC44F20041C4F200018842EE
:10B1B0002BD044F60001C4F20001884225D044F6A9
:10B1C0000041C4F2000188421FD011E045F20001A5
:10B1D000C4F20001884218D048F20001C4F2000114
:10B1E000884212D043F60001C4F2010188420CD01B
:10B1F000A0694FF49F7100284EF2FC70C0F6000069
:10B2000008BF40F24311F8F76FF8D4F8880028B966
:10B21000002084F884002046FBF734FF2420C4F883
:10B2200088002068A16A026822F00102026011B160
:10B23000204600F019F82046F9F7F6FE08B1012083
:10B2400010BD2168486820F490404860886820F06C
:10B250002A008860086840F0010220460A60BDE8C4
:06B26000104000F01FB9D0
:02B26600FEE701
:10B2680010B50446806AB0F5807F07D34EF2FC70B3
:10B27800C0F6000040F6AE41F8F732F894F828001E
:10B28800000714D5A06B40F40040B0F5004F07D07C
:10B298004EF2FC70C0F6000040F6B341F8F720F813
:10B2A8002068A16B426822F400421143416094F87F
:10B2B8002800C00714D0E06A40F40030B0F5003F21
:10B2C80007D04EF2FC70C0F6000040F6BA41F8F71D
:10B2D80007F82068E16A426822F4003211434160AD
:10B2E80094F82800800714D5206B40F48030B0F51E
:10B2F800803F07D04EF2FC70C0F6000040F6C14116
:10B30800F7F7EEFF2068216B426822F48032114380
:10B31800416094F82800400714D5606B40F4802001
:10B32800B0F5802F07D04EF2FC70C0F6000040F652
:10B33800C841F7F7D5FF2068616B426822F4802284
:10B348001143416094F82800C00614D5E06B40F41E
:10B358008050B0F5805F07D04EF2FC70C0F6000058
:10B3680040F6CF41F7F7BCFF2068E16B826822F412
:10B3780080521143816094F82800800614D5206C0F
:10B3880040F40050B0F5005F07D04EF2FC70C0F6F4
:10B39800000040F6D641F7F7A3FF2068216C8268C9
:10B3A80022F400521143816094F8280040065AD5CF
:10B3B800206844F6FF31C4F20001884212DD44F6E9
:10B3C8000041C4F20001884220D045F20001C4F2D5
:10B3D800000188421AD043F60001C4F201018842F4
:10B3E80014D00BE044F20041C4F2000188420DD0B1
:10B3F80044F60001C4F20001884207D04EF2FC7006
:10B40800C0F6000040F6DD41F7F76AFF606C40F4D3
:10B418008010B0F5801F07D04EF2FC70C0F6000017
:10B4280040F6DE41F7F75CFF2068616C4268B1F5D1
:10B43800801F22F4801242EA0102426013D1A06CFC
:10B448004FEA7050042807D34EF2FC70C0F6000093
:10B4580040F6E341F7F744FF2068A16C426822F404
:10B46800C0021143416094F82800000614D5E06C2E
:10B4780040F40020B0F5002F07D04EF2FC70C0F663
:10B48800000040F6EB41F7F72BFF2068E16C4268BB
:0AB4980022F400221143416010BDB0
:02B4A200FEE7C3
:10B4A400B0B582B004460020C4F89000F8F7A2F8C2
:10B4B40021680546096809071AD56FF07E4C2046B5
:10B4C4004FF4001100222B46CDF800C0F9F794FF89
:10B4D40070B100BF206850E8000F216820F08000A0
:10B4E40041E80002002AF5D103202021882232E01D
:10B4F40020680068400725D56FF07E4C20464FF445
:10B50400800100222B46CDF800C0F9F775FFC8B1C1
:10B51400206850E8000F216820F4907041E8000290
:10B52400002AF5D12068083050E8000F216820F087
:10B534000100083141E80002002AF3D10320202150
:10B544008C2208E02020C4F88800C4F88C00002174
:10B5540070220020E166A150002184F8841002B01A
:02B56400B0BD78
:02B56600FEE7FE
:10B56800D0F88830202B09D1944600294FF00102E9
:10B5780018BFBCF1000F04D11046704702221046D4
:10B588007047B0B5002221230165A0F854C0A0F887
:10B5980056C0C0F89020C0F88830C36F13B34BF280
:10B5A8007165C0F600054BF219644BF25D6E5D6380
:10B5B8000568C0F60004C0F6000EC3E90B4E9A6396
:10B5C80005F12802044618466346FDF7D1FC0146FA
:10B5D800204639B11021C0F890102021C0F88810F9
:10B5E800012210E0016840220A6200BF01680831A8
:10B5F80051E8001F026841F08001083242E8001358
:0EB60800002BF3D10022BDE8B0401046704781
:02B61600FEE74D
:10B618000168806A0968890619D40021A0F85610C3
:10B628000168083151E8001F026821F080010832E2
:10B6380042E80013002BF3D1016851E8001F0268AB
:10B6480041F0400142E80013002BF5D17047FAF7AA
:02B6580013BD20
:02B65A004300AB
:06B65C00806A00F069BAEB
:0EB6620041F27471C1F20001096800F029B8CC
:10B67000B0B5846A2168D4F88800D4F88C50896801
:10B68000090607D5212805D10020A4F85600204638
:10B69000F9F78CFF20688068400607D5222D05D178
:10B6A0000020A4F85E00204600F01CF8D4F89000BA
:10B6B00040F010012046C4F89010BDE8B040FAF701
:02B6C0007DBC4F
:10B6C20080B50B468DF803000DF103000121012224
:10B6D20000F000FA9DF80310002808BF411E08463A
:02B6E20008BDA1
:10B6E400016851E8001F026821F4907142E80013D8
:10B6F400002BF5D14FF6FE7CCEF6FF7C02680832B3
:10B7040052E8002F036802EA0C02083343E80021E0
:10B714000029F3D1C16E01290AD100BF016851E8A3
:10B72400001F026821F0100142E80013002BF5D13C
:0EB734002021C0F88C100021C16641677047CB
:10B7420038B541F27471C1F2000104460D6802F08D
:10B7520020FF02462846214600F0C2FA013004D0FA
:0EB762000A20BDE83840FFF77BBFC04338BD6A
:10B7700070B5046840F62F03E2692168A66813409B
:10B78000202B05D101F0200306F080555B1936D13E
:10B7900040F60F0313400CD00123C1F2000306EA68
:10B7A000030C40F22013C0F200430B4013EB0C03D8
:10B7B0002BD1C36ED50616D5012B14D111F0100371
:10B7C00011D010212162A168490600F1AA80B0F8C9
:10B7D0005C10B0F85E20B0F85E30002B18BF9142CC
:10B7E00040F0358170BDD30278D516F4800375D052
:10B7F0004FF480112162BDE8704000F08DBA416FB6
:10B800000029EFD0BDE870400847D30718BF11F4F6
:10B81000807307D001232362D0F8903043F00103F6
:10B82000C0F89030930706F0010E0AD5BEF1000F64
:10B8300007D002232362D0F8903043F00403C0F80D
:10B84000903053070AD5BEF1000F07D004232362BE
:10B85000D0F8903043F00203C0F8903013070CD5B5
:10B8600001F0200353EA0C0307D008232362D0F829
:10B87000903043F00803C0F8903013050BD511F059
:10B88000806308D04FF400632362D0F8903043F017
:10B890002003C0F89030D0F89030002BA2D0920650
:10B8A0000AD501F0200106F08052891804D0416FBA
:10B8B00011B10446884720460168D0F89020896875
:10B8C00002F0280201F040010446891840F08A8005
:10B8D000FAF774FB0020C4F8900070BD130606D57B
:10B8E00001F0800306F400069B1940F0E280530645
:10B8F00040F1A48011F0400300F0A080016851E8FD
:10B90000001F026821F0400142E80013002BF5D12E
:10B910002021C0F8881000218167BDE87040FAF747
:10B92000AFBBD0F880100A6851688BB2002B4ED0A4
:10B93000B0F85C60B3424AD2A0F85E101168890684
:10B9400039D400BF016851E8001F026821F48071FA
:10B9500042E80013002BF5D10168083151E8001FBF
:10B96000026821F00101083242E80013002BF3D1F4
:10B970000168083151E8001F026821F040010832D7
:10B9800042E80013002BF3D12021C0F88C100021D5
:10B99000C16600BF016851E8001F026821F0100174
:10B9A00042E80013002BF5D1D0F880100446084679
:10B9B000FDF73EFB204602210167B0F85C10B0F8AD
:10B9C0005E20891A89B2BDE8704000F09BB8B0F8DB
:10B9D0005C1099427FF406AF126892067FF502AFC1
:10B9E000022261E0FFF77EFE216820468968490651
:10B9F00020D500BF0168083151E8001F026821F01E
:10BA00004001083242E80013002BF3D1D0F8801037
:10BA100081B145F2E150C0F6000088630846FDF7A9
:10BA20003FFB00283FF4DEAED4F88000816BBDE818
:10BA300070400847BDE87040FAF7C0BA13023FD51E
:10BA400011F080433CD0BDE8704000F0ADB9891AD8
:10BA5000026852E8002F036822F4907243E800263F
:10BA6000002EF5D14FF6FE72CEF6FF720368083352
:10BA700053E8003F06681340083646E80035002DBD
:10BA8000F4D12022C0F88C200022C266426700BF99
:10BA9000026852E8002F036822F0100243E80026F3
:10BAA000002EF5D1022289B20267BDE8704000F095
:10BAB00029B8816F00293FF495AEBDE87040084772
:10BAC000D2017FF58FAEB1F1FF3F3FF78BAEBDE8FE
:06BAD000704000F04DB9CA
:10BAD600F8B51D4617460C460646184602F0B9FC50
:10BAE600002803D407FB04F2A24201D20020F8BDCD
:0EBAF6002846314600F0F2F8B0FBF4F0F8BD3F
:02BB0400704788
:10BB060052EC10CBC2F30A5340F2FF718B4218BFBE
:10BB1600002B02D100210160704740F2FE3161F333
:0EBB26001E52A3F2FE31016042EC10CB7047BC
:02BB3400704758
:10BB36002DE9F8432DED028B8E1E00EBC6070D4650
:10BB460097ED008BD7E9022359EC108B4046494606
:10BB5600FAF73DFC53EC182B01F097FC032D41EC52
:10BB6600100B12D3741E17ED028B083F53EC102BEB
:10BB760040464946FAF72BFC53EC182B01F085FC9E
:10BB8600012E41EC100B2646ECD853EC102B404608
:10BB96004946FAF71CFC41EC100BBDEC028BBDE8E4
:02BBA600F88322
:02BBA8007047E4
:10BBAA002DE9F8430F46804600EBC10256EC109B84
:10BBBA007C1EA2F1080552E9022351EC100B01F098
:10BBCA0062FC4A463346FAF700FC022F41EC100B9E
:10BBDA002A462746ECD8D8E9002301F054FC41EC68
:06BBEA00100BBDE8F8831A
:02BBF00070479C
:10BBF20042694AB110B50446036A002B1CBF216991
:0ABC020098470020606110BD7047F4
:10BC0C00026848F20003C4F200039A4218D0B0B59F
:10BC1C00B1F1807F0CD34EF2FC72C0F600020446E8
:10BC2C0010460D4640F6AF21F7F758FB2946204643
:10BC3C000068426902F07F4211434161BDE8B040A7
:02BC4C0070473F
:0ABC4E00436A08460121FFF73FBFDB
:10BC58000168806A0968890634D40021A0F85E105A
:10BC6800016851E8001F026821F4807142E800135E
:10BC7800002BF5D10168083151E8001F026821F056
:10BC88000101083242E80013002BF3D101680831A2
:10BC980051E8001F026821F04001083242E8001311
:10BCA800002BF3D12021C0F88C10C16E012909D1D5
:10BCB800016851E8001F026821F0100142E80013F2
:10BCC800002BF5D100210167C16E012903D1B0F81D
:0ABCD8005C10FFF713BFFFF763BF16
:06BCE200006800F045B807
:10BCE800806A01210167C16E012904D1B0F85C1096
:0ABCF8004908FFF703BFFFF777BF0D
:10BD02000146C0680A6982426FEA000010449CBF83
:06BD120089680844704737
:02BD1800704772
:10BD1A002DE9F843144688460546C7684FF00009DE
:10BD2A002869F943B8420844A96898BF0844CE1B59
:10BD3A00B04238BF06466868A64228BF264638443D
:10BD4A0041463246FAF775FCA868F1190F1A18BF6E
:10BD5A000F46A41BB144B044BFF35F8FEF60DFD13D
:06BD6A004846BDE8F88325
:02BD700070471A
:10BD7200F8B540F6E413C1F2000314461B78002B19
:10BD82000D46064608BF02F084FBEFF311874FF021
:10BD9200200181F3118830462946224602F0CDFB6C
:06BDA20087F31188F8BDD3
:02BDA8007047E2
:10BDAA0084460020002918BF002A0ED0097848B21C
:10BDBA0000280BD4BCF1000F18BFCCF800100021EA
:10BDCA00C3E90011002818BF012070476FF0010075
:02BDDA007047B0
:10BDDC0010B5016844F6FF72C4F20002914212DC05
:10BDEC0044F20042C4F20002914229D044F600020F
:10BDFC00C4F20002914223D044F60042C4F2000285
:10BE0C0091421DD011E045F20002C4F200029142B1
:10BE1C0016D048F20002C4F20002914210D043F650
:10BE2C000002C4F2010291420AD04CF66E21C0F617
:10BE3C0000010446084640F23621F7F74FFA204637
:10BE4C0090F88410012901D1022010BD2421C0F8E2
:10BE5C00881001680A680B6822F0005223F0010375
:10BE6C000B60002343660A602021C0F8881080F81C
:06BE7C008430002010BD1F
:0EBE82007F298EBF6FF0010001700120704714
:10BE900001460120A1F8400000220020A1F8402026
:0ABEA000A1F84420A1F850207047DB
:10BEAA0053797374656D20636F726520636C6F6379
:0ABEBA006B3A2025754D487A0A0006
:10BEC4002DE9F04182B00DF105060C464FF0220831
:10BED4004FF47A7731463246032305468DF80580C0
:10BEE4000097F8F78DFE9DF80700314600F0070033
:10BEF40020438DF8060042208DF80500284632467E
:10BF040002230097F8F77CFE284631463246032385
:10BF14008DF805800097F8F773FE9DF80700204020
:10BF2400A04202D102B0BDE8F0814EF6F100C0F6A5
:0ABF34000000FFF704FC00BFFEE769
:10BF3E004261636B757052656769737465724461B3
:0EBF4E00746120617661696C61626C650D0042
:10BF5C000246D0F8880100219067B2F8CE00A2F812
:10BF6C007C00B2F8CC00A2F87E00D2F8D43040F2BB
:0EBF7C000000C1F20000C2F8803000F06DBB82
:10BF8A002E2E2E466C61736820756E6C6F636B651E
:02BF9A00640041
:10BF9C000246D0F8D4004FF47A73C2F88400D2F879
:10BFAC008400D2F88010401A41F2DC21C1F2000169
:10BFBC000968594391FBF0F340F20000C1F2000014
:0ABFCC000021C2F8883000F047BBE6
:10BFD600466C617368206F6220756E6C6F636B20B0
:06BFE6006572726F72002B
:10BFEC0040F20000C1F20000C16D4FF2F012CFF62A
:10BFFC00FF725143CB17C0E95813C16D4942C0F8C9
:10C00C004011C16D5143CA17C0E97812C16D494244
:06C01C00C0F8D8117047C6
:0EC02200466C61736820206C6F636B65640070
:10C03000824202D1002000B2704794469042B8BFBD
:10C040000246BCEB00009C4648BF404280B5DDF88C
:10C0500008E09942B8BF0B46BCEB010148BF49421A
:10C06000AEEB0202434301FB023191FBF0F0BDE86D
:06C07000804000B27047A1
:10C07600443A5C50726F6A656B74655C65637353B2
:10C086006D61727450726F5C7472756E6B5C6677FC
:10C096005F673437337263745C44726976657273B2
:10C0A6005C53544D3332473478785F48414C5F4493
:10C0B60072697665725C5372635C73746D33326752
:0AC0C6003478785F68616C2E630027
:10C0D000B0B504464EF61640C0F60000FFF731FB3F
:10C0E00040F2F835C1F2000541F2487105F118003F
:10C0F000C0F60001B822FAF7B0FAA868D0210130E2
:10C10000C5E9011001202870002000212A46D02313
:0EC1100000F034F82046BDE8B04000F097B8CB
:10C11E00443A5C50726F6A656B74655C6563735309
:10C12E006D61727450726F5C7472756E6B5C667753
:10C13E005F673437337263745C4472697665727309
:10C14E005C53544D3332473478785F48414C5F44EA
:10C15E0072697665725C5372635C73746D333267A9
:0EC16E003478785F68616C5F6164632E6300F3
:10C17C002DE9F04F83B0924606465818012241F241
:10C18C00F0181F4602EB901B0025C1F2000800BFFF
:10C19C008AB212FA87F23C4641EA8610402A28BF3E
:10C1AC00C1F140041AFA85F1A2B21FFA85F9CDE962
:10C1BC00001282B24046A02102234FF47A750295F8
:10C1CC00F7F7B0FF052001363F1B19FA84F5F7F796
:10C1DC0013FABBF1010B4FF00001D9D103B0BDE84C
:02C1EC00F08FD2
:10C1EE00443A5C50726F6A656B74655C6563735339
:10C1FE006D61727450726F5C7472756E6B5C667783
:10C20E005F673437337263745C4472697665727338
:10C21E005C53544D3332473478785F48414C5F4419
:10C22E0072697665725C5372635C73746D333267D8
:0EC23E003478785F68616C5F6372632E630012
:10C24C00F0B581B040F2F834C1F20004054600208C
:10C25C0000212246D023F9F76FFEA0692861A08B3C
:10C26C00A882E08BE882208C2883608CA883A08C29
:10C27C00E883E08C2884208D6884608DA5F87C0090
:10C28C00A08DA5F87E00E08DA5F89800208EA5F86D
:10C29C009A00608EA5F88C00A08EA5F8A000E08E08
:10C2AC00A5F8A80004F1380090E80F50D4E9146701
:10C2BC00C5F88000C5F88410C5F88820C5F8903002
:10C2CC00C5F89CC0C5F8A4E0C5F8AC60AF6704F134
:10C2DC00580007C8C5F89400C5F8B010C5F8B420CC
:10C2EC00B4F88800A5F85200B4F88A00A5F85000FC
:10C2FC00D4F88C00E865D4F890002866B4F8940063
:10C30C00A5F85400B4F89600A5F85600B4F89800B7
:10C31C00A5F85800B4F89A00A5F85A00B4F89C0097
:10C32C00A5F86400B4F89E00A5F86800B4F8A00065
:10C33C00A886B4F8A200E886B4F8A4002887B4F85C
:10C34C00A6006887B4F8A800A887B4F8AA00E88704
:10C35C00B4F8AC00A5F84000B4F8AE00A5F8420063
:10C36C00B4F8B000A5F84400B4F8B200A5F8460043
:10C37C00B4F8B400A5F84800B4F8B600A5F84A0023
:10C38C00B4F8B800A5F84C00B4F8BA00A5F84E0003
:10C39C00B4F8BC00A5F86A00B4F8BE00A5F86C00AF
:10C3AC00B4F8C000A5F86E00B4F8C200A5F870008F
:10C3BC00B4F8C400A5F87200B4F8C600A5F8B8002B
:10C3CC00B4F8C800A5F8BA00B4F8CA00A5F8BC00C7
:10C3DC00B4F8CC00A5F8BE00B4F8CE00A5F8C000A7
:10C3EC00E0686860A088E188227880F0D00089B28B
:10C3FC000843D1B281F00101084318BF012001B0FC
:02C40C00F0BD81
:10C40E00443A5C50726F6A656B74655C6563735316
:10C41E006D61727450726F5C7472756E6B5C667760
:10C42E005F673437337263745C4472697665727316
:10C43E005C53544D3332473478785F48414C5F44F7
:10C44E0072697665725C5372635C73746D333267B6
:0EC45E003478785F68616C5F646D612E6300F6
:10C46C00F0B581B004464EF6F410C0F60000FFF7AC
:10C47C0062F92046FFF7E4FEB4F87C0040F2F83293
:10C48C00C1F200025085B4F87E009085D4F880C0CB
:10C49C00D4F88410D4F88830B4F88C005086D4F8D2
:10C4AC009000D4F878E0D4F89450D4F8B060D4F874
:10C4BC00B4709565D6651766B4F89850D585B4F800
:10C4CC009A501586D4F89C50B4F8A0609686D4F88F
:10C4DC00A460B4F8A870D786D4F8AC70C2E9103058
:10C4EC0002F14800C2E90EC180E8E0404FF49640EA
:10C4FC004FF48031C2E906010021C2F82610C2F8BF
:10C50C00221040F2DE31A2F8881047F20011C0F27E
:10C51C0002014FF4FA13C2E923130A21A2F8941072
:10C52C006921A2F88A100221C3F2B061C2F89610F8
:10C53C0043F27001A2F89A100121C0F2020142F6F6
:10C54C00E06343F6D01702F19C0CC3F2D403C3F2A0
:10C55C00B0678CE88A004FF25421CFF6FF7101F5D9
:10C56C007A7301F5FA71A2F8BA103221A2F8B03040
:10C57C004FF63003A2F8BC104FF63001C1F27073C5
:10C58C00CFF6FF71C2F8B23041F27C5301F5E16194
:10C59C004FF6837641F27075CFF25423A2F8BE1099
:10C5AC0042F21071C0F27D06C1F27C55C2F8B63071
:10C5BC00C0F2070140F28433012702F1C00C0120C4
:10C5CC00C2E92A65C0F20103C3F2205764268CE845
:10C5DC008A00D0211084C2F8CC60516010701074A5
:10C5EC0060680021D0600020D023FFF7C1FD2046F9
:0AC5FC0001B0BDE8F040FFF723BED8
:10C60600443A5C50726F6A656B74655C656373531C
:10C616006D61727450726F5C7472756E6B5C667766
:10C626005F673437337263745C447269766572731C
:10C636005C53544D3332473478785F48414C5F44FD
:10C6460072697665725C5372635C73746D333267BC
:0EC656003478785F68616C5F6932632E630030
:10C664002DE9F04104464EF62B40C0F60000884602
:10C67400FFF765F8206940F2F836C1F20006B061B0
:10C68400A08AB8F1000FB083E08AF083208B308455
:10C69400A08B7084E08BB084208CF084608C308517
:10C6A400B4F87E00B085B4F87C007085B4F89800C6
:10C6B400F085B4F89A003086B4F88C007086B4F82B
:10C6C400A000B086B4F8A800F086D4F88000D4F8AE
:10C6D4008410D4F88820D4F89030D4F89C50D4F83E
:10C6E400A470D4F8ACC0D4F878E0B063F1633264D9
:10C6F4007364B564F764C6F850C0C6F854E0D4F85F
:10C70400940006F15803D4F8B010D4F8B42007C349
:10C71400B4F85200A6F88800B4F85000A6F88A00CD
:10C72400E06DC6F88C00206EC6F89000B4F8540092
:10C73400A6F89400B4F85600A6F89600B4F8580089
:10C74400A6F89800B4F85A00A6F89A00B4F8640061
:10C75400A6F89C00B4F86800A6F89E00A08EA6F87F
:10C76400A000E08EA6F8A200208FA6F8A400608F97
:10C77400A6F8A600A08FA6F8A800E08FA6F8AA0045
:10C78400B4F84000A6F8AC00B4F84200A6F8AE0035
:10C79400B4F84400A6F8B000B4F84600A6F8B20015
:10C7A400B4F84800A6F8B400B4F84A00A6F8B600F5
:10C7B400B4F84C00A6F8B800B4F84E00A6F8BA00D5
:10C7C400B4F86A00A6F8BC00B4F86C00A6F8BE0081
:10C7D400B4F86E00A6F8C000B4F87000A6F8C20061
:10C7E400B4F87200A6F8C400B4F8B800A6F8C600FD
:10C7F400B4F8BA00A6F8C800B4F8BC00A6F8CA0099
:10C80400B4F8BE00A6F8CC00B4F8C000B168A6F82D
:10C81400CE0001F101004FF0D001C6E901104FF044
:10C824000100307007D04EF65C70C0F60000FEF7D1
:10C8340086FF6068F06040F2F832C1F20002002026
:10C844000021D023FFF798FC2046BDE8F041FFF714
:02C85400FBBC2B
:10C85600443A5C50726F6A656B74655C65637353CA
:10C866006D61727450726F5C7472756E6B5C667714
:10C876005F673437337263745C44726976657273CA
:10C886005C53544D3332473478785F48414C5F44AB
:10C8960072697665725C5372635C73746D3332676A
:0EC8A6003478785F68616C5F7063642E6300A5
:10C8B40040F20001A0F50040C1F20001C1F8B0004F
:02C8C4007047BB
:10C8C600443A5C50726F6A656B74655C656373535A
:10C8D6006D61727450726F5C7472756E6B5C6677A4
:10C8E6005F673437337263745C447269766572735A
:10C8F6005C53544D3332473478785F48414C5F443B
:10C9060072697665725C5372635C73746D333267F9
:0EC916003478785F68616C5F7263632E630033
:10C9240010B582B09C460446ACF10300134610F1E6
:10C93400020F4FF009000A46049938BF4FF0010C6A
:10C94400022B38BF0A2000EB0C0E2046CDE900CEA6
:10C95400F5F7D8F90020A08484F82600E061C4F833
:06C964001F0002B010BD2F
:10C96A00443A5C50726F6A656B74655C65637353B5
:10C97A006D61727450726F5C7472756E6B5C6677FF
:10C98A005F673437337263745C44726976657273B5
:10C99A005C53544D3332473478785F48414C5F4496
:10C9AA0072697665725C5372635C73746D33326755
:0EC9BA003478785F68616C5F7274632E63007E
:10C9C800B0B50C460546F9F76BFB0146A01C295388
:02C9D800B0BDF0
:10C9DA00443A5C50726F6A656B74655C6563735345
:10C9EA006D61727450726F5C7472756E6B5C66778F
:10C9FA005F673437337263745C4472697665727345
:10CA0A005C53544D3332473478785F48414C5F4425
:10CA1A0072697665725C5372635C73746D333267E4
:0ECA2A003478785F68616C5F7370692E63000A
:10CA3800B0B5044610F8275FD0F8011205290DD3C8
:10CA4800F9F74CFB013009D035B140F20000C1F2D2
:10CA58000000008BA84201D10220B0BD0020C4F81C
:06CA680028022075B0BD9C
:10CA6E00443A5C50726F6A656B74655C65637353B0
:10CA7E006D61727450726F5C7472756E6B5C6677FA
:10CA8E005F673437337263745C44726976657273B0
:10CA9E005C53544D3332473478785F48414C5F4491
:10CAAE0072697665725C5372635C73746D33326750
:10CABE003478785F68616C5F756172745F65782E2B
:02CACE00630003
:10CAD00070B5014611F8273F002600F227150446DD
:10CAE000C0F82C6280F827312846012200F016F8A1
:10CAF00001462846FFF768FFC4F82C022046F9F7E4
:0ACB0000C7FAC4F82862267570BD5C
:10CB0A002D2D2D204761696E202043414C202D2D6B
:02CB1A002D00EC
:10CB1C0091F801C0BCF1100F09D0BCF1060F04D084
:10CB2C00BCF1030F05D100F011B8F9F7E5BAF9F72C
:10CB3C0013BB8CF08001831881540121901C597017
:02CB4C00704730
:0ACB4E0054736869703D25660A0003
:10CB58002DE9F04140F2000CC1F2000C002BBCF8AA
:10CB6800187018BF9F420CD10B794E7946EA0323FF
:10CB7800A3F17E0717F17E0F07D883218154032183
:10CB880014E0862181540B2110E091F80280CD78C1
:10CB980045EA082103EB010EAEF2FD1717F5FE7FFB
:10CBA80000EB020707D2832139700221104441703B
:10CBB800901CBDE8F08103243C7074007C708BB13C
:10CBC8004FEA482343EA45036344013313F8027BE1
:10CBD8008618B77013F8037C0131714502F102021F
:0ACBE800F770F3D3901CBDE8F08154
:10CBF2002D2D2D204761696E202043414C20454E4A
:06CC020044452D2D2D001C
:10CC080040F20000C1F200004FF0FF31A0F8061119
:06CC1800A0F804117047B2
:0ECC1E0064656C746120543D256620430A0055
:10CC2C0070B540F20004C1F20004B4F8740041F293
:10CC3C003035C1F2000598B1B4F8740001281ABF60
:10CC4C00B4F874000022012240F20040C4F6000047
:10CC5C004FF40061F7F782F9B4F87400288070BDC6
:10CC6C00288800284FF6FF7018BFA4F80601B4F806
:10CC7C00061119B1B4F80611814249D1D4F8D80083
:10CC8C00A18E884205DA4EF694400126C0F60000CB
:10CC9C0031E0D4F8E400B4F93C104FF47A7251430B
:10CCAC00884205DA4EF698700226C0F6000022E0A3
:10CCBC00B4F9CE00B4F94810884205DD4DF21A20C3
:10CCCC000326C0F6000016E0B4F9CC00B4F9481005
:10CCDC00884205DD04264EF67340C0F600000AE0DB
:10CCEC00B4F9CE00B4F94C10884254DA4EF63A201E
:10CCFC000526C0F60000FEF71EFD40F20040C4F60B
:10CD0C0000004FF400610022A4F80661F7F726F941
:10CD1C00B4F8060100289FD0D4F8D800E18E8842E0
:10CD2C009ADDD4F8E400B4F93C104FF47A72514314
:10CD3C00884291DDB4F9CE00B4F94A108842BFF6AE
:10CD4C008BAFB4F9CC00B4F94A108842BFF684AF6B
:10CD5C00B4F9CE00B4F94E1088427FF77DAFB4F928
:10CD6C00CC00B4F94E1088427FF776AFB4F80601C8
:10CD7C0002283FF471AFB4F8060107283FF46CAFFA
:10CD8C004DF27220C0F60000FEF7D5FC0020A4F88E
:10CD9C000601012258E7B4F9CC00B4F94C108842D2
:06CDAC00B6DA062697E747
:0ACDB20052656620493D25660A001F
:10CDBC0070B540F20004C1F20004B4F8760041F200
:10CDCC002E35C1F2000598B1B4F8760001281ABFCF
:10CDDC00B4F876000022012240F20040C4F60000B4
:10CDEC004FF48051F7F7BAF8B4F87600288070BD8C
:10CDFC00288800284FF6FF7018BFA4F80401B4F877
:10CE0C00041119B1B4F80411814255D1D4F8D800E9
:10CE1C00218F884205DD4EF6C8700126C0F6000051
:10CE2C003DE0D4F8E400B4F93E104FF47A7251436B
:10CE3C00884205DD4EF6B0700226C0F600002EE0EA
:10CE4C00B4F9CE00B4F94010884205DD4DF226301D
:10CE5C000326C0F6000022E0B4F9CC00B4F940106F
:10CE6C00884205DD4EF6D6400426C0F6000016E0DA
:10CE7C00B4F9CE00B4F94410884205DA4EF65D20C0
:10CE8C000526C0F600000AE0B4F9CC00B4F9441051
:10CE9C00884211DA4EF6B5400626C0F60000FEF7C1
:10CEAC004AFC40F20040C4F600004FF480510022CE
:10CEBC00A4F80461F7F752F8B4F80401002893D0F1
:10CECC00D4F8D800618F8842BFF68EAFD4F8E40056
:10CEDC00B4F93E104FF47A7251438842BFF684AFD6
:10CEEC00B4F9CE00B4F942108842BFF67DAFB4F964
:10CEFC00CC00B4F942108842BFF676AFB4F9CE003C
:10CF0C00B4F9461088427FF76FAFB4F9CC00B4F98E
:10CF1C00461088427FF768AFB4F8040102283FF44A
:10CF2C0063AFB4F8040107283FF45EAF4DF26630EE
:10CF3C00C0F60000FEF7FFFB0020A4F8040101225C
:02CF4C004AE7B2
:10CF4E004552524F52204144535F313236305F4981
:0ECF5E006E7075744D757853656C6563740064
:10CF6C0070B540F20004C1F20004B4F8BC0041F208
:10CF7C002035A0F10A06B4F8BC00D4F8D4100A305D
:10CF8C008142C1F200051CD9B4F8500141F26F7115
:10CF9C00884216D82878A0B94EF68020C0F600003A
:10CFAC00FEF7C9FB01202870B4F8C0004FF4005103
:10CFBC00B0FA80F0420940F60000C4F60000F6F723
:10CFCC00CDFFD4F8D400B04203D22878012808D081
:10CFDC001EE0B4F8500141F27171884218D32878E0
:10CFEC00B0B14EF6E870C0F60000FEF7A4FB0020CE
:10CFFC002870B4F8C02040F60000002A18BF0122A7
:10D00C00C4F600004FF40051BDE87040F6F7A6BF1F
:02D01C0070BDE5
:10D01E0046697273742073746172742064657465EA
:06D02E006374656421003B
:10D03400F0B581B040F20005C1F20005D5F8000159
:10D04400B5F8BC104FF47A7740F60004794341F206
:10D054001C36C4F600048842C1F2000613DD3078A1
:10D0640088B94EF68B20C0F60000FEF768FB01205D
:10D074003070B5F8C0004FF40051B0FA80F04209A6
:10D084002046F6F76FFFD5F80001B5F8BE107943D6
:10D09400884216DA3078A0B14EF6F470C0F600007B
:10D0A400FEF74DFB00203070B5F8C0202046002A62
:10D0B40018BF01224FF4005101B0BDE8F040F6F76B
:06D0C40051BF01B0F0BDF8
:0ED0CA0075617274206572726F72200A0D001B
:10D0D800B0B540F2000441F22A30C1F20004C1F2B6
:10D0E8000000B4F9CE10B0F90000A0F5FA7088423B
:10D0F8005CDBB4F9CC10884258DB41F22830C1F22D
:10D108000000B4F9CE10B0F9000000F5FA708842BA
:10D118004CDCB4F9CC10884248DC41F22630C1F22C
:10D128000000B4F9CE10B0F90000A0F5FA708842FA
:10D138003CDBB4F9CC10884238DB41F22230C1F232
:10D148000000B4F9CE10B0F9000000F5FA7088427A
:10D158002CDCB4F9CC10884228DC41F22C30C1F226
:10D168000000D4F8E410B0F900204DF6F0054FF0B7
:10D17800FF33CFF6FF754FF47A70C2FB00536A1A7B
:10D1880073EBE17112DB41F21E33C1F20003D4F8F4
:10D19800E410B3F90030002542F21072C3FB0025F9
:10D1A8004FEAE17C881A7CEB05001DDA41F2243550
:10D1B800C1F20005287800B1B0BD4EF6F740C0F6C0
:10D1C8000000FEF7BAFA01202870B4F8C000B0FADF
:10D1D80080F0420940F60000C4F600004FF4005108
:10D1E800BDE8B040F6F7BCBE41F22435C1F20005F7
:10D1F80028780028E0D14DF29A30C0F60000FEF7FA
:10D208009CFA00202870B4F8C020002A18BF012218
:02D21800E0E74D
:10D21A004F5554505554535F4C56505F5348554ED2
:10D22A00545F4F56455254454D50455241545552FC
:02D23A004500AD
:10D23C0040F20000C1F20000B0F8BA00032803D895
:10D24C00DFE800F0020F0B0D40F60000C4F6000002
:10D25C004FF400510022F6F781BEFFF7E5BEFFF751
:06D26C0035BFFFF77DBE97
:0ED272004F5554505554204C5650204F4B00F1
:10D2800040F20000C1F2000040F20A2101800021BA
:10D290004FF0FF324FF0010C4FF00043C0F8241163
:10D2A000C0F82011A0F81421C0F80C21C0F81021FA
:10D2B000A0F81C21A0F81E21A0F81821A0F81A211E
:10D2C000A0F808C041818181C0F8E8306FF00043C8
:10D2D000C0F8EC304FF4004348F20002A0F8D03020
:10D2E00047F6FF73CFF6FF72A0F8D230C0F8DC200B
:10D2F000C0F8E030A0F882110321A0F826C0018513
:10D3000005214185612180F8A011622180F8A111D9
:10D31000792180F8B6117A2180F8B7114FF47A712B
:06D32000A0F8D6117047D1
:10D326004F5554505554535F4F56505F5348554EC2
:10D33600545F4F56455254454D50455241545552EF
:02D346004500A0
:10D3480040F20000C1F20000D0F84811D0F848219E
:0ED35800002948BF5242C0F81021F8F75DBF0F
:0ED366004F5554505554204F5650204F4B00F9
:10D3740040F20000C1F20000016E4FF46162A1FBB3
:10D384000212C0E95C120021C0E95A11C0F8481128
:06D39400C0F820117047F3
:10D39A00415558206F66662028416C61726D204D98
:06D3AA006F6465290D000F
:10D3B0004EF68850CEF20000016841F47001016021
:02D3C0007047B4
:10D3C20053756E646179004D6F6E646179005475B6
:10D3D2006573646179005765646E65736461790091
:10D3E2005468757273646179004672696461790088
:0AD3F20053617475726461790000E4
:10D3FC0041F20C0CC4F2020C5CF8041C42F2004228
:10D40C00C1F3810341F28071C0F2F402C1F2000158
:10D41C00DFE803F02928020743F20062C0F26E1223
:10D42C0020E0DCF80000DCF8003000F003000228FB
:10D43C0043F20060C3F30313C0F26E1003F1010357
:10D44C0008BF1046DCF80020B0FBF3F0DCF800302D
:10D45C00C2F306225043C3F34162022303EB4202A0
:10D46C00B0FBF2F20A605CF8040C4FF20802C0F355
:10D47C000310C0F60002105C0A6822FA00F0086083
:02D48C007047E7
:02D48E002E006E
:10D4900030B591EA030F00F18280841A71EB030C1E
:10D4A00005D2121953EB0C03001B71EB0C0140F277
:10D4B000000CCFF6E07C1CEA430F52D0BCEB410FCE
:10D4C0005FD90C0DA4EB135E5FF0010C6CF31F51E0
:10D4D0006CF31F53DEF1200C2AD303FA0CF540192C
:10D4E00041F1000122FA0EF5401923FA0EF56941C7
:10D4F00012FA0CF2CD0208D349085FEA30005FEA65
:10D50000320228BF42F00102641C641E5FEA500C24
:10D5100072F1004250F1000051EB04514FF400133E
:10D5200013EB410F38BF30BD6FF31301002030BD46
:10D53000BEF1200EBEF1200F1ED223FA0EF54019C7
:10D5400041F10001CEF1200C124218BF012203FA72
:10D550000CF52A43CEE711EA5C0F04BF002000213E
:10D5600030BD1CEA410F04BF01F00041002030BD76
:10D5700001F00041002030BD21F4801101EB045185
:10D5800030BD004218BF41F00101BCEB410F08BFA4
:10D5900030BD4FF0FE4141F47801002030BD83F0F2
:10D5A0000043841A71EB030E07D28EF0004E001B6D
:10D5B00071EB0E01121953EB0E0340F2000CCFF683
:10D5C000E07C1CEA430FC6D0BCEB410F72D90C0DB6
:10D5D000A4EB135EC90241EA5051C00241F0004180
:10D5E000DB0243EA5253D20243F00043DEF1200C47
:10D5F00041D312FA0CF522FA0EF203FA0CF542EAC4
:10D60000050218BF42F0010223FA0EF3801A994175
:10D61000E30AC4F30A0411F0404F03D418D0641E87
:10D6200040004941641E23D44205C00A40EA4150EB
:10D63000C90A51EAC3715FEA500C72F1004250F11D
:10D64000000051EB045130BD01002FD00020203CE0
:10D650000029F9D0B1FA81FCDCF1200E11FA0CF1AD
:10D6600030FA0EF510FA0CF02943A4EB0C04D9E7BC
:10D670000020D90730BDAEF1200EBEF1200F0DD233
:10D68000CEF1200C03FA0CF533FA0EF32A4318BF3F
:10D6900043F00103C01A61F10001B9E721F0004134
:10D6A000C00A40EA4150C90A01EB045130BD0020D4
:10D6B000002130BD004218BF41F00101BCEB410F19
:0ED6C0007FF467AFBCEB430F3FF463AF30BDA8
:01D6CE00005B
:10D6D0002DE9F04391EA030E0EF0004E40F20007F0
:10D6E000CFF6E07717EA41051EBFBD4217EA4305B2
:10D6F000BD4200F09F807F0D17EA135623EA47537F
:10D7000043F4801317EA115521EA475141F480117F
:10D71000AD1B05F2FD354FEAD31C1CF1010C4FF097
:10D720000047B7FBFCF77F01A2FB079C0024E3FB4B
:10D7300007C4D9F100096CEB4C0CA0FB0762002078
:10D74000E1FB072000275FEAC628E0FB0987760D8A
:10D7500046EAC226520DF61900277A41E0FB0C6218
:10D760005FEAC823E2FB09375FEA585848EAC6284F
:10D77000760D18EB070800214E41E2FB0C8602EB08
:10D78000C020DA02E6FB09215B0D43EAC8235FEA09
:10D7900058585B18002758EB0708E6FB0C38D102F5
:10D7A000E8FB0917520D42EAC3225B0DD21900278C
:10D7B0007B41E8FB0C2308EBC6265FEAC128E3FBAC
:10D7C0000987490D41EAC221520DC91942F10002EF
:10D7D000E3FB0C12470019EB08095CEB010C72EB40
:10D7E000040453EBC62047EB56530026B3F5000F55
:10D7F0007641AD19B61CD6F1200910FA09F4F040B3
:10D8000013FA09F21043F340E40F001943F1000347
:10D81000B3F5001F24BF5B086D1C40F2FE77BD42CC
:10D8200004D24EEA05511944BDE8F0832D4224D5B7
:10D83000714626E0004218BF41F00101124218BFB4
:10D8400043F00103B7EB410F2CBFB7EB430F1BE0D5
:10D85000B7EB410F04BFB7EB430F15E017EA410FD9
:10D8600004BF17EA430F0FE017EA410FE0D017EAB1
:10D87000430F02D0B7EB430FDAD04EF0FE4141F434
:10D8800070010020BDE8F08340F20001C7F6F87196
:02D89000F7E7B8
:10D8920057726F6E6720706172616D657465727325
:10D8A2002076616C75653A2066696C652025732067
:0DD8B2006F6E206C696E652025640D0A0004
:0DD8BF004144533132363020496E69740007
:10D8CC00C1F30A5340F21E42D21A0EDD202A0AD8A6
:10D8DC00CB0243EA505040F00040D04090EAE17057
:10D8EC00B0EBE1707047002070474B00004218BF4E
:10D8FC0043F0010313F5001F88BF21F0004111F024
:0AD90C00004058BF6FF00040704764
:10D9160053484F52545F434952435549545F5052FE
:09D926004F54454354494F4E0093
:10D92F002E2E2E466C617368206F6220756E6C6FA1
:05D93F00636B6564004C
:10D9440010F0004160B148BF40420A0D02F21D428E
:10D95400B0FA80F3D21A9840C30A400503EB02518F
:02D9640070470A
:10D966002E2E2E44697361626C65206C6F636B208A
:10D9760070726F636573732066696E697368656438
:01D9860000A0
:10D98700466C617368204F7074696F6E6279746555
:10D997002070726F6772616D6D206661696C656476
:01D9A700007F
:10D9A80070B5CC1760406140001BA141DD176A408B
:10D9B8006B40521BAB4100F023F862406340121BDE
:0ED9C800A3416C4060406140001BA14170BD56
:10D9D6002E2E2E466C617368206C6F636B20616C13
:0DD9E6007265616479206163746976650083
:10D9F3002E2E2E456E61626C65206C6F636B206505
:05DA030072726F720059
:10DA0800002B35D129B9B0FBF2FC0CFB12026046A1
:10DA18007047914215D22DE9F041B2FA82F39A404B
:10DA28009940D3F1200C30FA0CFC51EA0C019840D3
:10DA380000F04EF8280036FA03F200210023BDE872
:10DA4800F081F0B5B1FBF2FC0CFB1211B2FA82F3D3
:10DA58009A409940D3F1200630FA06F631439840AF
:10DA680000F036F8614628003200DA400023F0BDA5
:10DA7800F3B5B3FA83FC49085FEA300013FA0CF3F4
:10DA8800DCF1200432FA04F423430CB41A0000F049
:10DA98001FF80CBC33FA0CF3DCF11F0C35FA0CF54B
:10DAA80018BF6D1E03BCA5FB026705FB0377801B2F
:10DAB800B941904271EB030C05D3821A71EB030351
:10DAC800681C0021F0BD02000B0028000021F0BDF9
:10DAD800940D4FF6C2752D02B5FBF4F4D60A761CE8
:10DAE80004FB04F5A5FB0656F64306EB0416550899
:10DAF80032BF002777086D1C05FB1677A6FB074782
:10DB08007F0807EBC63714001500E7FB02457F1BAB
:10DB18004D1C0400E7FB014505FB1206A64284BF25
:0EDB28006D1EB618964224BF6D1CB61A7047CB
:10DB3600443A5C50726F6A656B74655C65637353D7
:10DB46006D61727450726F5C7472756E6B5C667721
:10DB56005F673437337263745C44726976657273D7
:10DB66005C53544D3332473478785F48414C5F44B8
:10DB760072697665725C5372635C73746D33326777
:10DB86003478785F68616C5F6164635F65782E6383
:01DB9600008E
:10DB9700443A5C50726F6A656B74655C6563735376
:10DBA7006D61727450726F5C7472756E6B5C6677C0
:10DBB7005F673437337263745C4472697665727376
:10DBC7005C53544D3332473478785F48414C5F4457
:10DBD70072697665725C5372635C73746D33326716
:10DBE7003478785F68616C5F636F727465782E63F1
:01DBF700002D
:10DBF8002DE9F04F89B01546894682460020CAF8BB
:10DC080000000DF10E0819F8011B252906D000297E
:10DC180000F04F82504600F067FBF4E72C460027DF
:10DC28004A4619F8010BA0F12003102B0DD88021CA
:10DC3800DFE803F0091B1B191B1B1B151B1B3018E6
:10DC48001B101B1B120040210DE05E280DD14FF464
:10DC5800805108E0102106E04FF4007103E04FF412
:10DC6800004100E020210F43DAE7A0F13001C9B2FA
:10DC780009294FF000010BD801EB810100EB4101AC
:10DC880019F8010BA0F13002D2B230390A2AF3D3C5
:10DC980025460CE0254655F8040B010048BF4142D3
:10DCA800102303EAD060074302F1020950782E28B6
:10DCB8000BD14A4612F8010B2A2809D155F804BBA2
:10DCC80099F8010009F1020218E04FF0000B1EE07C
:10DCD800A0F13003DBB2092B4FF0000B14D80BEB8B
:10DCE8008B0300EB430312F8010BA0F130095FFA34
:10DCF80089F9B9F10A0FA3F1300BF0D3BBF1000F8A
:10DD080004D447F4807701E047F480779146A0F186
:10DD18006802D3B2D20142EA5302D2B2092A22D807
:10DD2800DFE802F0050E122121210F21210F4A46BA
:10DD380012F8010B682812D199F8010008370BE096
:10DD4800023719F8010B0EE04A4612F8010B6C284D
:10DD580007D199F80100023709F1020903E00437F5
:10DD680000E001379146622821EAE17620DDA0F142
:10DD7800630115293FF647AFDFE811F038001700B7
:10DD880016001600160016001700160016001600DA
:10DD980016009A0044000601160016002900160015
:10DDA8004E001600160022002DE747F4804737E0A2
:10DDB800252800F08A80582840F08C8147F40057C5
:10DDC80043F2580278281ED143F278021BE00195ED
:10DDD8002D68002D04BF4EF69E25C0F60005F805F7
:10DDE800284600F1458100F0D1FB44E12C78013E42
:10DDF80050463946324600F0C9FA5046214600F0EE
:10DE080073FA4AE13022390602EAE1710291F90512
:10DE180008D527F4007705E0F90548BF27F400770F
:10DE28000021029179044FEA8771009604D40029F1
:10DE380009D4291D00240CE0002913D4294651F8DF
:10DE4800045BEC1714E0E91D21F0070505F1080152
:10DE58006C687A072D6814D417F0080F13D00024C3
:10DE6800EDB210E0E91D21F007014C6851F8085B9C
:10DE78000191790709D439070AD545F3C0146DB261
:10DE880006E0ADB20024019126E045F3C0342DB27E
:10DE9800002C07DBB9061DD47906029A48BF202258
:10DEA800029219E000216D4261EB04042D2112E079
:10DEB80055F8040B3907DAF8001000F1F880BA07B2
:10DEC80052BF0160002206C09DE65046252100F0A1
:10DED8000BFA98E62B210291F90548BF27F4007741
:10DEE800F90558BF4FF0010B00266E2821DD6F3869
:10DEF800092800F27980DFE800F005567777777710
:10DF08002277775655EA04006ED0E80840EA447054
:10DF1800062262F3DF0508F80650013650EAD401FC
:10DF28004FEAD4044FEAD001054641EA4470F0D1E3
:10DF38005AE0582837D0642818BF692854D155EAC0
:10DF4800040051D0380407D506F00300032802BFA7
:10DF58002C2008F806000136284621460A2200230C
:10DF6800FFF74EFD00EB8002A5EB4202D5F1090355
:10DF78000023A34142F0300208F8062006F101060A
:10DF880005460C46DED32FE02846009650F8045B81
:10DF980001903806232101EAE070029047F4807767
:10DFA80000244FF0080B002655EA04001CD04FF25D
:10DFB8002000C0F60000B9045CBF4FF23000C0F684
:10DFC8000000290941EA047105F00F020D46825C40
:10DFD80008F80620013651EA14114FEA14144FEAE2
:10DFE800151141EA0471EFD1ABEB060020EAE07BA2
:10DFF80006EB0B000099029D0C1A4FF0FF30FF2D25
:10E0080088BF0138002D18BF0444B80505D4504610
:10E018003946224600F0BAF90024FF2D04D9290A0E
:10E02800504600F061F900E01DB15046294600F065
:10E038005BF950463946224600F0A8F9504630218F
:10E048005A4600F093F9012E08DB751E504618F861
:10E05800051000F049F9012E2E46F6D8F806019D64
:10E068007FF5D1AD50462021224600F07FF9CAE560
:10E07800594600F0A1FA044627F40077361A5046AC
:10E088003946324600F082F934B115F8011B504682
:10E0980000F02AF9013CF8D1019D0435F8067FF516
:10E0A800B2AD50462021324600F060F9ABE5017070
:10E0B800A9E5DAF80C0028B1DAE9001291423CBF70
:10E0C800002242545046FDF790FDDAF8000009B0EE
:10E0D800BDE8F08F00287FF496AD5046FDF785FD2A
:06E0E8004FF0FF30F3E7EA
:10E0EE00443A5C50726F6A656B74655C656373531A
:10E0FE006D61727450726F5C7472756E6B5C667764
:10E10E005F673437337263745C4472697665727319
:10E11E005C53544D3332473478785F48414C5F44FA
:10E12E0072697665725C5372635C73746D333267B9
:10E13E003478785F68616C5F6372635F65782E63B5
:01E14E0000D0
:10E14F00443A5C50726F6A656B74655C65637353B8
:10E15F006D61727450726F5C7472756E6B5C667702
:10E16F005F673437337263745C44726976657273B8
:10E17F005C53544D3332473478785F48414C5F4499
:10E18F0072697665725C5372635C73746D33326758
:10E19F003478785F68616C5F6932635F65782E638E
:01E1AF00006F
:10E1B0004AB1884207D007D28018891852428B5C36
:10E1C0008354521CFBD17047521E8B5C8354FBD18D
:02E1D000704796
:10E1D200443A5C50726F6A656B74655C6563735335
:10E1E2006D61727450726F5C7472756E6B5C66777F
:10E1F2005F673437337263745C4472697665727335
:10E202005C53544D3332473478785F48414C5F4415
:10E2120072697665725C5372635C73746D333267D4
:10E222003478785F68616C5F7077725F65782E63AF
:01E2320000EB
:10E23300443A5C50726F6A656B74655C65637353D3
:10E243006D61727450726F5C7472756E6B5C66771D
:10E253005F673437337263745C44726976657273D3
:10E263005C53544D3332473478785F48414C5F44B4
:10E2730072697665725C5372635C73746D33326773
:10E283003478785F68616C5F7263635F65782E636F
:01E29300008A
:10E29400010002000400060008000A000C0010003F
:08E2A400200040008000000191
:10E2AC0051EC102BC1F30A53002B1CBF40F2FF7C26
:10E2BC00634514D01844604506DB0020C7F6F070A7
:10E2CC0060F31E01002208E00028C7BF6FF31E5147
:10E2DC0041EA005101F00041002241EC102B704743
:04E2EC00F4F730B95A
:10E2F00010B582B0044600698DF8071078B1D4E9F2
:10E3000000239A4231D26269531C63618154D4E97B
:10E310000501884229D12046FDF76BFC25E0E06825
:10E3200050B1D4E9002C62451FD2531CB3EB0C034F
:10E3300018BF0B46835418E0A06858B1D4E9002CEC
:10E34000624512D2531CB3EB0C0318BFCBB240F89A
:10E3500022300AE0236A43B1D4E90001884204D2A2
:10E360000DF1070120460122984720680130206006
:04E3700002B010BD2A
:10E37400012A0CDBF8B514460D460646671E3046E6
:10E384002946FFF7B3FF012C3C46F7D8F8BD704788
:10E39400CB0606D43023890558BF20231946FFF73E
:04E3A400E7BF704718
:10E3A80070B514460D460646F8F7A6F901463046FC
:0CE3B8002A462346BDE8704000F000B883
:10E3C4002DE9F04F03AF8DB047F83C3C91460C4625
:10E3D400064600F05BF80546EB46073020F00700E0
:10E3E400ADEB0008C546A7F1380A504600212422A7
:10E3F400F8F754F947E908546FF0004047F8340C33
:10E404004BF64F40C0F6000047F8288C47E9060653
:10E414005046494657F83C2CFFF7ECFBDD46A7F184
:08E424000C04A546BDE8F08FD1
:10E42C0083B000B582B0CDE9031241F2747CC1F225
:10E43C00000C059303AA01920146DCF80000FFF7DB
:0CE44C00ADFF02B05DF804EB03B07047B8
:10E4580041F27871C1F2000141F27472C1F2000216
:10E468000968126841F27C73C1F20003411A1B6803
:10E4780018BF0121821A18BF01221140C01A18BF03
:08E488000120084040427047EA
:04E490004020704771
:10E4940040F6E410C1F2000003214EF61D52C0F60E
:10E4A40000020161416141F23631C1F20001826131
:10E4B400C1614FF480610162002181624162C162E5
:10E4C40041F23673C1F2000302664366102282668B
:10E4D4000167C1664EF60C52C0F600024167BFF3F5
:10E4E4005F8F531ADB7B435401311029F9D1BFF3F9
:04E4F4005F8F70477F
:10E4F8002DE9F04104468068E66815466268871B86
:10E508009019BD4206D22A46F8F794F8BFF35F8FF8
:10E5180035440CE088463A46F8F78CF8ED1B08EBD2
:10E52800070160682A46F8F785F8BFF35F8FE56052
:04E53800BDE8F081C9
:10E53C0070B500EB400040F6E413C1F2000303EBAE
:10E54C00C00303F11806D86A022818D00D461446E9
:10E55C00012807D020B93046FDF7CDFBA04207D2E9
:10E56C0000240AE03046FDF7C6FBA04238BF044643
:10E57C00304629462246FFF7B9FF204670BD30468B
:08E58C00BDE87040FDF7C3BBC0
:10E59400017889B14FF0013C0346194653F8042B26
:10E5A400CCFA52F2002AF8D092FAA2F2B2FA82F22B
:0CE5B40001EBD201081A704700207047EC
:10E5C00000291CBF0278002A01D10020704700B545
:10E5D0000429D0F800E0024609D34FF0013CCCFA00
:10E5E0005EF323B90439032952F804EFF7D84FF04A
:10E5F0000133C3FA5EF393FAA3F3B3FA83F3101A69
:0CE60000B1EBD30F88BFD908084400BD5F
:10E60C007F280BD84FF24002C0F600024EF686531C
:10E61C00C0F60003105C595C08407047002070473E
:0CE62C00A0F161011A2938BF20387047A6
:0CE63800A0F141011A2938BF20307047C2
:10E644007F280BD84FF24002C0F600024EF68653E4
:10E65400C0F60003105C595C084070470020704706
:0CE66400A0F161011A2938BF203870476E
:0CE67000A0F141011A2938BF203070478A
:0FE67C005465737420646562756720696F0D00C3
:10E68B00666163746F727920726573746F72652E35
:03E69B002E2E0020
:10E69E0043616E6E6F74206A756D7020696E2044D2
:0BE6AE0045425547206D6F6465210058
:0FE6B9006572726F722068616E646C65720D001D
:10E6C800466C61736820756E6C6F636B206572723F
:03E6D8006F72005E
:10E6DB00443A5C50726F6A656B74655C6563735327
:10E6EB006D61727450726F5C7472756E6B5C667771
:10E6FB005F673437337263745C4472697665727327
:10E70B005C53544D3332473478785F48414C5F4407
:10E71B0072697665725C5372635C73746D333267C6
:10E72B003478785F68616C5F666C6173685F65787D
:03E73B002E63004A
:10E73E00443A5C50726F6A656B74655C65637353C3
:10E74E006D61727450726F5C7472756E6B5C66770D
:10E75E005F673437337263745C44726976657273C3
:10E76E005C53544D3332473478785F48414C5F44A4
:10E77E0072697665725C5372635C73746D33326763
:0FE78E003478785F68616C5F6770696F2E630025
:10E79D00443A5C50726F6A656B74655C6563735364
:10E7AD006D61727450726F5C7472756E6B5C6677AE
:10E7BD005F673437337263745C4472697665727364
:10E7CD005C53544D3332473478785F48414C5F4445
:10E7DD0072697665725C5372635C73746D33326704
:0FE7ED003478785F68616C5F697764672E6300CA
:10E7FC00443A5C50726F6A656B74655C6563735305
:10E80C006D61727450726F5C7472756E6B5C66774E
:10E81C005F673437337263745C4472697665727304
:10E82C005C53544D3332473478785F48414C5F44E5
:10E83C0072697665725C5372635C73746D333267A4
:0FE84C003478785F68616C5F756172742E630059
:0FE85B0049205265666572656E7A3D25660A0032
:0BE86A00547368756E743D25660A004B
:10E875002D2D2D204761696E2044726966742043F1
:07E88500414C202D2D2D0058
:0FE88C0041637475616C20543D256620430A007A
:10E89B0041637574616C20493D2566204128776979
:10E8AB0074686F7574206761696E2074656D702074
:10E8BB00647269667420636F7272656374696F6EDC
:03E8CB00290A0017
:10E8CE004B6F7272656B74757266616B746F723DAD
:10E8DE002566205B2031202F2043656C736975738C
:03E8EE005D0A00C0
:10E8F1004552524F52204144535F313236305F53BB
:0BE9010065744461746152617465002C
:10E90C004552524F52204144535F313236305F539F
:0BE91C00657443686F704D6F64650008
:10E9270054696D652025643A20456D7074792065BA
:10E9370076656E742831292C20636E3D25642C2062
:10E9470063613D25642C2074446973636861726751
:10E95700653D25642C20753D25642C20693D256483
:03E967000D0A0096
:10E96A0054696D652025643A20456D707479206577
:10E97A0076656E742832292C20636E3D25642C201E
:10E98A0063613D25642C207444697363686172670E
:10E99A00653D25642C20753D25642C20693D256440
:03E9AA000D0A0053
:10E9AD00454550524F4D20776173206368616E6706
:10E9BD00656421205765206E65656420746F207035
:10E9CD00726573657276652063616C6962726174DC
:10E9DD00696F6E20616E642073657474696E677300
:07E9ED002064617461210048
:10E9F400454550524F4D20464143544F52592052A1
:0FEA04004553544F52452F55504441544521001E
:10EA130055617274204572726F7220626569206E4F
:10EA230065757374617274206E61636820466568EE
:07EA33006C6572200A0D0062
:10EA3A004F5554505554535F4C56505F5348554E9A
:10EA4A00545F554E44455254454D504552415455D4
:03EA5A0052450022
:10EA5D004F5554505554535F4F56505F5348554E74
:10EA6D00545F554E44455254454D504552415455B1
:03EA7D00524500FF
:0BEA8000486561746572206F6E0D0028
:10EA8B00415558206F6E2028534F43204D6F6465BE
:03EA9B00290D0042
:07EA9E00286E756C6C290065
:10EAA5004A616E7561727900466562727561727947
:10EAB500004D6172636800417072696C004D617947
:10EAC500004A756E65004A756C7900417567757306
:10EAD500740053657074656D626572004F63746F81
:10EAE500626572004E6F76656D626572004465639E
:07EAF500656D62657200000F
:07EAFC00414D00504D0000E8
:0FEB0300256120256220256520255420255900F5
:10EB1200443A5C50726F6A656B74655C65637353EB
:10EB22006D61727450726F5C7472756E6B5C667735
:10EB32005F673437337263745C44726976657273EB
:10EB42005C53544D3332473478785F48414C5F44CC
:10EB520072697665725C5372635C73746D3332678B
:10EB62003478785F68616C5F7274635F65782E6376
:01EB720000A2
:10EB7300492028776974686F757420636F6D7065B9
:0DEB83006E736174696F6E293D25660A008E
:10EB90004144535F313236305F426174746572793B
:10EBA00043757272656E744761696E43616C696228
:10EBB000726174696F6E53746172743A2045525277
:10EBC0004F5220494E2043414C4942524154494FF3
:10EBD0004E2C204E4F205245464552454E4345202F
:09EBE00043555252454E542100E8
:10EBE9004E6F726D616C20737461727420776974F1
:10EBF900686F757420454550524F4D206368616EAA
:0DEC0900676573206465746563746564005D
:10EC1600454550524F4D2046554C4C205245535475
:05EC26004F52452100E2
:10EC2B00454550524F4D2053544F524520434F4E64
:05EC3B004649472100DD
:10EC40004D4220444D41204572726F7221200A0DC1
:01EC500000C3
:10EC51004D42204F5245204572726F7221200A0D9C
:01EC610000B2
:10EC62004552524F52205561727420494E49540DFB
:01EC720000A1
:10EC73004F5554505554535F4C56505F4348495079
:10EC83005F4F56455254454D504552415455524598
:01EC93000080
:10EC94004F5554505554535F4C56505F4241545451
:10ECA4004552595F554E444552564F4C5441474581
:01ECB400005F
:10ECB5004F5554505554535F4F56505F4348495034
:10ECC5005F554E444554454D504552415455524566
:01ECD500003E
:10ECD6004F5554505554535F4F56505F4348495013
:10ECE6005F4F56455254454D504552415455524535
:01ECF600001D
:10ECF700415558206F6E2028416C61726D204D6F11
:05ED07006465290D0008
:10ED0C000000000000005454522052454747455320
:01ED1C0000F6
:09ED1D005465726D696E616C00B1
:09ED2600256D2F25642F257900CD
:09ED2F0025483A254D3A25530010
:10ED380053756E004D6F6E0054756500576564001D
:0DED48005468750046726900536174000044
:10ED55004A616E00466562004D6172004170720045
:10ED65004D6179004A756E004A756C004175670002
:10ED7500536570004F6374004E6F76004465630001
:01ED8500008D
:0DED86000007032004170201085710408009
:10ED94002067000820670008206700082067000833
:04EDA40020670008DC
:04EDA800FDD300088F
:10EDAC00554E4B4E4F574E20434F4D4D414E440008
:10EDBC00466C617368204F7074696F6E627974650C
:0CEDCC002070726F6772616D6D656400ED
:10EDD800537461727420656E61626C65207265613E
:10EDE800646F75742070726F74656374696F6E00F8
:10EDF8002E2E2E466C61736820756E6C6F636B00E7
:10EE0800466C617368204F7074696F6E62797465BF
:08EE1800206C6F636B65640060
:10EE20002E2E2E456E61626C65206C6F636B2070B8
:10EE3000726F636573732066696E697368656400D9
:10EE4000443A5C50726F6A656B74655C65637353BA
:10EE50006D61727450726F5C7472756E6B5C667704
:10EE60005F673437337263745C44726976657273BA
:10EE70005C53544D3332473478785F48414C5F449B
:10EE800072697665725C5372635C73746D3332675A
:10EE90003478785F68616C5F666463616E2E6300CE
:08EEA00001010103070100005C
:08EEA800080402040801010145
:10EEB0004B6F7272656B74757266616B746F723DC5
:04EEC00025660A00B9
:10EEC4002D2D2D204761696E20447269667420439C
:0CEED400414C20454E4445202D2D2D00C2
:10EEE0004552524F52204144535F313236305F53C6
:10EEF0006574496E7465726E616C526566657265A3
:04EF00006E636500D7
:10EF040054696D652025643A2042617474657269A0
:10EF1400652046756C6C206576656E74206D41685D
:10EF24004361726765643D25642C20744368617293
:10EF340067653D25642C2063656641683D25642C26
:10EF44002063656657683D25642C20753D25642C37
:08EF540020693D25640D0A004F
:0CEF5C0057726974696E6720534E2100E3
:10EF68004D42204645204572726F7221200A0D00DD
:10EF78004D42205045204572726F7221200A0D00C3
:10EF88004D42204E45204572726F7221200A0D00B5
:10EF98004F5554505554535F4C56505F4F56455239
:08EFA80043555252454E54003E
:10EFB0004F5554505554535F4F56505F4F5645521E
:08EFC00043555252454E540026
:10EFC8004F5554505554535F4F56505F4241545417
:10EFD8004552595F4F564552564F4C54414745008C
:0CEFE800486561746572206F66660D005C
:10EFF400415558206F66662028534F43204D6F6457
:04F0040065290D006D
:10F0080000000000000000000102030406070809D0
:08F018000000000001020304E6
:10F02000303132333435363738394142434445463E
:10F03000303132333435363738396162636465666E
:10F040002020202020202020206828282828202058
:10F0500020202020202020202020202020202020B0
:10F060004810101010101010101010101010101068
:10F070008484848484848484848410101010101008
:10F080001081818181818101010101010101010161
:10F090000101010101010101010101101010101015
:10F0A0001082828282828202020202020202020232
:10F0B00002020202020202020202021010101020DA
:10F0C00000B506480649884205D00268043003B4FA
:10F0D000904703BCF7E708BC18470000A8ED0008FC
:04F0E000ACED00088B
:10F0E40081F10008000000101D13000081F10008E8
:10F0F4001E1300100300000081F100082213001009
:10F104000300000081F10008261300102004000011
:10F1140081F10008841700100400000081F1000848
:10F12400000000205C03000093F100088817001021
:10F1340054F1000814000000A7F100084C17001057
:10F1440068F1000838000000C1F000089B63000863
:10F15400206700082067000820670008206700086F
:10F1640020670008FFFFFE01FFEE100144C41210E7
:0CF17400C8121094CC121024F40000000B
:10F18000206861680834002200E04254491EFCD522
:02F190007047C6
:10F1920020686168A2680C3401E08B5C8354521EC3
:04F1A200FBD57047E2
:10F1A60020686168A2680C340B78491C0826002583
:10F1B6005B0801D20D78491C0570401C521E02D016
:08F1C600761EF4D1F0E770475A
:04000005080063A5E7
:00000001FF
